:020000040800F2
:1000000000000110B5B00308D1890308190F0108D9
:10001000B9B10308B9B10308B9B103080000000081
:10002000000000000000000000000000199003081C
:100030001590030800000000119003081DC9000876
:10004000B9B10308B9B10308B9B10308B9B10308DC
:10005000B9B10308B9B10308EDD4000819D60008F6
:10006000DDD50008A1D5000865D500085DBC0008F5
:100070004DBC00083DBC00082DBC00081DBC00089C
:1000800009BC0008F5BB0008B9B10308B9B1030801
:10009000B9B10308B9B10308B9B1030829D50008FB
:1000A00035190108B9B10308B9B10308B9B103089A
:1000B0008519010875190108B9B10308B9B1030818
:1000C000B9B10308B9B10308B9B10308B9B103085C
:1000D000B9B1030889CA0008B9B10308EDC900081D
:1000E000B1D40008B9B1030835900308B9B10308C9
:1000F00045190108B9B1030855190108E1BB000809
:10010000B9B10308B9B1030865190108B9B1030809
:10011000B9B10308B9B10308C1F80108A5F801088D
:10012000CDBB0008B9BB0008A5BB000891BB000807
:100130007DBB0008B9B10308B9B10308B9B1030820
:10014000B9B10308B9B10308B9B10308D5890308E7
:1001500069BB000855BB000841BB000851C9000835
:10016000B9B10308B9B10308B9B10308B9B10308BB
:10017000B9B10308B9B10308B9B10308B9B10308AB
:08018000B9B10308B9B103088D
:1001880016000800EC240020F424002000000000E1
:100198001006000827000400D0280020D8290020D5
:1001A800000000001806000801010400303000209B
:1001B800AC3E00200000000000000000080209001A
:1001C800263E0020B03E002000000000B5BE00081A
:1001D80002000C00303E0020BC3E00200000000061
:1001E80000000000F7010600203E0020C83E002065
:1001F800000000001C0600080A020A00C0300020A7
:10020800D03E002000000000220600080312330040
:100218006741002034410020000000002C0600083F
:1002280025005A0080400020DA400020000000002D
:1002380000000000F6110C00744000206840002007
:100248000000000060060008012008006442002049
:10025800B0420020000000006C0600081A000800E8
:100268004C420020B842002000000000740600083C
:1002780015007000F8440020484A002000000000E3
:100288000000000003000100F4440020B84A0020E8
:1002980000000000000000002A0060000444002064
:1002A800BC4A002000000000193B020809020100B6
:1002B800AC4B00208C580020000000007C06000891
:1002C80005000600AA5A0020745B00200000000008
:1002D800800600080C002400725A00207C5B002075
:1002E8000000000029EE01080E20EA006A590020EB
:1002F800A05B002000000000D91C020813000400C5
:10030800C05A00208C5C002000000000880600080D
:10031800020103004F590020905C002000000000FB
:1003280051EE0108F511620094580020945C0020F9
:1003380000000000A582000829005000B05F0020DE
:10034800BC63002000000000000000001400020050
:10035800AC5F00200C640020000000008C06000840
:100368000102050034680020A46D00200000000090
:1003780049B902080002050010640020AC6D002095
:1003880000000000000000001E0004002C66002091
:10039800B46D0020000000008E06000822000C004A
:1003A800246D0020B86D00200000000092060008AF
:1003B800FB010100147B0020487B002000000000A6
:1003C80021FD0008FC010900E07900204C7B002099
:1003D80000000000EDFC00080A101200B4790020AB
:1003E800587B0020000000009E060008060016004A
:1003F800847600206C7B002000000000F91C0208B5
:1004080034001000F0740020847B002000000000FD
:10041800413B02080D003400BC740020947B00208E
:100428000000000049B8010812100C00A074002058
:10043800C87B002000000000B00600080C02010084
:100448009C740020D47B002000000000BC0600083B
:1004580002020300B0740020D87B002000000000D6
:1004680000000000FA010200787C00207C7C00205B
:100478000000000079FD0008FD012400047C002034
:10048800807C00200000000035BE0008FE01080046
:10049800F07B0020A47C0020000000005DFD000827
:1004A8001F000E00F07D0020107E002000000000DC
:1004B800BE06000805020100D87D0020207E00202D
:1004C80000000000CC060008030106006A7D002039
:1004D800247E002000000000CE0600081B00F40067
:1004E800347E0020F88000200000000059B902087E
:1004F80026000E00FC810020EC8100200000000096
:10050800F112030810000300888400208C84002066
:1005180000000000D406000828000C007C8400209D
:100528009084002000000000D80600082300100076
:100538006C8400209C84002000000000859B020839
:100548001900050064840020AC840020000000002D
:10055800E4060008F811010060840020B48400203B
:1005680000000000EA060008000104005C84002086
:10057800B884002000000000EC0600082F001100DD
:1005880048840020BC84002000000000F006000819
:100598000400800014A00020A4A100200000000096
:1005A80000000000F90104002095002024A200208A
:1005B80000000000A5BE000818102C00F0940020D0
:1005C80028A2002000000000BD5503082C001000E0
:1005D80028A4002018A400200000000031530308BC
:1005E8002B0024005CA4002038A400200000000098
:1005F800015303080B201000D4A600200CA70020EC
:080608000000000002070008D9
:10061000C409000019012828200300001800010067
:10062000000000004A01B400D601000000000000F4
:1006300000000000000000000000000000000000BA
:1006400000000000000000000000000000000000AA
:100650000000000000000000000000000000010099
:10066000000000000000000000000000E80364003B
:10067000040A00017E05EA05B405320013000000FB
:100680002000030001000000080004000300000037
:100690000100C800141E010064002C012800003075
:1006A0000100005A0000000090012C01C800640005
:1006B0000000000100054B495749000001000000FF
:1006C000000000000100000000050000000004011F
:1006D0000100000000010500000000010000000012
:1006E000000000000000280100000400BC01000020
:1006F00000000000000000000000000000000000FA
:1007000000002B21231E64010200000001000A01E9
:020710002900BE
:10071200010100005001000007000000020000007B
:10072200000000000000000001020304060708099F
:1007320001010000D01204084C4B04080000000024
:1007420000000000E0120408E812040800000000A3
:1007520001200000EC120408F4110408000000005B
:1007620001400000F41204083826040800000000CA
:1007720001200000001304080C130408000000000C
:100782000400000010130408744204080000000072
:10079200040000001C130408C03D0408000000000F
:1007A20001000000020100000000803F0000803FC5
:1007B200FF0000006D880308258803087587030879
:1007C2000000000065840308E985030869860308C0
:1007D200518503080000000000000000598403084E
:1007E2003D840308398403083584030829840308F7
:1007F20025840308318403082D8403084D840308EB
:1008020041840308298503083D85030815850308EB
:1008120001850308ED84030804E7030805080400C2
:1008220000000000E801040884010408F0E603085F
:100832000000000030E7030805080A00000000007D
:10084200E8010408840104080C0204080000000006
:10085200FFFFFFFF0000803F0100000001010100D7
:10086200F04104080F000000497202080000000075
:1008720000000000D0020020B44104080000000083
:100882000000000000000000000000004C4B0408C3
:1008920000000000000000006C07002004000000BF
:1008A200404104080D000000718B02084807002037
:1008B20000000000BC4404080D000000418B020847
:1008C2003C07002000000000D4410408080000009A
:1008D200000000003007002004000000C4410408AA
:1008E2000D000000FD8A020824070020000000001D
:1008F2005840040803000000B18D02080C070020D4
:1009020000000000CC41040803000000B18D020881
:10091200F4060020000000005C4004080100000012
:1009220000000000000000000000000000000000C5
:100932000E000000000000000000000000000000A7
:10094200B4410408000000000000000000000000A4
:10095200000000004C4B04080000000000000000F2
:100962006C07002004000000E440040803000000BB
:100972004D780208DC06002008000000C44104088B
:100982000D000000FD8A020824070020000000007C
:100992005840040803000000B18D02080C07002033
:1009A20000000000CC41040803000000B18D0208E1
:1009B200F4060020000000005C4004080100000072
:1009C2000000000000000000000000000000000025
:1009D2000E00000000000000000000000000000007
:1009E200DC410408000000000000000000000000DC
:1009F200000000004C4B0408000000000000000052
:100A02006C07002004000000EC4004080300000012
:100A1200B18D020854070020000000005C40040869
:100A220001000000000000000000000000000000C3
:100A3200000000000E0000000000000000000000A6
:100A4200000000002D202D2D202D2D2D2D202D2DAF
:100A52002D2D00000000000000000000000000003A
:100A620000000000464B002088130C170100000014
:100A7200484B002088130C17000000003040040887
:100A82000000000000000000000000000000000064
:100A9200404004080800000000000000600300203D
:100AA200040000004C4004080800000000000000A0
:100AB2005403002000000000584004080400000015
:100AC2008578020800000000000000005C40040875
:100AD2000100000000000000000000000000000013
:100AE200000000000E0000000000000000000000F6
:100AF20000000000444B002088130C170100000086
:100B0200424B002088130C17000000009440040898
:100B12000F000000A17202080000000000000000A7
:100B22006C030020A34B002001000000A801040870
:100B3200404B002001000000B4010408D47D0020D5
:100B420002000000BC010408DAA00020000000003E
:100B520000000000D8A000200000000000000000FB
:100B6200D6A000200000000000000000D4A0002059
:100B72000000000000000000D2A0002000000000E1
:100B820000000000D0A000200000000000000000D3
:100B9200101E002000000000000000003F4B00205B
:100BA20002000000C80104089C4004080000000084
:100BB20000000000000000000000000040400408A7
:100BC2000800000000000000F00300200400000004
:100BD2004C4004080800000000000000E40300206C
:100BE200000000005840040804000000817202085E
:100BF20000000000000000005C400408010000004A
:100C020000000000000000000000000000000000E2
:100C12000E000000000000000000000000000000C4
:100C2200AC400408000000000000000000000000CA
:100C320000000000BC4004080D000000998A020870
:100C42002C04002004000000C84004080D0000002D
:100C5200C57202082004002004000000D4400408E9
:100C62000D000000618A0208140400200000000048
:100C7200E04004080300000069780208FC03002039
:100C820008000000EC40040803000000B18D0208D7
:100C920054070020000000005C400408010000002E
:100CA2000000000000000000000000000000000042
:100CB2000E00000000000000000000000000000024
:100CC200F4400408000000000000000000000000E2
:100CD20000000000FC40040804000000A1780208A3
:100CE20000000000000000005C4004080100000059
:100CF20000000000000000000000000000000000F2
:100D02000E000000000000000000000000000000D3
:100D1200484104080000000000000000000000003C
:100D2200000000002C3704080D0000000000000045
:100D32008C04002004000000584104080800000050
:100D42000000000080040020040000006441040848
:100D520008000000000000007404002004000000ED
:100D62006C41040808000000000000006804002034
:100D720004000000744104080800000000000000A4
:100D82005C040020040000007C410408080000000C
:100D92000000000050040020040000008441040808
:100DA20008000000000000004404002004000000CD
:100DB2008C410408080000000000000038040020F4
:100DC200040000005C400408010000000000000074
:100DD2000000000000000000000000000E00000003
:100DE2000000000000000000000000009441040820
:100DF2000F000000917202080000000000000000D5
:100E0200980400209C4104080F000000000000002C
:100E1200000000000000000010050020A4410408AA
:100E22000F000000000000000000000000000000B1
:100E3200B0050020A44B002004000000D4010408E7
:100E420088580020E0150C1700000000A14B00207C
:100E52000800000084010408A24B002005000000E5
:100E6200E8010408AC4104080F0000000000000083
:100E72000000000000000000000600202D202D2DA3
:100E8200202D2D2D2D202D2D2D00000000000000E5
:100E920000000000000000000000000020700020A0
:100EA200702D7200FC4904080F00000000000000D1
:100EB20000000000000000002C1B0020FFFFFFFFCD
:100EC200FA00000001000000010000005C4204087A
:100ED20064420408F440040800000000000000001E
:100EE200000000000000000044420408040000006A
:100EF200DF77020800000000000000005C400408E8
:100F020001000000000000000000000000000000DE
:100F1200000000000E0000000000000000000000C1
:100F2200000000006E7F00200100C40900000000E4
:100F32006C7F00200100C409000000006A7F0020CD
:100F42000100C40900000000687F00200100C409FC
:100F520000000000647F00200100C40900000000BE
:100F6200667F00200100C40900000000627F0020AB
:100F72000100C40900000000607F00200100C409D4
:100F820000000000005900200100C800010000001C
:100F9200FE5800203200307532000000FC5800205C
:100FA200055A0500F758002000FF0100FB580020F9
:100FB20001000000BC070020F958002002000000D8
:100FC20000020408F658002000FF0100FA58002031
:100FD20001000000BC070020F858002002000000B9
:100FE20000020408A84204080F00000000000000EC
:100FF2000000000000000000C4070020A87D0020BF
:101002009CFF2C01000000004E0100200A0000009D
:101012000C0204083C4B0020E0150C1700000000F5
:101022004D01002008000000840104084C0100204A
:1010320005000000E80104083E4B00200200000009
:1010420024020408B05A00200100FF7F01000000C2
:10105200A85A00200200000030020408585900205B
:10106200030000004002040857590020030000005A
:10107200400204085C5A00200000F4010100000054
:101082005A5A00200000F40101000000585A0020C2
:101092000000F40101000000565A00200000F40193
:1010A20001000000545A002000FF0100705A002085
:1010B200E803D0070A0000006E5A00200064010015
:1010C2000A0000006F5A0020006401000A000000BC
:1010D200685A0020006401000A0000006D5A0020D6
:1010E200006401000A0000006C5A00200064010044
:1010F2000A0000006B5A0020006401000A00000090
:10110200675A002000FF01000A000000665A002012
:1011120000FF01000A000000665900200000F401EF
:1011220001000000645900200000F40101000000E9
:10113200625900200000F401010000006059002003
:101142000000F40101000000635A002000C8010001
:10115200625A002000C80100615A002000C8010044
:10116200605A0020006401000A0000005F5A00205B
:1011720000FF01000A0000009F5A002000C8010081
:101182009E5A002000C801009D5A002000C801009C
:101192009C5A002000C801009B5A002000C8010090
:1011A2009A5A002000C80100995A002000C8010084
:1011B200985A002000C80100975A002000C8010078
:1011C200B04204080000000000000000000000001F
:1011D20000000000C04204080900000000000000F6
:1011E2006808002004000000C8420408090000004A
:1011F200000000005C080020040000005C480408B5
:101202000900000000000000500800200400000057
:10121200001104080900000000000000440800203A
:1012220004000000D0420408090000000000000091
:101232003808002004000000D84204080900000019
:10124200000000002C08002004000000E042040816
:101252000900000000000000200800200400000037
:10126200E842040809000000000000001408002001
:10127200040000005C4004080100000000000000BF
:101282000000000000000000000000000E0000004E
:10129200000000000000000000000000C04304083D
:1012A200000000000000000000000000000000003C
:1012B200EC11040807000000000000008C08002068
:1012C20000000000D04304080800000000000000F5
:1012D2008008002000000000DC4304080800000031
:1012E2000000000074080020000000005C400408B8
:1012F20001000000000000000000000000000000EB
:10130200000000000E0000000000000000000000CD
:1013120000000000E4430408000000000000000098
:101322000000000000000000F44304080D0000006B
:1013320000000000C808002000000000FC43040870
:101342000D00000000000000BC08002000000000AA
:10135200044404080700000000000000B408002054
:10136200000000000C4404080D0000000000000012
:10137200A808002000000000144404080D0000002A
:10138200000000009C080020000000001C4404082B
:101392000700000000000000940800200000000088
:1013A2005C40040801000000000000000000000092
:1013B20000000000000000000E000000000000001D
:1013C20000000000000000002444040800000000A7
:1013D200000000000000000000000000EC11040802
:1013E2000C00000000000000025900200000000074
:1013F200384404080C0000000000000004590020DA
:1014020000000000484404080C0000000000000036
:101412003A59002000000000584404080C00000063
:10142200000000002E590020000000006C44040857
:101432000C0000000000000006590020000000001F
:10144200784404080C000000000000000859002045
:1014520000000000804404080C00000000000000AE
:101462000A59002000000000944404080C00000007
:10147200000000000C590020000000009C440408F9
:101482000C000000000000000E59002000000000C7
:10149200A44404080C0000000000000010590020C1
:1014A20000000000B04404080C000000000000002E
:1014B20012590020000000008C3004080C000000CB
:1014C200000000001459002000000000B844040885
:1014D2000C0000000000000016590020000000006F
:1014E200C44404080C000000000000001859002049
:1014F20000000000041204080C00000000000000BC
:101502001A59002000000000D04404080C0000001A
:10151200000000001C59002000000000DC44040808
:101522000C000000000000001E5900200000000016
:10153200E84404080C0000000000000032590020BA
:1015420000000000F04404080C000000000000004D
:101552003059002000000000F84404080C0000008C
:10156200000000003E59002000000000044504086D
:101572000C000000000000004059002000000000A4
:10158200104504080C00000000000000465900202D
:1015920000000000201204080C00000000000000FF
:1015A2002059002000000000C44104080C00000083
:1015B2000000000028590020000000001C4504081B
:1015C2000C00000000000000225900200000000072
:1015D200284504080C0000000000000024590020E7
:1015E20000000000344504080C0000000000000068
:1015F20026590020000000003C4504080C000000B1
:10160200000000002A590020000000008C34040869
:101612000C0000000000000034590020000000000F
:10162200484504080C000000000000002C5900206E
:1016320000000000781104080C0000000000000007
:101642003C59002000000000544504080C00000032
:101652000000000036590020000000005C4504082C
:101662000C000000000000003859002000000000BB
:10167200644504080C0000000000000042590020EC
:10168200000000006C4504080C000000000000008F
:1016920044590020000000005C40040801000000E2
:1016A2000000000000000000000000000000000038
:1016B2000E0000000000000000000000000000001A
:1016C2007445040800000000000000000000000053
:1016D200000000008445040805000000000000002E
:1016E20056590020000000005C4004080100000080
:1016F20000000000000000000000000000000000E8
:101702000E000000000000000000000000000000C9
:101712008C450408000000000000000000000000EA
:10172200000000004C4B0408000000000000000014
:101732003403002004000000FC1004080D00000027
:101742002578020828090020000000004041040812
:101752000D000000157202081C09002000000000A4
:10176200BC4404080D000000E171020810090020C9
:1017720000000000D441040808000000000000003E
:101782000409002004000000C44104080D00000008
:10179200CD710208F80800200000000098450408F6
:1017A2000900000000000000EC0800200400000016
:1017B2005840040803000000B18D0208D40800203C
:1017C200000000005C40040801000000000000006E
:1017D2000000000000000000000000000E000000F9
:1017E200000000000000000000000000A045040806
:1017F20000000000000000000000000000000000E7
:10180200B04504080D00000000000000400900205F
:1018120000000000B84504080A00000000000000B3
:101822001C5B002000000000C44504080A00000000
:1018320000000000245B002000000000CC450408EA
:101842000A000000000000002C5B002000000000E5
:10185200D4450408080000000000000034090020FC
:1018620000000000DC45040804000000F58E0208B8
:1018720000000000000000005C40040801000000BD
:101882000000000000000000000000000000000056
:101892000E00000000000000000000000000000038
:1018A200E8450408000000000000000000000000FD
:1018B20000000000FC4504080D00000000000000CC
:1018C20058090020000000000C4604080400000033
:1018D200F58B020800000000000000001446040816
:1018E2000D000000000000004C0900200000000074
:1018F2002846040804000000D18B02080000000002
:10190200000000005C40040801000000000000002C
:101912000000000000000000000000000E000000B7
:101922000000000000000000000000003046040833
:1019320000000000000000000000000000000000A5
:10194200444604080700000000000000940900203B
:1019520000000000504604080800000000000000DB
:1019620088090020000000005C460408080000000E
:10197200000000007C090020000000006846040806
:1019820008000000000000007009002000000000B4
:1019920074460408080000000000000064090020EA
:1019A200000000005C40040801000000000000008C
:1019B2000000000000000000000000000E00000017
:1019C2000000000000000000000000008046040843
:1019D20000000000000000008F070020000000004F
:1019E2008C4604080B00000000000000FC090020E7
:1019F20000000000944604080B00000000000000F4
:101A0200F009002000000000A04604080B000000BE
:101A120000000000E409002000000000AC460408B9
:101A22000B00000000000000D809002000000000A8
:101A3200B84604080B00000000000000CC0900209A
:101A420000000000C44604080B0000000000000073
:101A5200C009002000000000CC4604080B00000072
:101A620000000000B409002000000000D84604086D
:101A72000B00000000000000A80900200000000088
:101A8200E446040808000000000000009C09002051
:101A9200000000005C40040801000000000000009B
:101AA2000000000000000000000000000E00000026
:101AB200000000000000000000000000F0460408E2
:101AC2000000000000000000000000000000000014
:101AD2000447040808000000000000002C0A00204F
:101AE2000000000010470408080000000000000089
:101AF200200A0020000000001C4704080800000023
:101B020000000000140A002000000000284704081A
:101B12000800000000000000080A00200000000089
:101B22005C4004080100000000000000000000000A
:101B320000000000000000000E0000000000000095
:101B42000000000000000000304704080000000010
:101B5200000000008C07002000000000404704083D
:101B62000B000000000000005C0A002000000000E2
:101B72004C4704080B00000000000000500A00203F
:101B820000000000584704080700000000000000A1
:101B9200480A002000000000644704080700000013
:101BA20000000000400A0020000000007047040806
:101BB2000700000000000000380A002000000000BA
:101BC2005C4004080100000000000000000000006A
:101BD20000000000000000000E00000000000000F5
:101BE20000000000000000007C4704080000000024
:101BF200000000008C070020000000008847040855
:101C02000700000000000000A80A002000000000F9
:101C1200904704080700000000000000A00A00200E
:101C220000000000984704080700000000000000C0
:101C3200980A002000000000A047040807000000E6
:101C420000000000900A002000000000A8470408DD
:101C52000700000000000000880A002000000000C9
:101C6200B04704080700000000000000800A0020BE
:101C720000000000B8470408070000000000000050
:101C8200780A002000000000C04704080700000096
:101C920000000000700A002000000000C84704088D
:101CA2000700000000000000680A00200000000099
:101CB2005C40040801000000000000000000000079
:101CC20000000000000000000E0000000000000004
:101CD2000000000000000000D04704080F000000D0
:101CE200000000004D87020800000000B00A00203A
:101CF20054590020170000005002040853590020D4
:101D02000A3201005259002001FA01004E59002006
:101D120000C801004C590020E803D0070100000070
:101D22004B495749463400009258002000030100F5
:101D32009158002000030100D84704080F0000005A
:101D4200718602084D860208000000008C0B0020FC
:101D5200E44704080F0000000D860208C58502084A
:101D620000000000040C0020F04704080F000000EF
:101D7200AD8602089586020800000000B80C00201B
:101D8200FC4704080F0000006387020800000000FF
:101D9200A18B0208B00F0020044804080F000000C5
:101DA2002F71020800000000000000000010002057
:101DB2000C4804080F000000D58E0208B189020801
:101DC200AD890208DC100020144804080F0000004E
:101DD2008987020800000000000000009011002026
:101DE2001C4804080F00000029880208F98702082D
:101DF200000000001C120020244804080F0000000C
:101E0200A5880208E988020800000000BC12002030
:101E1200645A002001030100304804080F0000004A
:101E2200C58702089D87020800000000AC1300204D
:101E3200384804080F00000059880208198C02086B
:101E42000000000038140020444804080F0000007D
:101E520015890208618C020800000000D8140020D5
:101E62005E5A0020010301004C48040800000000F3
:101E720000000000000000000000000058480408B4
:101E8200080000000000000004160020000000000E
:101E9200604804080700000000000000FC15002054
:101EA2000000000070480408070000000000000065
:101EB200F4150020000000007C4804080700000020
:101EC20000000000EC150020000000008848040813
:101ED2000D00000000000000E015002000000000DE
:101EE2009448040803000000B18D0208C8150020C0
:101EF200000000005C400408010000000000000037
:101F02000000000000000000000000000E000000C1
:101F12000000000000000000000000009C480408CF
:101F220000000000000000000000000000000000AF
:101F3200AC4804080A0000000000000088120408EF
:101F420000000000B44804080A000000000000007D
:101F52005412040800000000BC4804080A000000F3
:101F620000000000A05A002000000000C44804083D
:101F72000A0000000000000010160020000000000F
:101F82005C400408010000000000000000000000A6
:101F920000000000000000000E0000000000000031
:101FA2000000000000000000CC480408000000000F
:101FB200000000000000000000000000D8480408F3
:101FC20003000000B18D0208581600200000000036
:101FD200E847040803000000B18D02084016002003
:101FE20000000000DC47040803000000B18D020875
:101FF2002816002000000000E44804080500000044
:10200200000000009058002000000000EC48040886
:102012000700000000000000201600200000000061
:10202200F84804080700000000000000181600200D
:10203200000000005C4004080100000000000000F5
:102042000000000000000000000000000E00000080
:102052000000000000000000000000000449040825
:10206200000000000000000000000000000000006E
:102072002C12040803000000B18D0208A0160020F3
:10208200000000001849040803000000B18D020896
:102092005001002000000000204904080300000055
:1020A200B18D0208881600200000000028490408AB
:1020B20003000000B18D020870160020000000002D
:1020C2005C40040801000000000000000000000065
:1020D20000000000000000000E00000000000000F0
:1020E2000000000000000000344904080000000065
:1020F2000000000000000000000000004049040849
:1021020007000000AD8C02085017002000000000FC
:102112003845040803000000B18D0208381700207A
:10212200000000004C49040803000000B18D0208C1
:10213200201700200000000054490408030000009A
:10214200B18D020808170020000000005C49040855
:1021520007000000918C0208001700200000000018
:102162005C41040803000000B18D0208E81600205B
:10217200000000006849040803000000B18D020855
:10218200D01600200000000074490408030000007B
:10219200B18D0208B8160020000000005C4004085F
:1021A200010000000000000000000000000000002C
:1021B200000000000E00000000000000000000000F
:1021C20000000000804904080F000000098702088F
:1021D200C58602080000000058170020884904083C
:1021E2000F000000818902080000000000000000CA
:1021F2000C180020944904080F000000A985020869
:102202008D85020800000000981800209C490408EF
:102212000F000000000000000000000000000000AD
:102222004C190020AC4904080F000000598902082B
:10223200C98C020800000000D8190020B449040823
:10224200000000000000000000000000000000008C
:10225200C049040803000000B18D0208141B0020CD
:1022620000000000A049040803000000B18D02082C
:10227200FC1A002000000000984904080300000036
:10228200B18D0208E41A002000000000C8490408C9
:1022920003000000B18D0208CC1A002000000000EB
:1022A200D449040803000000B18D0208B41A0020CA
:1022B20000000000DC49040802000000418F02080F
:1022C2000000000000000000E449040802000000D1
:1022D200418F02080100000000000000F0490408DC
:1022E20002000000418F020802000000000000000E
:1022F200000000000E0000000000000000000000CE
:102302000000000005A1020800000000000000001B
:102312000001010101000000E00108000000803F0F
:10232200080001000060024010600240000000004E
:10233200000B000000002000000000000000000070
:10234200006002402860024000000000060C00000D
:1023520000002000000000000000000000600240B9
:102362004060024000000000100D0000000020004C
:1023720000000000000000000060024058600240BF
:1023820000000000160E0000000020000000000007
:102392000000000000600240706002400000000087
:1023A200200F0000000020000000000000000000DC
:1023B2000060024088600240000000002610000019
:1023C2000000200000000000000000000060024049
:1023D200A060024000000000301100000000200058
:1023E200000000000000000000600240B8600240EF
:1023F20000000000362F0000000020000000000056
:10240200000000000064024010640240000000006E
:102412000038000000004000000000000000000042
:1024220000640240286402400000000006390000F7
:1024320000004000000000000000000000640240B4
:102442004064024000000000103A0000000040001A
:1024520000000000000000000064024058640240D6
:1024620000000000163B00000000400000000000D9
:10247200000000000064024070640240000000009E
:10248200203C0000000040000000000000000000AE
:1024920000640240886402400000000026440000FC
:1024A2000000400000000000000000000064024044
:1024B200A06402400000000030450000000040001F
:1024C200000000000000000000640240B864024006
:1024D200000000003646000000004000000000003E
:1024E20000000000000000010000000000000000E9
:1024F2000000000000FFFF0000000000AA550300DA
:102502009FAA5505010000AA550701000001AA551E
:102512000B010000AA5509020000000001000000A2
:10252200C012000000000101FFFF0000B8340408DF
:10253200000000000000000065EE0108A086010016
:102542000400000000000000000000000000000085
:102552000000000000000000000000000000000079
:1025620038450408E0300408000000000147010873
:102572007D000000060000000000000000000000D6
:102582000000000000000000000000000000000049
:1025920000000000504B0408000000000000000092
:1025A20049980308E803000003000000000000004F
:1025B2000000000000000000000000000000000019
:1025C2000000000000000000584B0408000000005A
:1025D20000000000F91D020810270000030000009F
:1025E20000000000000000000000000000000000E9
:1025F200000000000000000000000000B0430408DA
:1026020000000000C1510308E1950108204E0000BE
:1026120005000000000000000000000000000000B3
:1026220000000000000000000000000000000000A8
:102632002C36040800000000000000000593030887
:102642001027000001000000000000000000000050
:102652000000000000000000000000000000000078
:1026620000000000644B04080000000000000000AD
:10267200B9FC0008E80300000500000000000000AB
:102682000000000000000000000000000000000048
:102692000000000000000000704B04080000000071
:1026A200000000001DF10108204E000003000000A0
:1026B2000000000000000000000000000000000018
:1026C200000000000000000000000000804B040831
:1026D200000000000000000025EF0108204E00006D
:1026E20003000000000000000000000000000000E5
:1026F20000000000000000000000000000000000D8
:10270200904B0408000000000000000095900308B0
:10271200400D030003000000000000000000000064
:1027220000000000000000000000000000000000A7
:10273200000000006C3504080000000000000000EA
:10274200D1CF0108102700000100000000000000A6
:102752000000000000000000000000000000000077
:102762000000000000000000FC300408000000002F
:102772000000000011D10208102700000300000031
:102782000000000000000000000000000000000047
:1027920000000000000000000000000034360408C1
:1027A2000000000000000000B51D0108A00F00009D
:1027B2000100000000000000000000000000000016
:1027C2000000000000000000000000000000000007
:1027D200A04B04080000000000000000F9160308E6
:1027E20010270000010000000000000000000000AF
:1027F20000000000000000000000000000000000D7
:1028020000000000984904080000000000000000D9
:10281200C5A800081A4100000100000000000000E5
:1028220000000000000000000000000000000000A6
:1028320000000000000000009836040800000000BC
:10284200000000005D0203081027000001000000E4
:102852000000000000000000000000000000000076
:10286200000000000000000000000000D830040852
:1028720000000000000000008D9002081A410000D4
:102882000100000000000000000000000000000045
:102892000000000000000000000000000000000036
:1028A200AC4B0408000000000000000015A603085D
:1028B200400D0300000000000000000000000000C6
:1028C2000000000000000000000000000000000006
:1028D20000000000B44B04080000000000000000EB
:1028E200D1A50308400D0300000000000000000015
:1028F20000000000000000000000000000000000D6
:102902000000000000000000BC4B040800000000B2
:1029120000000000E5B80108A086010003000000E5
:1029220000000000000000000000000000000000A5
:1029320000000000000000000000000030303030D5
:102942002D30312D30315430303A30303A30300081
:10295200010100000000000001020304010203045F
:1029620006070809040309041201000202020040DA
:1029720083044057000201020301000009024300E0
:10298200020100C032090400000102020100052414
:10299200001001052401000104240202052406009E
:1029A20001070582030800FF09040100020A000072
:1029B20000070501024000000705810240000000F7
:1029C200FF0000005589030895860308F56B03088C
:1029D200A984030801890308B9840308D58403087C
:1029E20099840308898403080000000000000000A5
:1029F2004300000000000000000000000000000092
:102A020000000000000000000000000000000000C4
:102A12004300000000000000000000000000000071
:102A220000000000000000000000000000000000A4
:102A32004300000000000000000000000000000051
:102A42000000000000000000000000000000000084
:102A52004300000000000000000000000000000031
:102A62000000000000000000000000000000000064
:102A72004300000000000000000000000000000011
:102A82000000000000000000000000000000000044
:102A920043000000000000000000000000000000F1
:102AA2000000000000000000000000000000000024
:102AB20043000000000000000000000000000000D1
:102AC2000000000000000000000000000000000004
:102AD20011B7030851B50308000000006350040851
:102AE2003F420408C93F0408C93F0408C93F04081B
:102AF200C93F0408C93F0408C93F0408C93F040884
:102B0200C93F0408C93F0408FFFFFFFFFFFFFFFFA3
:102B1200FFFFFFFFFFFF000001004153434949004F
:102B220000000000000000000000000000000000A3
:102B3200000000000000000000004153434949002A
:102B42000000000000000000000000000000000083
:102B520000000000000000000000000050240020DF
:102B62000000000000000000000000000000000063
:102B72000000000000000000000000000000000053
:102B82000000000000000000000000000000000043
:102B92000000000000000000000000000000000033
:102BA2000000000000000000000000000000000023
:102BB2000000000000000000000000000000000013
:042BC200010000000E
:10800000002870B51EDB0928044620DD012303EBA0
:1080100083035B00B0FBF3F2092AF8D87BB10E4E64
:10802000B4FBF3F00928CCBF57223022A6FB03E5AE
:10803000024403FB1044EB0801F8012BF0D10023AC
:108040000B7070BD2D230B7040420131DBE73030E7
:1080500001F8010BF3E700BFCDCCCCCC884230B4A3
:108060004FF001042ED301FB04F4B0FBF4F58D4274
:10807000F9D284B1AAB901E0B0FBF4F5092DCCBF67
:10808000572230222A4404FB150003F8012BB4FBCD
:10809000F1F4002CF0D100221A7030BC7047B0FB14
:1080A000F4F5092DCCBF372230222A4404FB1500F9
:1080B00003F8012BB4FBF1F4002CF0D100221A706C
:1080C00030BC70470546002AEBD1D7E703685A1C3D
:1080D00002601970704700BF2DE9F047089C2578B1
:1080E000002B804689460CBF4FF0200A4FF0300A23
:1080F000661C35B3002A29DD334601E0024698B1FB
:1081000013F8011B501E0029F8D1971E60B13D469F
:10811000013D51464046C8476B1C002BF8DC2578D2
:1081200027EAE770013055B1041B29464046C8478D
:10813000301916F8015B002DF7D1BDE8F087BDE8D6
:10814000F087002A04DC2846BDE8F0870020EBE732
:10815000571EDCE783684268D0ED037A00EB8301A9
:108160000133934281ED040A836004BF00238360DE
:1081700000EB830393ED047A036870EE277A9A424A
:10818000C0ED037A77EEC77AC0ED037A0CDA0133DB
:1081900007EE103AF8EEC76AB7EE007A87EEA60A45
:1081A000036030EE070A704707EE102AB8EEC77A70
:1081B00087EE870A704700BF90ED057A90ED004A80
:1081C000D0ED066AD0ED014AD0ED047A90ED035A65
:1081D000D0ED025AA4EE007AB0EE406AB0EE470A43
:1081E000B0EE667AA6EE247A67EEC07AA0EE457A03
:1081F000E6EE257A80ED057AC0ED067A704700BF7D
:10820000D0ED057A90ED013AD0ED003AD0ED064A76
:1082100090ED024A90ED077A90ED035A90ED086ACE
:10822000D0ED045AC0ED067AF0EE406A27EE830ADC
:10823000C0ED056AA3EEA60A80ED087AA4EE240A32
:10824000A5EE470AA5EEC60A80ED070A704700BFF3
:10825000D0ED007A90ED017A30EE670AE7EE007A11
:10826000B0EE670AC0ED007A704700BF704700BFEC
:108270000A44914214D030B40139551E41F2210212
:1082800011F8014F082380EA042004044CBF82EA5D
:1082900040004000013B80B2F7D18D42F0D130BCAC
:1082A000704700BFF0B540F6280340F62C0240F6B8
:1082B000360540F6210440F64D1140F66A1740F6A7
:1082C000E1060380428040F6791340F68112458131
:1082D000848140F6611540F6DA04C18140F633012D
:1082E0000782468240F6F70740F6A7168382C282CD
:1082F00040F6C71340F6E7120583448340F6411564
:1083000040F65914818340F64911C783068440F62C
:108310004C0740F601064384828440F6011340F680
:108320002112C584048540F6410540F62F1441858D
:1083300040F62E118785468640F60A1740F68816C5
:108340008386C28640F6C80340F652020586C4877B
:1083500040F68A0540F63714818740F61711A0F8D9
:10836000447006878380C380038140F6530CC28526
:1083700014234FF0013E4FF0011745874FF00126BF
:10838000A0F846200125A0F84040A0F842100B4C70
:108390000B49A0F848C02822C0F84AE0C0F84E7047
:1083A000C0F8526080F85B50C465C0F8561080F881
:1083B000612080F85A3080F86030F0BD000A010A70
:1083C000980864004FF480538382704750F8043C4F
:1083D000012280F84520103803B11847704700BFCC
:1083E000BFF34F8F0549064BCA6802F4E06213439E
:1083F000CB60BFF34F8F00BFFDE700BF00ED00E093
:108400000400FA0570B4037B04681F2B08D9203BD5
:108410002021626801FA03F31A421CD170BC704734
:108420002021226801FA03F31A42F7D04269144965
:10843000582000FB021251685689CD6808682968E7
:1084400021F001012960828992B222EA060282812A
:10845000A36070BC704742690949582000FB0212B2
:1084600051685689CD680868296821F001012960A2
:10847000828992B222EA06028281E36070BC704770
:10848000AC76002030B4094B1C786CB1084A00254A
:1084900002EBC404116893884D6288890832034353
:1084A0009BB2A2428B81F5D130BC70476C79002021
:1084B0007079002010B4037B01681F2B09D9203B81
:1084C00020224C6802FA03F31C4214D15DF8044BDD
:1084D000704720220C6802FA03F31C42F6D00C4AC3
:1084E00040680024147002685DF8044B22F0010219
:1084F00002608B607047064A40680024147002686E
:108500005DF8044B22F001020260CB60704700BFAF
:10851000377F002070B5044682B00830656A0623B4
:108520006A463B21A847A8B19DF804009DF8006069
:108530009DF801109DF802509DF803209DF805302C
:1085400041EA062143EA002342EA0522E18222832E
:108550006383012002B070BD2DE9F0410446164D41
:10856000084616460F4632F0C7F82A6802301168EE
:108570009072D4723B4610464F6922460221B8479A
:1085800028680E4B0268C472152181725769142144
:108590002246B847304632F0AFF8296816300D68E9
:1085A0008872CC7222466C6933460846A44616216E
:1085B000BDE8F041604700BFB42400201810040853
:1085C000014B186804F022BB78A7002038B5054697
:1085D00000BF084C2368986804F008FF2368294608
:1085E000586805F08FF82368986804F005FF00BF0D
:1085F00038BD00BF687C0020F0B5044690F85900F3
:1086000083B0002840F0AA806A4E3779002F43D00B
:1086100004F114054FF48071A06905F0ABF894F8EB
:1086200052201A21284603F059FC012004F07EF85C
:108630000421A06905F09EF828460623E56D6A46E8
:108640004321A847D8B19DF802609DF803309DF8FA
:1086500000509DF801109DF804009DF8052043EAA4
:1086600006231BB2E3875BB241EA052142EA0022FE
:108670000133A187A4F8402006D003B0F0BDB4F9BF
:108680003E305BB20133F8D194F93C300133F4D180
:10869000062003F0AFFDF0E704F114054FF48071FC
:1086A000A06905F067F880226B21284603F016FCCC
:1086B000962004F095F803226821284603F00EFC6A
:1086C000962004F08DF803226B21284603F006FC67
:1086D0000F2004F02BF810226A21284603F0FEFB3D
:1086E0000F2004F023F83A466C21284603F0F6FBED
:1086F0000F2004F01BF894F854201921284603F0A9
:10870000EDFB0F2004F012F818221B21284603F07D
:10871000E5FB0F2004F00AF810221C21284603F084
:10872000DDFB0F2004F002F810223721284603F069
:10873000D5FB0F2003F0FAFF01223821284603F071
:10874000CDFB0F2003F0F2FF0421A06905F012F821
:10875000012003F0EBFF012333715BE704F0FCFB26
:108760000546D8B1202300218371C17104F086FD34
:108770002146114B41F8103F284631F041FDAB88AE
:10878000B3FA83F3C3F11F03012212FA03F33FF498
:108790003BAF0A490A6813430B6035E7014604F012
:1087A0006DFD2146044B41F8103F284631F028FD6D
:1087B0002AE700BFB4240020CD830008003C01401C
:1087C000F8B5057B466903681F2D29D9A5F120045A
:1087D0005F682021A1400F422A4613D01022A240F8
:1087E000D960DA605A68E240D10703D5012202FA63
:1087F00004F4DC600446304604F094F9227B2368DC
:108800001F2A20D9A2F1200008215A688140114274
:1088100000D0D9600422596882400A4221D1F8BDB3
:1088200020211C68A9400C422A460CD01022AA40E4
:1088300099609A601A68EA40D207DBD5012202FAF1
:1088400005F59D60D6E7082118689140014200D0E7
:1088500099600421186801FA02F2024203D09A607A
:10886000F8BDDA60F8BDF8BD70B582B0044669465F
:10887000143031F033FDB0B19DF805009DF8016072
:108880009DF802109DF803509DF804209DF80630D5
:1088900041EA062143EA002342EA0522A187E28752
:1088A000A4F84030012002B070BDF8B5174D2B7808
:1088B000A32B28D16B78BE2B25D1022229464FF657
:1088C000FF70FFF7D5FC124FAC1C22884AB1A618E6
:1088D000BE4218D2052A16D92146FFF7C9FC3446F4
:1088E000F3E721460222FFF7C3FC0222A118FFF79B
:1088F000BFFC0634074B641B1C8041F60F53C31AA0
:1089000058425841F8BD0020F8BD00BF00400008A3
:1089100000800008E83E00202DE9F04FDFF84C9180
:108920004D4F8BB00326A7EB09071822002104A89E
:1089300035F037F9494BCDF8109005971A69002AA0
:1089400004DA474A5A6002F188325A6001228DF8EF
:108950002420F322DA60434B434C1B88ADF80030EF
:108960000222694604A805F0C5F9022269464FF6BD
:10897000FF70FFF77DFCDFF8F8A080464FF0000B9A
:10898000544539D30AAC002524F8245D022221463F
:1089900004A805F0AFF9022221464046FFF768FC23
:1089A00040BAC043ADF80800022202A904A805F0AD
:1089B000A1F9079878B106ABC0F104022946184422
:1089C00035F0EFF8089818B9069904A805F0F4F8FE
:1089D0000023089007939DF82430089A23B11F497B
:1089E0000B6943F000430B61013E2DD0002A9CD15E
:1089F000FFF75BFF50B32CE065888DF80DB0C5F331
:108A00000B05AB1DADF808302388C3F30B02ADF89E
:108A10000A201B0B062202A904A88DF80C3005F0D1
:108A200069F9062202A94046FFF722FC61688046E8
:108A30002A4604A805F05EF9616840462A46FFF719
:108A400017FC143480469BE7002AD1D0052003F0A0
:108A5000D1FB0BB0BDE8F08F00800008003C024065
:108A6000230167450CDD0308880100080040000869
:108A7000100600080378202B024600F10100F9D00F
:108A8000092BF7D02D2B2CD02B2B03BF5378B7EE0F
:108A9000000A0246B7EE000AA3F13001C8B2092865
:108AA0009FED467A10D8F2EE046A07EE901AF8EEBF
:108AB000E77A12F8013FE7EE267AA3F13001C8B257
:108AC0000928B0EE677AF0D92E2B4CD003F0DF03E3
:108AD000452B0BD0F7EE007A67EE276A20EE260AC8
:108AE00070475378BFEE000A0246D5E710B45178BC
:108AF0002D2959D02B290ABF9178501C901C002495
:108B0000A1F13003092B53D8002303EB830301EBBE
:108B1000430310F8011FA1F13002092AA3F1300329
:108B2000F3D9B3F59A7F28BF4FF49A73072B42D934
:108B3000DFED236A1A46F7EE007A083A072A67EE55
:108B4000A67AFAD803F007032BB1F2EE046A013BD0
:108B500067EEA67AFBD124B3C7EE276A5DF8044B13
:108B600020EE260A70475378A3F13001C8B20928D5
:108B700002F10102AAD8F2EE046AF0EE665A07EE9C
:108B8000901AF8EEE77A12F8013F87EEA66AA3F191
:108B90003001C8B2092866EEA56A37EE067AEED92A
:108BA00094E767EE276AD9E7901C91780124A7E73C
:108BB000F7EE007ACFE7F7EE007AC5E70000000095
:108BC00020BCBE4CB5EEC00ADFED317AF1EE10FAF2
:108BD000CCBF30EE270A30EE670ADFED2E7A20EEAA
:108BE000270A30B5FDEEC07A87B017EE904A0546E9
:108BF00084EAE470002303A9A0EBE47001930093DE
:108C0000029326F0C5FC002CACBF20232D2303A823
:108C10008DF8003031F070FD012803A924D002281E
:108C20002DD0032805BF3023684668468DF80130F3
:108C300034F0DDFF684631F05FFD0338C4B22246F0
:108C40006946284635F031F800232B55284631F087
:108C500053FD2E22431C2A540DEB0401E81834F076
:108C6000E3FF284607B030BD302368468DF8013059
:108C70008DF802308DF8033034F0B9FFDAE7302395
:108C800068468DF801308DF8023034F0B0FFD1E73E
:108C90006F12033A00007A442DE9F041064615466A
:108CA0000846B6FBF2F43CB905FB1464124B1B5D9D
:108CB00000F8013BBDE8F081B4FBF2F767B90E4B59
:108CC00005FB174705FB1464DA5D00F8012B1B5DFB
:108CD00000F8013BBDE8F081B7FBF2F8B8F1000FF6
:108CE00002D04046FFF7D8FF05FB1878024B13F877
:108CF000082000F8012BE3E71C10040830B40268D8
:108D00001146531C036011F8024B0160D31C5178CB
:108D100003609378151D05601B0443EA0123D07896
:108D2000234343EA006030BC704700BF0368591C0E
:108D30001A46016012F8021B0260587841EA0020CE
:108D4000704700BF03685A1C02601878704700BF64
:108D500038B504460068154632F00CFC22682A44F7
:108D6000226038BD036810B40A0E5C1C04601A70DF
:108D700003680A0C5C1C04601A7003680A0A5C1C15
:108D800004601A7003685A1C026019705DF8044B85
:108D9000704700BF036810B40A0A5C1C04601A70B4
:108DA00003685A1C026019705DF8044B704700BFDD
:108DB00003685A1C026010B4197003680A0A5C1C2C
:108DC00004601A7003680A0C5C1C04601A70036863
:108DD000090E5A1C026019705DF8044B704700BF01
:108DE00003685A1C026019700368090A5A1C026061
:108DF000197070472DE9F047002488B080460F466F
:108E00001E46A14605AD531C0393117839B325299D
:108E100033D1931CCDF810900393507830284ED066
:108E20004FF0000AA0F13003DBB2092B42D96C28C5
:108E300019D0642800F0938024D825281CD063D949
:108E4000582876D063281BD131784046B847039A1A
:108E5000531C03931178043601340029D7D12046DE
:108E600008B0BDE8F087039B5A1C03921B78642B63
:108E70007CD02AD8252B54D1252140460134B8472F
:108E8000039AC0E7732833D044D975284FD106F12F
:108E9000040E30682B4600220A217646FFF7DEF8E2
:108EA000049A0095534639464046FFF715F9039A50
:108EB0000444A8E704AA03A926F046FBB7E7D31C9D
:108EC000039390784FF0010AACE7732B10D05BD975
:108ED000752B3AD0782B96D1A3F15802B2FA82F2D0
:108EE000306852092B4610210436FFF7B7F8D7E750
:108EF0003368049A0093394600234046FFF7ECF8A4
:108F000004360444039A7EE70028B9D1204608B00D
:108F1000BDE8F0876E28B3D1039A336804361C602D
:108F200071E72AD9582BD7D0632B8DD06BE77828DF
:108F3000A6D1A0F15802B2FA82F2306852092B464B
:108F40001021FFF78BF80436AAE706F1040E30680B
:108F50002B4600220A217646FFF780F8A0E7331D52
:108F6000306829461E46FFF74BF899E7331D3068F5
:108F700029461E46FFF744F892E7002B7FF443AFE3
:108F8000204608B0BDE8F0876E2BC6D03BE700BF97
:108F90000EB400B584B005AB019053F8042B06491C
:108FA000039301A8FFF726FF019B00221A7004B06B
:108FB0005DF804EB03B07047CD8000080FB430B506
:108FC00083B006AB0A490B4853F8042B09680068C4
:108FD0000193FFF70FFF084C0546206803F002FEDF
:108FE0000028FAD0284603B0BDE8304004B07047EE
:108FF000FC3D0020003E002078A70020DFED2B7A0A
:10900000B4EEE70AF1EE10FA4ADDDFED296A9FEDD2
:10901000297A01E0B0EE670AB4EEC70AF1EE10FA61
:1090200070EE667AF6DC9FED247AF4EEC77AF1EE04
:1090300010FA38D5DFED1E6A9FED207A01E0F0EEE0
:10904000407AF4EEC77AF1EE10FA37EEA60AF6D4BB
:10905000DFED1B7AB4EEE70AF1EE10FA14DDDFED76
:10906000137A37EEC00A60EE006A9FED166A9FED34
:10907000167ADFED167AA6EE867A20EE266AE6EEFE
:10908000877AA6EE270A7047DFED117AB4EEE70A79
:10909000F1EE10FA44BFDFED087A37EEC00AE2E7DE
:1090A000F0EE407ABFE7B0EE670AD1E7DB0F494048
:1090B000DB0FC940E4CB1641DB0F49C0E4CB16C13E
:1090C000DB0FC93F92E741B99730083C15A82ABE8B
:1090D000DB0FC9BF09B909E0194690FBF1F301FBA9
:1090E00013030846002BF7D1084670470146FBE7FB
:1090F000F0EEC07AB0EEE07AB4EEE77AF1EE10FA74
:10910000B4BFB0EE676AB0EE476AB5EE406AF1EE02
:1091100010FA46D0B4EEE77AF1EE10FA8CBFF0EE1A
:10912000675AF0EE475AC5EE866A9FED1F3A9FEDEB
:109130001F6A9FED1F4A9FED1F5ADFED1F3ADFEDBB
:109140001F4ADFED1F5AA6EEC36AE6EEA34AA6EE5B
:10915000864AB7EE006AA6EE845AA6EEA46AE6EE48
:10916000855AC5EE866AB4EEE77AF1EE10FA48BF8A
:10917000DFED147AF5EEC00A48BF77EEE66AF1EE4D
:1091800010FA48BFDFED107AB5EEC00A48BF77EE9F
:10919000E66AF1EE10FA48BFF1EE666AB0EE660AD2
:1091A0007047DFED076ADEE739094E3DE3B59E3EC5
:1091B00088FA163E45FE7F3F99FB243F69A2163E82
:1091C000A7DFA834DB0FC93FDB0F4940DFED317A61
:1091D00030EE277AFDEEC76A16EE903A2033402B28
:1091E00002D99FED2D0A7047B4EEE70AF1EE10FAAE
:1091F0004DDD9FED2A6ADFED2A6A01E0B0EE677A65
:10920000B4EEE67AF1EE10FA77EE467AF6DC9FEDF0
:10921000257AF4EEC77AF1EE10FA35D5DFED1F6A44
:109220009FED217A01E0F0EE407AF4EEC77AF1EE9C
:1092300010FA37EEA60AF6D4DFED167AB4EEE70A96
:10924000F1EE10FA1BDCDFED197AB4EEE70AF1EE6D
:1092500010FA44BFDFED137A37EEC00A60EE006A01
:109260009FED136A9FED137ADFED137AA6EE867AEF
:1092700020EE266AE6EE877AA6EE270A7047DFED33
:109280000F7A37EEC00AE9E7B0EE670AD4E7F0EEEE
:10929000477ABCE7DB0FC93F00000000DB0FC94085
:1092A000E4CB1641DB0F49C0E4CB16C1DB0FC9BFCD
:1092B00092E741B99730083C15A82ABEDB0F494018
:1092C000FDEEC07A17EE903A2033402B51D8DFEDF7
:1092D0002D7AB4EEE70AF1EE10FA50DDDFED2A6ADE
:1092E0009FED2A7A01E0B0EE670AB4EEC70AF1EE0C
:1092F00010FA70EE667AF6DC9FED257AF4EEC77A06
:10930000F1EE10FA38D5DFED206A9FED227A01E008
:10931000F0EE407AF4EEC77AF1EE10FA37EEA60AD4
:10932000F6D4DFED1D7AB4EEE70AF1EE10FA1BDC9D
:10933000DFED1A7AB4EEE70AF1EE10FA44BFDFED82
:10934000147A37EEC00A60EE006A9FED156A9FED51
:10935000157ADFED157AA6EE867A20EE266AE6EE1D
:10936000877AA6EE270A7047DFED067A37EEC00A45
:10937000E9E79FED0E0A7047B0EE670AD1E7F0EE1D
:10938000407AB9E7DB0F4940DB0FC940E4CB164117
:10939000DB0F49C0E4CB16C1DB0FC93FDB0FC9BFF0
:1093A00092E741B99730083C15A82ABE000000009A
:1093B00010B507EE901A2DED028BB8EE678ADFED3F
:1093C000217A28EE008A044628EE278AB0EE480A61
:1093D00032F026FBF0EE408AB0EE480A32F082FA14
:1093E000F7EE007A9FED187AF0EE675AE8EE875AAA
:1093F0000023A361B0EE676AC7EEA56A63612362CA
:10940000E361A8EEC76ABDEC028B77EEC07AB6EED8
:10941000007AF8EE005A27EE877A20EE250A27EE2A
:10942000267A26EE266A67EEA67A20EE260A84EDD4
:10943000046AC4ED017A84ED007A84ED027A84ED49
:10944000030A10BD27D4D236F304353F10B44C09BB
:10945000012250F8243001F01F0102FA01F10B4300
:1094600040F824305DF8044B704700BF4B0901F011
:109470001F0150F82320012303FA01F1114214BF08
:1094800018460020704700BFAA4B33F81020110582
:1094900013D52DE9F043A8490446400904F01F05FF
:1094A00051F820000121A940014291B006D0A34902
:1094B000097819B111B0BDE8F083704702F01F07B9
:1094C000C2F34415242CF5D8DFE814F0430055000E
:1094D0009000A2005201960196019B044A036A0380
:1094E0007002A002BA02C502D802E302F402FD0231
:1094F000C901CB04BD040A05D9010D020D023702D2
:109500004A024A028E03EF03FC030D041E048F047B
:10951000510480042500DFF85482D8F820200AB1D5
:10952000B2F90820864908AE3046FFF731FD3046D3
:1095300031F0E2F8D8F800403844A0722068E572B3
:109540002A463346456939462046A84711B0BDE84A
:10955000F0837C4B7C491A88DFF81082642303FB7C
:1095600002F39B1208AE632BA8BF6323304601228F
:10957000FFF70EFDDBE7754B754A1B781088022B51
:1095800000F00785734B744C5A781978247802EBF5
:109590008202520000EB800301EB81015B0093FB30
:1095A000F4F39B1AC3EBC303C2EB410293FBF2F348
:1095B000062BA8BF062323EAE373C3F19603DBB2AD
:1095C000664A8DF82030A2FB0032D20802EB8203FB
:1095D000A0EB4303624906209BB200900DF12100ED
:1095E000FFF7D6FC08AEDFF88481A0E7DFF87C81C6
:1095F000D8F8000003681B69984710AEB0F5F07FFB
:10960000584B46F8203D0CBF072506250D278EE751
:1096100093F86120544993F86060B1F9000002EBBF
:10962000820253005F4206EB8606B8424FEA4606C6
:1096300003DB8342A8BF03461F46B1F902307542DF
:10964000AB4203DBB342A8BF33461D46DFF81C81A3
:10965000D8F8000003681B699847B0F5F07F05EB68
:10966000850518BF0224BB0048BF3F3305EB8505C5
:1096700095FBF6F6293EC6EBA313512B40F22A8642
:1096800007EB4705002D2B46B8BF05F13F03C6EB9E
:10969000A313512B40F20186ED1B002D2B46B8BFC2
:1096A00005F13F03C6EBA313512B40F2D985ED1B07
:1096B000002D2B46B8BF05F13F03C6EBA313512B7A
:1096C00040F28A85ED1B002D2B46B8BF05F13F0304
:1096D000C6EBA313512B40F2E184ED1B002D2B466A
:1096E000B8BF05F13F03C6EBA313512B40F2B98479
:1096F000ED1B002D2B46B8BF05F13F03C6EBA313AE
:10970000512B40F29184ED1B002D2B46B8BF05F183
:109710003F03C6EBA313512B40F26984ED1B48BFF6
:109720003F35C6EBA516512E40F2FA840420FFF710
:10973000ABFEBFE694580020206600200000002009
:1097400094100408887F002064100408907F002093
:10975000E87D0020D4A60020FE7D0020CDCCCCCC1E
:109760006C100408267E2700CCA60020B42400201C
:10977000DFF8E883D8F8000003681B699847B0F564
:10978000F07F0CBF0727062707F1040614BF032448
:1097900004240825D8F800000368C4728572D3F841
:1097A0001890224613230721C847D8F80000162234
:1097B0000368C472827222460134D3F818901521CE
:1097C0001323E4B2C847A642E4D1D8F80000092226
:1097D0000368C77282729C693A4603230821A04736
:1097E000D8F8000015220368C77282729C693A4655
:1097F00002231421A0475DE603EB4403B3F8523083
:1098000013F00F0200F0DC83022A8CBF20219C2180
:10981000012AC3F303148DF8201000F0D685C0F0A0
:10982000D483022A00F0BE850023DFF830831A4675
:109830001846012C40F0B083A74EA84CA849A6FBBF
:109840000060400BA4FB00646409642606FB14005E
:1098500000900DF12100FFF79BFB08AE67E6A14BDE
:10986000A14A1868A149047A83790194C0790090CB
:1098700008AE3046FFF78CFBDFF8E08257E69C4BE2
:109880009C4A1B8812789C4903EB8303022A0978BF
:109890004FEA430393FBF1F300F07983974A517841
:1098A000127801EB8101490002EB82005A1AC2EBE7
:1098B000C202C1EB400192FBF1F2062AA8BF0622C8
:1098C00022EAE272C2F19602D2B284488DF82020D8
:1098D00080FB0320DA17C2EB60126424884906205B
:1098E00004FB123379E6874A874B8849DFF86C829C
:1098F00092E84100182C08BF064683FB06234FEA76
:10990000E672C2EBA35203A814BF602364238DF850
:109910002030FFF73DFB32467C4905A8FFF738FBB6
:1099200003A830F0E9FE05AB034403AA78490DF122
:109930002100FFF72DFB08AEF9E576487649B0F92E
:109940000230B0F90020B0F90640B0F904000090F0
:1099500008AE01943046FFF71BFBDFF80082E6E516
:109960006E4B6F486F49DFF8F4811A2C0CBFB3F9C6
:109970000220B3F9002080FB0230D317C3EBA00410
:1099800004EB8400A2EB400383EAE370002AA0EB1F
:10999000E37008AE84EAE4730090ACBF20222D226D
:1099A000A3EBE4733046FFF7F3FAC0E55E4E31688F
:1099B00000248DF80B408DF80C40002900F02D8517
:1099C0000A68D269002A00F00A8503A90DF10B008C
:1099D000904731688DF8144031B10B68196A19B19C
:1099E00005A888479DF814109DF80C404F489DF835
:1099F0000B204F4B825C009108AE53F824304D4948
:109A0000DFF858813046FFF7C3FA90E54A4B3348F8
:109A10001B684A49DFF8448183EAE37EAEEBE37ECC
:109A200080FB0E304FEAEE72C2EB601208AE64208B
:109A30009A2400FB12E300943046FFF7A9FA76E57A
:109A40003D4B3F499A68DFF8148108AE3046072342
:109A5000FFF79EFA6BE52B4B3A4ADB893A49DFF870
:109A6000FC8003EBC3039B0082FB030208AEDB1701
:109A7000C3EBA2123046FFF78BFA58E5214B33496E
:109A80001B7DDFF8D88008AE30461F22FFF780FA32
:109A90004DE593F85B302E49DFF8C080002B0CBFFA
:109AA0000F220C2208AE0023009230461A46FFF720
:109AB0006FFA3CE50B4B274A18680C498478037809
:109AC00001944078D3E6074B234A18680749447944
:109AD000C37801940079CAE65917B7D11F85EB51B5
:109AE000C01004085C59002000110408EC100408A0
:109AF000E87D0020907F0020FE7D0020D4A600207D
:109B00004C110408F0A600206BCA5F6B9410040887
:109B100098100408087D002058110408CCA60020E5
:109B2000676666666C110408A84B00207C01040877
:109B300084010408DC100408B4A400207810040890
:109B400084100408D34D62108C10040864100408BB
:109B5000A8100408E8100408FC100408B42400202D
:109B6000C54B1A78002A00F0B6825C1E03F10F087C
:109B70000DF11F09667831F0DDFC30443246437840
:109B800003F00303022B14F8013F08BFA6F12002E3
:109B900009F8012F002B00F08480A045EAD180E075
:109BA000B64BB74AB3F90630B649DFF81C83B3F5B4
:109BB000FA6FA8BF4FF4FA63B3F57A7FB8BF4FF4DA
:109BC0007A73A3F57A7382FB0302DB17C3EBA2025D
:109BD000042405230DF122008DF820408DF821305A
:109BE00008AEFFF7D5F9A2E4A74BA84A1B899268F3
:109BF000A7499A1A9A42A8BF1A4622EAE27207EEC9
:109C0000902AA1FB0313DB08B8EEE77A07EE903A3F
:109C1000F8EEE77AC7EE276A16EE900A30F0D8FE23
:109C200041EC100B31F084FD51EC100B31F0BEF91A
:109C30008A23C0B28DF82030002840F09E818D2309
:109C40008DF821308D238DF82230022800F26B81AF
:109C50008D238DF823308D238DF824308D238DF8BE
:109C600025308D238DF826308D238DF827308D23D8
:109C70008DF828308D238DF829308D238DF82A30EA
:109C80008D238DF82B30431E8F22092B8DF82C202D
:109C900004D810AB18448E2300F81F3C00238DF825
:109CA0002D3008AEDFF8208241E47A4B1B78DB07C9
:109CB0003FF500AC08AE30467749DFF80C82FFF77D
:109CC00067F934E4754B1B7803F00303032B00F0B2
:109CD00019832D238DF8203000238DF8213008AE14
:109CE000DFF8E48123E46D4A127802F00302032ACC
:109CF00000F03B832D2200238DF820208DF82130A9
:109D000008AEDFF8C48112E4654B5D4AB3F9043054
:109D100064486549DFF8B08182FB0342DB17C3EB7F
:109D2000A2031BB2162404EB430480FB0462161941
:109D3000E217C2EB66224FF4347606FB124280FB38
:109D400002401044D217C2EB6012D2B2C2F1180224
:109D5000504200F00F0002F00F0258BF4242603242
:109D600008AED2B23046FFF713F9FFF7E0BB4C4B19
:109D7000434CB3F904304B484C49DFF84C8184FB29
:109D80000324DA17C2EBA4021623022412FB0432C6
:109D900080FB02439C18D317C3EB64234FF4347445
:109DA00004FB132380FB03021A44DB17C3EB62138B
:109DB00051FA83F308AE186859681C7A334603C316
:109DC00000221C708DF82920FFF7B1BBDFF8F88066
:109DD000D8F820200AB192F90120354908AE304662
:109DE0000E23FFF7D5F8FFF7A2BB08AE00233046DD
:109DF000009368222F49DFF8D080FFF7C9F8FFF7FA
:109E000096BB2D4B1B68DC0040F1CE802B4B032210
:109E10002B490988480500F18380CE0700F1BF82F5
:109E200001F00201274800291CBF032203462649EE
:109E300008683A4404688272C57239462A466469E1
:109E4000A047FFF737BB214A214953781278DFF842
:109E5000788008AE013301323046FFF799F8FFF7FA
:109E600066BB1C4A094B10881B681B4A1B49DFF85C
:109E7000588003FB00F3F7E548840020607F002052
:109E80006766666694100408D4A60020B4A4002077
:109E9000A38B2EBA747D002078110408ECA6002054
:109EA000CCA60020B7600BB68411040810DD0308AF
:109EB000A01004088C110408208400204410040819
:109EC0008A7F002060100408B4240020A0740020C1
:109ED0000C110408E87D0020D34D62100411040821
:109EE0000021CC48FFF7C2FA002840F03281CA4B6B
:109EF0001B7813F0020FC94B1B7802D1002B00F026
:109F00007882012B00F00381022B40F0F28008AE32
:109F10003046C349DFF84483FFF73AF8FFF707BB41
:109F20000422C04B83E78B2303288DF823307FF670
:109F300092AE04288DF824307FF690AE05288DF877
:109F400025307FF68EAE06288DF826307FF68CAE53
:109F500007288DF827307FF68AAE08288DF828303C
:109F60007FF688AE09288DF829307FF686AE0A285C
:109F70008DF82A303FF685AE82E68B2301288DF8D6
:109F8000213018BF8DF822307FF45FAE5AE6972259
:109F90009BE49723FFF714BBA3490DF12100FEF7C3
:109FA000F7FF08AEFFF7C3BAA04AA1491268A14B58
:109FB00002F48002002A0ABF0B460322042227E78C
:109FC0009B22C3F303148DF8202002F063FB9A4B0D
:109FD0009A4ADFF88882A3FB00139B0C82FB0312D2
:109FE0001A445211C2EB0211A3EB810321E49449FC
:109FF000D8F8000081FB0321DA17C2EB610204EB01
:10A00000020E02EBC2015B1A5FFA8EF20168C272A5
:10A010004FF0120E80F80AE0803BD1F81890DBB2C6
:10A020001121C847FFF77ABB8549D8F8000081FBAA
:10A030000321DA17C2EB610204EB020E02EBC2014C
:10A040005B1A5FFA8EF20168C2724FF0110E80F84F
:10A050000AE0803BD1F81890DBB21021C847FFF727
:10A0600052BB7749D8F8000081FB0321DA17C2EB15
:10A07000610204EB020E02EBC2015B1A5FFA8EF280
:10A080000168C2724FF0100E80F80AE0803BD1F8F0
:10A090001890DBB20F21C847FFF72ABB6849D8F8F0
:10A0A000000081FB0321DA17C2EB610204EB020E10
:10A0B00002EBC2015B1A5FFA8EF20168C2724FF0C6
:10A0C0000F0E80F80AE0803BD1F81890DBB20E2129
:10A0D000C847FFF702BB5B4BDFF8808193E80700BE
:10A0E00008AE334603C323F8022B120C1A70FFF795
:10A0F0001EBADFF8688198F81C30002B3FF4DAA90B
:10A1000008AE30465049FEF743FFFFF710BA08AEDD
:10A1100030464E49DFF84481FEF73AFFFFF707BAB1
:10A12000474AD8F8000082FB0632F317C3EB6203FC
:10A13000E21803EBC3031324D2B2F61A0168C27209
:10A14000A6F1800384728C69DBB21221A047FFF76D
:10A15000EDBA3F4B1B88002B3FF4C9AEDC0700F182
:10A160006081C3F340025ABB580700F1748119079C
:10A1700000F16F81DA0600F16A819E0600F16581C7
:10A180005C0600F16081180600F15B81D90500F1E1
:10A1900056819A0500F151815E0500F14C811C0544
:10A1A00000F14781D80400F14281990400F13D811A
:10A1B0005A0400F13881DB0B18BF0F223FF471AD58
:10A1C000244B254953F82220DFF8908008AE304612
:10A1D000FEF7DEFEFFF7ABB91949D8F8000081FBA6
:10A1E0000321DA17C2EB610204EB020E02EBC2019B
:10A1F0005B1A5FFA8EF20168C2724FF00E0E80F8A1
:10A200000AE0803BD1F81890DBB20D21C847FFF778
:10A2100059BA00BF20840020747D0020907F002068
:10A220003411040850100408B4100408D879002030
:10A23000481004084410040883DE1B43898888887A
:10A24000398EE338D010040840110408281104089E
:10A25000B87F0020A0E7030814110408B4240020EC
:10A260007E49D8F8000081FB0321DA17C2EB6102B6
:10A2700004EB020E02EBC2015B1A5FFA8EF2016878
:10A28000C2724FF00D0E80F80AE0803BD1F81890B2
:10A29000DBB20C21C847FFF70ABA7049D8F80000B2
:10A2A00081FB0321DA17C2EB610204EB020E02EB21
:10A2B000C2015B1A5FFA8EF20168C2724FF00C0E97
:10A2C00080F80AE0803BD1F81890DBB20B21C84738
:10A2D000FFF7E2B96149D8F8000081FB0321DA17E2
:10A2E000C2EB6102A51802EBC2015B1AEAB2016877
:10A2F000C2720B25803B85728D69DBB20A21A847AB
:10A30000FFF7BEB9564B1B88002B6CD0554B5648F7
:10A31000B3F90430554A5649B2F9002080FB034096
:10A32000DB17C3EBA0031BB2D21A5200163281FB1B
:10A3300002039818D317C3EB60234FF4347000FB6B
:10A34000132381FB03121A44DB17C3EB6213DBB246
:10A35000C3F118035A4202F00F0203F00F0358BF73
:10A36000534260338DF82030B6E43D4A93F85B30B9
:10A370001288002B3BD14FF4A4733E4903FB02F239
:10A3800081FB0213D217C2EB63120F2308AE3046D3
:10A390003949DFF80481FEF7FBFDFFF7C8B8374BFA
:10A3A000042244E5DFF8F0803549D8F81800354A32
:10A3B000A1FB0031890C82FB01320A445211C2EB2D
:10A3C0000213A1EB8303FFF734BADFF8CC802C4BE8
:10A3D000D8F808002B4AA3FB0013990CEBE78DF883
:10A3E0001420FFF7FABA05238DF8203074E40C230B
:10A3F000CCE7254A254B2649927B1B88097893FB9D
:10A40000F1F39A427FF675AE08AE30462149DFF887
:10A410008880FEF7BDFDFFF78AB88DF81410FFF7AE
:10A42000E3BA0022CCE60E22CAE60D22C8E60C22D0
:10A43000C6E60B22C4E60A22C2E60922C0E60822CA
:10A44000BEE60722BCE60622BAE60522B8E60422EA
:10A45000B6E60322B4E60222B2E600BF398EE33844
:10A46000D46C0020CCA6002067666666D66C0020FF
:10A47000B7600BB61F85EB51A010040858100408F4
:10A4800083DE1B4389888888D4A60020E87D0020CD
:10A49000FE7D002018110408B4240020074A084B50
:10A4A00010781B78074A834296BFC31AC3F1800312
:10A4B0000020126818441044704700BF98820020A2
:10A4C00014820020A85F0020064A074B10781B78F2
:10A4D00083428ABFC3F18003C01AC018C0F17F0055
:10A4E000704700BF988200201482002030B5144CC1
:10A4F000237883B01BB90120237003B030BD05223F
:10A5000000238DF800208DF8013000BF0D4D2B6821
:10A51000986802F06BFF2B6801AA694658682FF013
:10A52000EDFC2B68986802F067FF00BF9DF80530CE
:10A5300003F0010383F00100237003B030BD00BFBE
:10A540007A7C0020687C002070B5064C06462568A1
:10A5500003E023685B1BB34203D8FFF7C7FF002863
:10A56000F7D070BD607C00202DE9F04F89B0B2F1CA
:10A57000000A02900491039340F3B0800B4600223E
:10A5800001EB8A0153F8040B8B420244FAD1039B7E
:10A590000592002B00F09A80059B002B6AD0544B4B
:10A5A000059A1B68DFF85C9100920099DAB25118A5
:10A5B000B1F5807F8CBFC2F58072009A01924D4A3E
:10A5C00092689A426DD9190C1A0A4FF002040620BB
:10A5D0008DF81F308DF81E208DF81D108DF81C4051
:10A5E000FFF7B2FF0620FDF7F1FF434A0123137086
:10A5F00000BFD9F80030986802F0F8FED9F80030B2
:10A6000007A9586800222FF02BFC0024049D029E0D
:10A61000019FA34629684FEA840800220B460134B3
:10A6200071B1B9422AD2D9F800003168406803F00C
:10A63000CDF82A68336813443360BF1AC5F800B0F8
:10A64000A24505F1040506F10406E3D1D9F800306E
:10A65000986802F0D1FE00BF254B019900981B6855
:10A66000421A0092224A0B441360039A32B3009AB2
:10A67000002A9AD1059809B0BDE8F08F029CD9F85C
:10A68000003054F80810586800223B4603F09EF84A
:10A6900054F808202B683A44DF1B44F808202F6048
:10A6A000D4E70598009C1549154A001B05900598AC
:10A6B00000230B70137009B0BDE8F08F059B009A62
:10A6C0009B1A0593059809B0BDE8F08FFFF70EFFC0
:10A6D00000287FF461AF039B0593CBE7039C1CB973
:10A6E000FFF704FF0594C5E700230593C2E700BF09
:10A6F000A85F0020D41D00207A7C002098820020D2
:10A7000014820020687C002070B5104D104E2B780C
:10A7100031788B4284B016D00E4A03921A440292CA
:10A720008CBF0C46CA1A04A98CBFC3F18002002456
:10A73000012341F8102D02A802220194FFF714FF13
:10A74000002333702B7004B070BD00BF1482002052
:10A75000988200201882002070B5194C194D23787A
:10A760002978994284B027D0174A03921A4402925A
:10A7700034BF0E46CA1A04A934BFC3F180020026B2
:10A78000002341F8102D02A802220196FFF7ECFEEB
:10A7900023781844C0B203062B7848BF80F08000AD
:10A7A0008342207002D0002004B070BD002301203D
:10A7B0002B70237004B070BD012004B070BD00BFC9
:10A7C00014820020988200201882002008B545F2EB
:10A7D0000820FFF7B9FE0620FDF7F8FE064B012220
:10A7E000C7201A70FDF7F2FE04480549054A002308
:10A7F00003700B70136008BD7A7C002098820020E3
:10A8000014820020A85F00202DE9F04182B00346A9
:10A81000060C050A032406208DF8073088461746E3
:10A820008DF805608DF806508DF80440FFF78CFE1A
:10A83000C0B100BF0D4C2368986802F0D7FD2368B3
:10A8400001A9586800222FF00BFB23684246002123
:10A8500058683B4602F0BAFF2368986802F0CCFDC6
:10A8600000BF384602B0BDE8F08100BF687C002020
:10A87000F0B5124B9D6885B00DB905B0F0BDED0A7D
:10A8800014D0002704AE7C196410E002102269463F
:10A89000FFF7BAFF0F2809DD6B4653F8042B01328E
:10A8A0000AD1B342F9D12546AF42ECDBFFF72CFFCA
:10A8B000034BED021D60E0E7671CF5E7D41D0020A7
:10A8C000A85F00202DE9F04F744B754C1B788DB0BC
:10A8D00005460BB101232377626A724BA3FB021377
:10A8E0009B0803EB8303511CD31A616240F0B980CB
:10A8F000DFF8E4B194F828109BF8007007F0010726
:10A90000B94200F09781002F40F0EE80D4F800802B
:10A91000654ED8F8003040469B6898472068FF2372
:10A9200088F80D300122036888F80C2011210222DA
:10A930008172C272D3F814805C4B1146C04796F8FE
:10A940005230002B40F0A38309230693082305937C
:10A950000623049305234FF00A084FF0070A0393D8
:10A960004FF00409032796F85330002B40F03F8343
:10A9700096F84A30DFF8648123B198F800309B07DD
:10A9800000F14C8496F85430CBB196F85B30B4F9B2
:10A990001620002B00F0C9830C23454909A8FEF7B7
:10A9A000F7FA384609AA4349FDF7D6FD049BCDF8CE
:10A9B00010A0DDF814A04F46DDF80C90039396F834
:10A9C0004B30002B40F0BB8296F85130DFF810A1DD
:10A9D000002B40F0EE8296F84C30002B40F0D282F3
:10A9E000354B9B79002B40F04782DFF8F89096F8C2
:10A9F0004F30002B40F0688296F85030CBB12F4B8F
:10AA00009B783BB3032B25D0012B00F06B840022F5
:10AA1000114609ABB2FBF1F2184692B228490793EE
:10AA2000FEF7B6FA7B1C3846079A2649DFB2FDF7D7
:10AA300093FD96F855306BB1204B9B7853B1032BA7
:10AA400008D009A9002024F0A3FD09AA38461E4910
:10AA5000FDF782FD1D4A1E4E2A4400233260A36189
:10AA600069E020680368DB689847236863B193F95D
:10AA70000E30002B08DD174A138843F480439BB245
:10AA800013800DB0BDE8F08F124A138823F4804381
:10AA90009BB213800DB0BDE8F08F00BF387F00205F
:10AAA000B4240020CDCCCCCC94580020A0110408B4
:10AAB000A0100408BC110408D4A60020AA5A002043
:10AAC000441204082C120408381204080087930367
:10AAD00028660020B87F0020747D0020ECA60020AE
:10AAE000E87D0020B4A40020266863613068A3617B
:10AAF0004FF0FA714FF4C6028368E160304622617C
:10AB000098472068DFF86083DFF860A3DFF8609380
:10AB1000FF237373012203683273112107228172AC
:10AB2000C2725F69C04BC14E0C21B84705F5F422D3
:10AB300002F5907232609BF8001001F0010184F878
:10AB40002810BB4BDFF82CE3DB89BA4803EBC303C7
:10AB50009B008EFB03CEDB170788B4F90C00C3EB18
:10AB6000AE131BB29842B8BFA381B4F90E00BAF875
:10AB700000309842C8BFE381AF48D9F800304FF0A9
:10AB8000640E80FB03C0DB170EFB07F7C3EB6013FB
:10AB9000B4F910E01BB29E45B8BF2382B4F912305D
:10ABA000C7F38727BB42B4F91430C8BF6782002BB4
:10ABB000BCBF0023A38298F8003084F8297003F00A
:10ABC0000303032B2ED039B1E36AA068A169EB1A05
:10ABD00018440B44A060A361E5626AB1AA1A002A76
:10ABE00031DB27683B6838469B6898470121FF2284
:10ABF000002339737A7333609049914F914A3B68CF
:10AC0000AD09A1FB0515C5F3801515701D0100F1F7
:10AC10000581236853B393F90E20002A26DD002214
:10AC2000227723E7884BB4F916001B889842B8BFF7
:10AC3000E382C8E77D4EDFF830823268DFF82CA26D
:10AC4000DFF82C927DE7814AB2F9061040F2D66314
:10AC5000994203DCB2F902209A4201DD00233360FD
:10AC6000206803681B6A98472368D8E7784E94F8F1
:10AC7000293096F85A209A4240F22181754D2B686E
:10AC800043F00103744A1278002A40F0138123F440
:10AC9000C00323F0020398F80020900700F1078119
:10ACA00043F48043B6F85C802B6008F00F02012A61
:10ACB00000F0B282C0F0AC82022A00F04382002091
:10ACC000664A4FEA182802FB08F2002A00F06A825E
:10ACD000824200F2678243F02003B6F85E802B6068
:10ACE00008F00F02012A00F09182C0F06382022A6C
:10ACF00040F05E82A069594A4FEA182802FB08F228
:10AD0000002A00F04C82824200F2498243F0400364
:10AD1000D9F80820B6F856109142B6F85820D4BF9A
:10AD200043F0102323F01023002A00F03E8223F486
:10AD3000004326682B60336830469B6898470122A1
:10AD4000FF233273737313214548FEF78FFB0028EE
:10AD500086D1444D2B68990700F1AD820120FEF7A2
:10AD600093FB0020FEF790FB0220FEF78DFB0520F1
:10AD7000FEF78AFB0620FEF787FB0720FEF784FB21
:10AD80000920FEF781FB0A20FEF77EFB0B20FEF771
:10AD90007BFB0C20FEF778FB0820FEF775FB0F20ED
:10ADA000FEF772FB1020FEF76FFB1120FEF76CFB25
:10ADB0001220FEF769FB1320FEF766FB1420FEF756
:10ADC00063FB1520FEF760FB1620FEF75DFB1920E4
:10ADD000FEF75AFB1A20FEF757FB1B20FEF754FB29
:10ADE0001C20FEF751FB1D20FEF74EFB2020FEF736
:10ADF0004BFB2120FEF748FB2220FEF745FB2B688A
:10AE00009A0600F145823B681B017FF529AF23209C
:10AE1000FEF73AFB2420FEF737FB21E7FF2026F060
:10AE200063F92062F5E600BF981104082866002047
:10AE3000F0A60020887F00201F85EB51632D3E0582
:10AE4000D879002000000020D46C0020607F002012
:10AE50009458002020660020907F002000879303F4
:10AE600020840020E8A60020ECA60020E87D002039
:10AE7000B4A40020D34D621096F84D30002B40F062
:10AE8000E48196F84E30DFF87C93002B3FF4AFADB1
:10AE9000D9F80820C94909A80723FEF779F87B1CCF
:10AEA000384609AAC649DFB2FDF756FB9FE523F4F1
:10AEB0008043F7E643F4C00343F00203EBE6C14DE1
:10AEC0002B6823F00103DDE696F85B10B4F914E07B
:10AED000002940F039810EEB8E000EEBC00EBA4A0D
:10AEE000BA4B4FEACE004FEAE07E82FB00C2CEEBC7
:10AEF0002232002A83FB00C0B8BF5242DEEB601E44
:10AF000000F1DD8183FB0E314FEAEE73C3EB611379
:10AF10006420AF4900FB13E381FB0301DB17C3EBA4
:10AF2000A1030F21009109A8AA49FEF731F87B1C63
:10AF3000384609AAA849DFB2FDF70EFB5CE5B4F973
:10AF40000E30A34AA54982FB0302D817C0EBA20228
:10AF500002EB82004FF0060EA3EB40031BB212B2CD
:10AF6000CDF800E009A8FEF713F8384609AA9C4975
:10AF7000FDF7F2FA049BCDF810A04F46DDF80C90D7
:10AF8000039321E509AA1146B4F91200049224F0B2
:10AF9000FFFA049A10462FF0AFFB924B049A1B88DD
:10AFA000135291493846FDF7D7FA4F46DDF80C9019
:10AFB00016E5BAF800308D4A8849A2FB0302D20890
:10AFC00002EB82004FF0060EA3EB40039BB2CDF8DC
:10AFD00000E009A8FDF7DCFF384609AA8449FDF71F
:10AFE000BBFA049B4F46DDF80C900393F3E4B6F8EC
:10AFF0005E3003F00F02012AC3F30313079300F03E
:10B00000C980C0F06B81022A40F06481D4F818E056
:10B01000784B794AA3FB0E139B0C82FB03121A4454
:10B020005211C2EB0211A3EB81030799012940F0F1
:10B030002881DFF8D4C165487049ACFB0ECE4FEAD9
:10B040005E3EA0FB0EC040094FF0640C0CFB10EEFE
:10B05000CDF800E009A80790FDF79AFFB6F85E303A
:10B060006749079A03F00F03384651F82310FDF79C
:10B0700073FA049BCDF810A04F46DDF80C900393B3
:10B08000069BDDF814A0CDF81880059370E4B6F89F
:10B090005C3003F00F02012AC3F303187DD0C0F027
:10B0A0001681022A40F00F81A069524B524AA3FB3D
:10B0B00000139B0C82FB03121A445211C2EB0217BD
:10B0C000A3EB8703B8F1010F40F0D480DFF838E13B
:10B0D0003E4F4A49AEFB00E0400BA7FB00E77F096B
:10B0E0004FF0640E0EFB170009AF0090384607972B
:10B0F000FDF74EFFB6F85C304149079A03F00F03A5
:10B10000032051F82310FDF727FA0A230693092399
:10B1100005930723049306234FF00B084FF0080A0A
:10B1200003934FF0050904271DE402EB820302EBB1
:10B13000C3022649D30081FB0321DA17C2EB611257
:10B140000F232AE4A069BBE5204A4FEAEE7382FB95
:10B150000E02C3EB6212002AB8BF5242BEF1000FCA
:10B16000C0F2AF80DFF864C08CFB0E0CC3EB6C1335
:10B1700017484FF0640C0CFB13E380FB03E0DB1774
:10B18000C3EBA003002BB8BF5B4200290CBF0F210B
:10B190000C21C7E6D4F808E03AE7A06885E723F079
:10B1A0004003B5E523F0200397E543F40043C0E5F1
:10B1B0000020A0E501F06EFA2B689CE5A0100408C1
:10B1C0000412040820660020AD8BDB681F85EB515C
:10B1D00067666666101204081C1204086C100408E6
:10B1E000CC110408E4110408E8110408CDCCCCCC3F
:10B1F000D811040883DE1B4389888888C01004089E
:10B2000000020408B4A400205917B7D1A06872E561
:10B2100001F040FA2B6853E5A06851E509A9B4F99B
:10B220000C0024F0B5F9384609AA3949FDF794F91C
:10B23000049BCDF810A04F46DDF80C900393069BBD
:10B24000DDF814A00593FFF79DBB09AA1146B4F9D8
:10B250001000039224F09CF9039A10462FF04CFA48
:10B260002C4B039A1B8813522B493846FDF774F96F
:10B270004F4606E609A9079108462849FDF788FECA
:10B2800038E709A9079108462449FDF781FEE5E65C
:10B290000E20FEF7F9F80D20FEF7F6F81820FEF75D
:10B2A000F3F81720FEF7F0F81F20FEF7EDF81E2048
:10B2B000FEF7EAF8A7E50320FEF7E6F84EE54FEAC9
:10B2C000EE7352424EE73B463A463846FAE601F004
:10B2D000E1F9EAE600231A469E46A6E601F0DAF90D
:10B2E000864695E6FFF702F938B909AB18460C49CE
:10B2F0000793FDF74DFEFFF795BB0A4B9968890A46
:10B30000FFF7CCF86423820A03FB02F2FFF781BB4C
:10B31000B0110408F4110408F8110408B41004086A
:10B320004C120408D41D00202DE9F043314A324E5E
:10B3300013683060042B89B004D0304C591C44F899
:10B34000230011602E4B2F4A1B78002103F00103CC
:10B350001160516086F82830012702F0BBF9A02364
:10B360000424FDB203E00134E4B21C2C13D0FF2B03
:10B37000F9DC306802688472C572611E0134D2F84B
:10B38000188003F10109C9B2DBB22A46E4B2C04712
:10B390001C2C4B46EBD10137052FE1D168461A4AE8
:10B3A0001A49FDF7F5FD6B4606221421306802F0BC
:10B3B0006DF9174B30680822072102F067F9154B29
:10B3C000306809220B2102F061F9134B30680A2220
:10B3D0000B2102F05BF9306802F054F901F05AF9E0
:10B3E0000E4B00F5741000F51060186009B0BDE850
:10B3F000F08300BF385B0020B42400203C5B0020B9
:10B40000747D002020660020541204085C12040899
:10B4100060120408701204087C12040828660020D8
:10B420002DE9F84FDFF8A890DFF8A880D9F80000E0
:10B43000DFF8A4A0234E012388F8003001F0D6FFE6
:10B4400005202EF0A9FD00202EF0A6FD06202EF0EE
:10B45000A3FD00202EF0A0FD9AF80040042044F047
:10B4600001042EF099FD20462EF096FD33888BB115
:10B47000154D164F002415F804B007202EF08CFD52
:10B4800058462EF089FD2A5D33883A550134A4B21E
:10B49000A342F0D807202EF07FFDFF202EF07CFD88
:10B4A0009AF8004004202EF077FD20462EF074FD1F
:10B4B000D9F8000001F0A0FF002388F80030BDE8B3
:10B4C000F88F00BF081C0020186400204868002086
:10B4D0009474002030680020396800202DE9F04184
:10B4E000474E306801F082FF464B1B78012B78D025
:10B4F0005FD3022B0AD1DFF82C81082388F80030B3
:10B500000D254FF4C373404F3B8010E0DFF81481EA
:10B510003D4F98F8003003F04003002B14BF4FF468
:10B52000F0734FF4C3733B8014BF10250D25002426
:10B5300004F11000C0B22EF02FFD013401202EF0D6
:10B540002BFDA3B2AB42F3D398F800402F4D00205F
:10B550002EF022FD20462EF01FFD2D4B1C780220E0
:10B560002EF01AFD20462EF017FD2A4B1C780320E2
:10B570002EF012FD20462EF00FFD274B1C780420E4
:10B5800004432EF009FD20462EF006FD306801F040
:10B5900033FF3A882148002132F003FB6B7833B146
:10B5A0001F4B1B7833B300236B70BDE8F081BDE8FF
:10B5B000F081A0202EF0F0FC00202EF0EDFC00F039
:10B5C0000603022BDFF85C8007D000F0050001289D
:10B5D00003D1482388F8003008E0082388F80030B9
:10B5E0008EE7DFF84080482388F8003010254FF4BC
:10B5F000F07388E7FFF714FF00236B70BDE8F0815C
:10B6000094740020AC740020081C0020000000206E
:10B61000B3740020B474002039680020486800200A
:10B62000306800200A1C00200C4B984213D0A3F570
:10B63000806398420FD003F5804398420BD003F506
:10B640008063984207D003F58063984203D0044B8F
:10B65000186840087047024B1868704700040140A2
:10B66000C0750020F0B5774B774A87B019689142D2
:10B6700000AF00F0DB800023744A3B607B601368FE
:10B6800043F48033136003E03B68B3F5A04F09D067
:10B69000136803F400337B603B6801333B607B68D5
:10B6A000002BF1D0694B1B6813F4003318BF012342
:10B6B0007B607B68012B7BD0654D644B654AEA60FB
:10B6C0006549586F654A0860AA605E6B644C654ABC
:10B6D000654826F080065E635E6F46F080765E67A2
:10B6E000196B0C431C63596B5963996B9963196C03
:10B6F00041F05B5141F47B1141F41F6141F00F01B6
:10B700001964596C07F118040A4348F2FF715A642E
:10B7100044F8101D002621460123FB733E737E73FF
:10B72000BE732BF0E7FC21464FF6FF734F48BB601A
:10B730002BF0E0FC4FF6FF7321464D48BB602BF029
:10B74000D9FC21464B482BF0D5FC21464A482BF02A
:10B75000D1FC214649482BF0CDFC214648482BF02E
:10B76000C9FC214647482BF0C5FC214646482BF032
:10B77000C1FC20462BF0B0FE444B454C1B68BA6818
:10B7800044484549A4FB03439B09A0FB0202013B3B
:10B79000920CB3F1807F0A6007D2404AF020072163
:10B7A000536085F82300966011601C37BD46F0BDDC
:10B7B000264B3B4C1A6C3B4942F080521A6420687D
:10B7C0008A684D68C96840F4404020609868986075
:10B7D0009868120640F40040986042EA8512986822
:10B7E00042F48002490842F00802013942EA01426B
:10B7F00040F4A05098605A601A6842F080721A6053
:10B800001A689201FCD52849104A40F20570086078
:10B81000996821F003019960996841F002019960EB
:10B82000936803F00C03082BFAD145E700221A6055
:10B8300062B61E4B1B6883F308881D4B1B68984734
:10B84000FEE700BFFCFF0120EFBEADDE0038024086
:10B8500000ED00E00005FA051C950020000000083E
:10B86000FF916700335F07000000024000040240C0
:10B8700000080240000C0240001002400014024088
:10B8800000180240001C024000200240C075002049
:10B89000D34D621083DE1B43647C002010E000E087
:10B8A0000070004000000020003C02400000FF1F2C
:10B8B0000400FF1F08B5054B1B6803B19847044BF4
:10B8C000044A1A6072B6FCF78BFD00BF10600020BE
:10B8D000FCFF0120EFBEADDE08B5034B1B6803B1D2
:10B8E000984772B6FCF77CFD10600020084B10B53D
:10B8F00007281B68C8BF143818440C46007E01F0A6
:10B900002BFB20B12146BDE8104001F07BBD10BDEE
:10B91000007C002038B50C4B07281B68CCBFA0F179
:10B920001404044623440546187E01F015FB50B16B
:10B9300001342722C47182712EF0FEFB28460021BB
:10B94000BDE83840D2E738BD007C002070B50F4C10
:10B950000F4DC0EBC00004EB8004286B2669304318
:10B96000286382B09209667BA1600025012101A8AD
:10B9700063618DF804608DF805208DF806508DF810
:10B98000071024F02DFE02B070BD00BF141C002073
:10B9900000380240074BC0EBC00030B403EB80001E
:10B9A000054C0569236B2B4323630176427630BC3B
:10B9B000704700BF141C0020003802402DE9F04FF2
:10B9C0005B4C54F8204083B0002C00F0AC80E66D56
:10B9D000002E00F0AA809046564A356922609946AA
:10B9E00004F2622204F162036361A2614FF4007306
:10B9F0007268A1600746E36023616265A246B5B143
:10BA00004D4B00205A68954203F11C0376D001305B
:10BA10001028F7D100207A1CD2B20C21FFF7BAFF10
:10BA2000636DB168326922630433A1632365F068F2
:10BA3000E8B1414B00215A68904203F11C035BD0EE
:10BA400001311029F7D100257A1CD2B20B212846EA
:10BA5000FFF7A0FF2346F27F38492846FFF776FF1D
:10BA6000636DB168F26862630433E163E36494F880
:10BA7000610001F071FA054694F8600001F06CFA7B
:10BA80008346307F00284BD119F0080F38D118F0C9
:10BA9000020F09D045B10B227B1CAA71EB7128461D
:10BAA000727F222101F01EFB18F0010F15D1A36B4C
:10BAB0007BB996F82020B17F8DF8063001A8930954
:10BAC00001228DF805308DF804108DF8072024F040
:10BAD00087FD504603B0BDE8F08FBBF1000FE6D004
:10BAE00001370C238BF807708BF806305846727FAD
:10BAF000222101F0F7FADAE7CDB2A5E7C0B28AE772
:10BB00000137FFB215B10B23EF71AB7119F0100FB4
:10BB1000284614BF02211221727F01F0E3FAC6E722
:10BB20002EF0ECFAB0E7A246D3E7B246D1E700BF69
:10BB3000083E002028DD0308141C0020C1870008EF
:10BB40000348D0F8AC3113B100F5D27018477047F4
:10BB5000141C00200348D0F8903113B100F5C470D4
:10BB600018477047141C00200348D0F8743113B1F3
:10BB700000F5B67018477047141C00200348D0F831
:10BB8000583113B100F5A87018477047141C0020F5
:10BB90000348D0F83C3113B100F59A70184770474C
:10BBA000141C00200348D0F8203113B100F58C702C
:10BBB00018477047141C00200348D0F804310BB11B
:10BBC000FC301847704700BF141C00200348D0F811
:10BBD000E8300BB1E0301847704700BF141C00205C
:10BBE0000348D0F8CC300BB1C4301847704700BFC1
:10BBF000141C00200348D0F8B0300BB1A83018470F
:10BC0000704700BF141C00200348D0F894300BB1DB
:10BC10008C301847704700BF141C00200248836F07
:10BC20000BB1703018477047141C00200248C36DD8
:10BC30000BB1543018477047141C00200248036CA5
:10BC40000BB1383018477047141C00200248436A73
:10BC50000BB11C3018477047141C00200248836841
:10BC600003B11847704700BF141C00201549164B3C
:10BC700016484A6810B4CC681549B2FBF4F203FBCD
:10BC800002F30360D1F88820124B134C42F4700287
:10BC9000C1F888201A68002042F001021A609860FA
:10BCA0001A6822F0847222F480321A605C601A688A
:10BCB0004FF0006422F480221A60D8608C605DF836
:10BCC000044B70470000002040420F00C075002068
:10BCD00000ED00E00038024010300024044B4FF427
:10BCE000F07002210A225860D9609A60FFF7BEBF47
:10BCF00000000020436A8269D154436A0169426BA3
:10BD000001338B4228BF00234362002A2FD0EFF378
:10BD10001182502383F31288436B1968C9072CD40E
:10BD200070B45E686EB9456A816A8D4217D08469C5
:10BD30000C44DC600ED9691A59608562002180F8D4
:10BD40005810196841F00101D2B2196082F31188CC
:10BD500070BC70470469611A59608662EEE701237E
:10BD600080F85830D2B282F3118870BC7047426DAF
:10BD7000D36843F08003D3607047D2B282F3118856
:10BD8000704700BF026B10B462B1836CC268446933
:10BD9000D11A013B615C5DF8044B08BF1346836414
:10BDA000C8B27047016A4369C4685B5C0131A14253
:10BDB00028BF114601625DF8044BD8B2704700BF3E
:10BDC000436B13B190F858007047836A406A181AA1
:10BDD000B0FA80F040097047416A836A99420AD3F9
:10BDE000CB1A416B026961B14968501E0B44834212
:10BDF0000AD2C01A704702691144CB1A416B00295C
:10BE0000F2D1501EC01A704700207047036B43B137
:10BE1000826C5B6893422FBF981AC0689B1AC01847
:10BE20007047C269036A9A422FBFD01AC06880184F
:10BE3000C01A70470A4B30B503F1140493F900207F
:10BE40005D78072AC8BF143A811804330D7313F8BC
:10BE5000025C855413F8012C0A76A342EED130BD62
:10BE600050DD030803682DE9F041DF691FB13B464F
:10BE7000BDE8F0411847002A164611DD04460D467C
:10BE80000E4400E023689B68204698470028F9D0BC
:10BE9000236815F8011B1B6820469847AE42F1D174
:10BEA000BDE8F081002325212422017042708370B7
:10BEB000C370704710B5084B03F10C0193F90020D3
:10BEC0005C78845402449C78D470DC789471043398
:10BED0008B42F3D110BD00BF64DD030830B4846829
:10BEE00014B12368A5885D83436840F2E93001E01E
:10BEF000002833D01D89013815F0020F80B2F7D029
:10BF000089B2998140F2E93101E0002950D01889C5
:10BF1000013910F0010F89B2F7D0998940F2E93167
:10BF200001E000292FD01889013910F0020F89B2E1
:10BF3000F7D092B29A8140F2E93201E0002A4BD068
:10BF40001989013A11F0010F92B2F7D09B8914B10F
:10BF50002368A2881A83012030BC70472C498B4289
:10BF600008D0A1F578418B424CD001F580618B421D
:10BF7000D4D10220274901EB00104189013189B257
:10BF800041814189CAE7224A934208D0A2F578420A
:10BF9000934235D002F580629342D8D102211D4BE5
:10BFA00003EB01114B8901339BB24B814B89CEE7E7
:10BFB0001748834207D018498B4227D001F580618A
:10BFC0008B42ABD10221134800EB011148890130AB
:10BFD00080B248814989A1E70D498B4207D00E4ABA
:10BFE000934211D002F580629342B0D10222094BF4
:10BFF00003EB0212538901339BB253815389A6E7A5
:10C000000121CCE70120B5E70122F0E70121DAE7C1
:10C0100000300140F8A700200038004030B5044649
:10C02000406D61718389A26823F400531B041B0CCB
:10C03000838185B0A379009213F0040230D04FF4CD
:10C04000805213F00203ADF8042056D1ADF806304B
:10C050004FF480630022ADF8083011F00103ADF811
:10C060000C2028D1ADF80A3008238D07694648BF57
:10C07000ADF80A3024F0ECFAA279636DD10724D42C
:10C0800012F0080F9A8A1BD122F008021204120C37
:10C090009A829A8992B242F400529A8105B030BDD8
:10C0A00013F00203ADF8042024D04FF400551346DA
:10C0B000ADF80650CEE70423ADF80A300C23D4E7E0
:10C0C00092B242F008029A82E3E70D498B420FD008
:10C0D000A1F548418B4209D00A498B42D0D10520B5
:10C0E0000121FFF703FCA279636DC9E70220F7E79E
:10C0F0000020F5E7ADF80630ACE74FF40053A5E7B4
:10C10000001001400014014010B50446406DA160CC
:10C11000838923F400531B041B0C8381A37984B00F
:10C1200013F00402009135D04FF4805213F0020353
:10C13000ADF8042056D1ADF806304FF48063627933
:10C14000ADF80830D1074FF00003ADF80A30ADF874
:10C150000C3045BF0423ADF80A3008230C23694690
:10C16000920748BFADF80A3024F072FAA279636DE5
:10C17000D1071FD412F0080F9A8A16D122F00802B4
:10C180001204120C9A829A8992B242F400529A8155
:10C1900004B010BD13F00203ADF804201FD04FF41B
:10C1A00000511346ADF80610C9E792B242F00802FA
:10C1B0009A82E8E70D498B420FD0A1F548418B42A6
:10C1C00009D00B498B42D5D105200121FFF78EFB09
:10C1D000A279636DCEE70220F7E70020F5E7ADF81E
:10C1E0000630ACE74FF40053A5E700BF0010014054
:10C1F000001401402DE98048013085B0C3B203939B
:10C200008A4D8B4F8B4C8C4E0A230293DFF82C9275
:10C2100023F00EF84FF4FA7A4FF0100C4FF47A70C6
:10C22000D9F80430C3F30803002B40F0C180EFF3CA
:10C230001183002B40F0BC802968A26800BF2B68E6
:10C240009942F9D1D7F800E000FB0EF39B1AB3FB3B
:10C25000FEF300FB01314FF0010E0191D9F80430DB
:10C26000C3F30803002B40F08780EFF31183002B0A
:10C2700040F082802B68A16800BF2A689342F9D100
:10C28000D7F800B000FB0BF2521AB2FBFBF200FB36
:10C290000323019A9B1AB3F57A7FDFD3BAF1010A1F
:10C2A000BED1039B002B40F0BD804FF47A7ADFF8BB
:10C2B0008C9150464FF0100CD9F80430C3F30803AA
:10C2C000002B40F09280EFF31183002B40F08D8023
:10C2D0002968A26800BF2B689942F9D1D7F800E01D
:10C2E00000FB0EF39B1AB3FBFEF300FB01314FF092
:10C2F000010E0191D9F80430C3F3080303BBEFF337
:10C300001183EBB92B68A16800BF2A689342F9D169
:10C31000D7F800B000FB0BF2521AB2FBFBF200FBA5
:10C320000323019A9B1AB3F57A7FE3D3BAF1010A8A
:10C33000C2D1029B013B02937FF468AFFFF7BAFAC8
:10C34000EFF311888CF31288A1682368DB0344BFE4
:10C35000C6F800E0A1682B6832685FFA88F888F3B5
:10C360001188D7F800801A4400FB08F35B1AB3FB6E
:10C37000F8F300FB0233D4E7EFF311888CF3128853
:10C38000A1682368DB0344BFC6F800E0A1682B68FE
:10C3900032685FFA88F888F31188D7F800801A4469
:10C3A00000FB08F35B1AB3FBF8F300FB023370E702
:10C3B000EFF311828CF31288D4F808E02368D903D4
:10C3C00003D501233360D4F808E02B683168D2B27A
:10C3D00082F311883A68194400FB02F3A3EB0E03C1
:10C3E000B3FBF2F300FB013135E7EFF311828CF37D
:10C3F0001288D4F808E02368D90303D501233360F9
:10C40000D4F808E02B683168D2B282F311883A6818
:10C41000194400FB02F3A3EB0E03B3FBF2F300FBA2
:10C42000013164E7184622F071FD3EE7607C002090
:10C43000647C002010E000E05C7C002000ED00E067
:10C440002DE9F04F013085B0C3B203930B46029142
:10C450008B4C8C4E002B00F099808B4D8B4FDFF86E
:10C46000309222F0E5FE4FF4FA7A4FF0100C4FF4C0
:10C470007A70D9F80430C3F30803002B40F0DE8053
:10C48000EFF31183002B40F0D9802968A26800BF28
:10C490002B689942F9D1D7F800E000FB0EF39B1A04
:10C4A000B3FBFEF300FB01314FF0010E0191D9F80F
:10C4B0000430C3F30803002B40F08780EFF31183AF
:10C4C000002B40F082802B68A16800BF2A6893424D
:10C4D000F9D1D7F800B000FB0BF2521AB2FBFBF215
:10C4E00000FB0323019A9B1AB3F57A7FDFD3BAF1DD
:10C4F000010ABED1039B002B40F0BD804FF47A7A35
:10C50000DFF88C9150464FF0100CD9F80430C3F38B
:10C510000803002B75D1EFF31183002B71D129682B
:10C52000A26800BF2B689942F9D1D7F800E000FB60
:10C530000EF39B1AB3FBFEF300FB01314FF0010E2B
:10C540000191D9F80430C3F3080313BBEFF311834F
:10C55000FBB92B68A16800BF2A689342F9D1D7F8CC
:10C5600000B000FB0BF2521AB2FBFBF200FB0323FC
:10C57000019A9B1AB3F57A7FE3D3BAF1010AC4D1C9
:10C58000029B013B0293002B7FF467AF05B0BDE82F
:10C59000F08FEFF311888CF31288A1682368DB0316
:10C5A00044BFC6F800E0A1682B6832685FFA88F8DB
:10C5B00088F31188D7F800801A4400FB08F35B1A4F
:10C5C000B3FBF8F300FB0233D2E7EFF311888CF3EF
:10C5D0001288A1682368DB0344BFC6F800E0A168A5
:10C5E0002B6832685FFA88F888F31188D7F80080E2
:10C5F0001A4400FB08F35B1AB3FBF8F300FB0233A9
:10C6000070E7EFF311828CF31288D4F808E0236806
:10C61000D90303D501233360D4F808E02B683168CF
:10C62000D2B282F311883A68194400FB02F3A3EBFB
:10C630000E03B3FBF2F300FB01317FE7EFF311824E
:10C640008CF31288D4F808E02368D90303D50123BA
:10C650003360D4F808E02B683168D2B282F31188D5
:10C660003A68194400FB02F3A3EB0E03B3FBF2F3A9
:10C6700000FB013118E7184622F048FC3EE700BFF6
:10C6800010E000E05C7C0020607C0020647C0020E6
:10C6900000ED00E0204B5B68C3F3080330B4BBB986
:10C6A000EFF31183A3B91D4B1D4C1868A16800BF9F
:10C6B0001A689042F9D11B4B1C684FF47A7202FB46
:10C6C00004F3591AB1FBF4F130BC02FB00107047BF
:10C6D000EFF31182102383F3128811498C680B68E1
:10C6E00013F4803F104B02D0012018608C680B4976
:10C6F000D2B20D68186882F311880A4B19684FF49A
:10C700007A72284402FB01F31B1B30BCB3FBF1F32C
:10C7100002FB0030704700BF00ED00E0607C0020AD
:10C7200010E000E0647C00205C7C00202DE9F84FE4
:10C730008046FFF7AFFF254E2549DFF8A0E0254AE8
:10C74000254D844610274FF47A740120DEF804301A
:10C75000C3F30803D3B9EFF31183BBB90B68D2F865
:10C7600008A000BFD1F800904B45F7D1D6F800B033
:10C7700004FB0BF9A9EB0A09B9FBFBF904FB0393D2
:10C78000A3EB0C034345E1D3BDE8F88FEFF3118A27
:10C7900087F31288D2F808B01368DB0344BF28601F
:10C7A000D2F808B00B68D5F800905FFA8AFA8AF3DD
:10C7B0001188D6F800A0994404FB0AF3A3EB0B03FD
:10C7C000B3FBFAF304FB0933DAE700BF647C002013
:10C7D000607C002010E000E05C7C002000ED00E0C8
:10C7E0002DE9F04FDFF830C1474A4849484E494DDE
:10C7F0008046102718F1FF38C0F08480DCF8043040
:10C80000C3F30803002B5CD1EFF31183002B58D145
:10C810000B68946800BF08688342F9D1D6F800908D
:10C820004FF47A7000FB09FEAEEB040EBEFBF9FE7E
:10C8300000FB03EEDCF80430C3F308034FF47A7412
:10C840000120FBB9EFF31183E3B90B68D2F808A01C
:10C8500000BFD1F800904B45F7D1D6F800B004FBEB
:10C860000BF9A9EB0A09B9FBFBF904FB0393A3EB52
:10C870000E03B3F57A7FBDD2DCF80430C3F30803AE
:10C88000002BDFD0EFF3118A87F31288D2F808B0BB
:10C890001368DB0344BF2860D2F808B00B68D5F8F2
:10C8A00000905FFA8AFA8AF31188D6F800A09944BA
:10C8B00004FB0AF3A3EB0B03B3FBFAF304FB09330A
:10C8C000D5E7EFF3118487F31288D2F80890136844
:10C8D000D80303D501232B60D2F808900B68286891
:10C8E000E4B284F31188D6F800A04FF47A7400EB18
:10C8F000030E04FB0AF3A3EB0903B3FBFAF304FBF7
:10C900000E3E97E7BDE8F08F10E000E0607C00206D
:10C91000647C00205C7C002000ED00E030B4EFF38C
:10C920001183102282F312880649074C0A680748CF
:10C93000013200250A602560DBB2026883F31188AA
:10C9400030BC7047607C00205C7C002010E000E080
:10C9500038B5254B5C69236B73B1636D626BCAB1EB
:10C96000998A1A88C90592B201D5D20700D438BD78
:10C970004FF6F7721A8038BD636D99891A88890657
:10C9800092B2EBD59206E9D5E26ACAB1988880B234
:10C990009047E2E799891A880D0692B2E0D5100611
:10C9A000DED5A26A616A8A4219D0A1692569885CCC
:10C9B00098800132B2FBF5F105FB1122A262CFE7AC
:10C9C0009B88E2696169DBB28B54E269E068636D60
:10C9D0000132B2FBF0F100FB1122E261BEE7DA683E
:10C9E00022F08002DA60BBE7083E002038B5254B14
:10C9F0009C68236B73B1636D626BCAB1998A1A88A4
:10CA0000C90592B201D5D20700D438BD4FF6F772EE
:10CA10001A8038BD636D99891A88890692B2EBD560
:10CA20009206E9D5E26ACAB1988880B29047E2E7F7
:10CA300099891A880D0692B2E0D51006DED5A26A51
:10CA4000616A8A4219D0A1692569885C988001329F
:10CA5000B2FBF5F105FB1122A262CFE79B88E269E8
:10CA60006169DBB28B54E269E068636D0132B2FB4D
:10CA7000F0F100FB1122E261BEE7DA6822F08002E9
:10CA8000DA60BBE7083E002038B5254B1C68236BF5
:10CA900073B1636D626BCAB1998A1A88C90592B283
:10CAA00001D5D20700D438BD4FF6F7721A8038BDD1
:10CAB000636D99891A88890692B2EBD59206E9D5F9
:10CAC000E26ACAB1988880B29047E2E799891A88E9
:10CAD0000D0692B2E0D51006DED5A26A616A8A42DE
:10CAE00019D0A1692569885C98800132B2FBF5F103
:10CAF00005FB1122A262CFE79B88E2696169DBB284
:10CB00008B54E269E068636D0132B2FBF0F100FB27
:10CB10001122E261BEE7DA6822F08002DA60BBE748
:10CB2000083E002070B4EFF31186502383F312887F
:10CB3000436B1A68D20720D45D686DB9446A826A73
:10CB4000944217D081691144D9600ED9A21A5A6053
:10CB50008462002280F858201A6842F00102F1B283
:10CB60001A6081F3118870BC704701698A1A5A6093
:10CB70008562EEE7012380F85830F3B283F3118821
:10CB800070BC704703685B6A03B11847704700BF09
:10CB900003681B6A03B11847704700BF03682DE99B
:10CBA000F041DF691FB13B46BDE8F0411847002A5C
:10CBB000164611DD04460D460E4400E023689B68CE
:10CBC000204698470028F9D0236815F8011B1B68F8
:10CBD00020469847AE42F1D1BDE8F08103689B69D9
:10CBE000184700BF03685B69184700BF03681B69EB
:10CBF000184700BF0368DB68184700BF03689B68DD
:10CC0000184700BF03685B68184700BF03681B68CC
:10CC1000184700BF38B50C46097849B105460134BC
:10CC20002B6828461B68984714F8011B0029F7D188
:10CC300038BD00BF064B53F820302BB11A689B88D3
:10CC400051690B4201D1138370475383704700BF72
:10CC50002C7C002003682DE9F04F03F13F4404F5DC
:10CC60007E04604EA40A0125345D04F01F066409A9
:10CC7000032C05FA06F500F0AF80042C00F0A78025
:10CC8000022C54D08588B5FA85F0C0F11F0080B21F
:10CC9000C40803EB840400F00700266A80000F2715
:10CCA000874026EA07062662276A01F0030602FA91
:10CCB00000F0721E3843012AC1F3810CC1F3001841
:10CCC0002062C1F3411137D90024224601274FF0D9
:10CCD000030E03E0102A04F1020426D007FA02F042
:10CCE000A84302F10102F5D1D3F800C00EFA04F016
:10CCF000C04300EA0C0CC3F800C0D3F8008006FA69
:10CD000004FC4CEA080CC3F800C0D3F80CC000EADD
:10CD10000C00D860D3F80CC001FA04F040EA0C0013
:10CD2000102AD86004F10204D8D1BDE8F08F2E4C4F
:10CD3000666C35436564A5E7002002464FF0010E9E
:10CD40004FF0030904E00132102A00F102003CD048
:10CD50000EFA02F737EA0504F5D1D3F800A009FA74
:10CD600000F4E4430AEA040AC3F800A0D3F800B0D0
:10CD700006FA00FA4AEA0B0AC3F800A0D3F808A0A2
:10CD800004EA0A0AC3F808A0D3F808B00CFA00FABB
:10CD90004AEA0B0AC3F808A0D3F804A02AEA070756
:10CDA0005F60D3F804A008FA02F747EA0A075F6059
:10CDB000DF683C40DC60DF6801FA00F401323C438C
:10CDC000102ADC6000F10200C2D1BDE8F08F064CF1
:10CDD000266B3543256355E7034C266C35432564A4
:10CDE00050E700BFE40F040800380240026802F177
:10CDF0003F4303F57E032DE9F04F9B0A544DEB5C56
:10CE000003F01F055B090124032B04FA05F400F06D
:10CE10009980042B00F09180022B3ED001F0030694
:10CE2000731E012BC1F3810CC1F300188588C1F377
:10CE3000411137D90024234601274FF0030E03E0A8
:10CE4000102B04F1020426D007FA03F0A84303F1E3
:10CE50000103F5D1D2F800C00EFA04F0C04300EA95
:10CE60000C0CC2F800C0D2F8008006FA04FC4CEAB0
:10CE7000080CC2F800C0D2F80CC000EA0C00D06068
:10CE8000D2F80CC001FA04F040EA0C00102BD0607C
:10CE900004F10204D8D1BDE8F08F2E4B5D6C2C4319
:10CEA0005C64BBE7002003464FF0010E4FF003091E
:10CEB00004E00133102B00F102003CD00EFA03F71E
:10CEC00037EA0504F5D1D2F800A009FA00F4E443EA
:10CED0000AEA040AC2F800A0D2F800B006FA00FA82
:10CEE0004AEA0B0AC2F800A0D2F808A004EA0A0A2B
:10CEF000C2F808A0D2F808B00CFA00FA4AEA0B0A05
:10CF0000C2F808A0D2F804A02AEA07075760D2F8AE
:10CF100004A008FA03F747EA0A075760D7683C40BD
:10CF2000D460D76801FA00F401333C43102BD4607D
:10CF300000F10200C2D1BDE8F08F064B1D6B2C43FF
:10CF40001C636BE7034B1D6C2C431C6466E700BF3E
:10CF5000E40F04080038024010B50409013C032C1A
:10CF600017D80D4B33F8142000F00F0042FA00F3ED
:10CF700013F001030DD0012303FA00F00138104033
:10CF80002EF084F8054A064B125D104403EBC000F6
:10CF900010BD002010BD00BF101004080C100408C4
:10CFA00010B000202DE9F04F4A484B494B4B4C4CF8
:10CFB0004FF0010A4FF002094FF004084FF0080C3F
:10CFC0004FF0100E20274026802530F8022B12F05B
:10CFD000010F03D01960A3F804A0083312F0020F68
:10CFE00003D01960A3F80490083312F0040F03D0A3
:10CFF0001960A3F80480083312F0080F03D01960F9
:10D00000A3F804C0083312F0100F03D01960A3F87E
:10D0100004E0083312F0200F02D019609F8008331B
:10D0200012F0400F02D019609E80083312F0800F7A
:10D0300002D019609D80083312F4807F05D04FF430
:10D04000807B1960A3F804B0083312F4007F05D088
:10D050004FF4007B1960A3F804B0083312F4806F1A
:10D0600005D04FF4806B1960A3F804B0083312F4B4
:10D07000006F05D04FF4006B1960A3F804B00833BB
:10D0800012F4805F05D04FF4805B1960A3F804B000
:10D09000083312F4005F05D04FF4005B1960A3F869
:10D0A00004B0083312F4804F05D04FF4804B196060
:10D0B000A3F804B00833D20B04D04FF40042196037
:10D0C0009A80083301F58061A1427FF47EAFBDE80C
:10D0D000F08F00BF101004080000024010B00020C4
:10D0E0000010024000286AD003682DE9F04F03F1D8
:10D0F0003F4404F57E045F4EA40A0125345D04F02C
:10D100001F066409032C05FA06F559D0042C00F01B
:10D11000AC80022C59D08588B5FA85F0C0F11F008B
:10D1200080B2C40803EB840400F00700266A800084
:10D130000F27874026EA07062662276A01F00306C2
:10D140008240701E3A430128C1F3810CC1F30018DC
:10D150002262C1F341113DD90024224601274FF03C
:10D16000030E03E0102A04F1020426D007FA02F0AD
:10D17000A84302F10102F5D1D3F800C00EFA04F081
:10D18000C04300EA0C0CC3F800C0D3F8008006FAD4
:10D1900004FC4CEA080CC3F800C0D3F80CC000EA49
:10D1A0000C00D860D3F80CC001FA04F040EA0C007F
:10D1B000102AD86004F10204D8D1BDE8F08F70477E
:10D1C0002D4C266C35432564A5E72B4C666C354306
:10D1D0006564A0E7002002464FF0010E4FF00309FE
:10D1E00004E00132102A00F102003CD00EFA02F7EE
:10D1F00037EA0504F5D1D3F800A009FA00F4E443B6
:10D200000AEA040AC3F800A0D3F800B006FA00FA4C
:10D210004AEA0B0AC3F800A0D3F808A004EA0A0AF5
:10D22000C3F808A0D3F808B00CFA00FA4AEA0B0ACF
:10D23000C3F808A0D3F804A02AEA07075F60D3F870
:10D2400004A008FA02F747EA0A075F60DF683C407B
:10D25000DC60DF6801FA00F401323C43102ADC6034
:10D2600000F10200C2D1BDE8F08F034C266B3543BC
:10D27000256350E7E40F040800380240002855D029
:10D28000026802F13F4303F57E032DE9F04F9B0A4C
:10D29000544DEB5C03F01F055B090124032B04FADA
:10D2A00005F444D0042B00F09780022B44D001F009
:10D2B0000306731E012BC1F3810CC1F3001885888E
:10D2C000C1F341113DD90024234601274FF0030E3D
:10D2D00003E0102B04F1020426D007FA03F0A84360
:10D2E00003F10103F5D1D2F800C00EFA04F0C043F7
:10D2F00000EA0C0CC2F800C0D2F8008006FA04FC68
:10D300004CEA080CC2F800C0D2F80CC000EA0C00CD
:10D31000D060D2F80CC001FA04F040EA0C00102BE7
:10D32000D06004F10204D8D1BDE8F08F70472E4BD5
:10D330001D6C2C431C64BAE72B4B5D6C2C435C6466
:10D34000B5E7002003464FF0010E4FF0030904E05B
:10D350000133102B00F102003CD00EFA03F737EA3C
:10D360000504F5D1D2F800A009FA00F4E4430AEA72
:10D37000040AC2F800A0D2F800B006FA00FA4AEA9D
:10D380000B0AC2F800A0D2F808A004EA0A0AC2F800
:10D3900008A0D2F808B00CFA00FA4AEA0B0AC2F860
:10D3A00008A0D2F804A02AEA07075760D2F804A020
:10D3B00008FA03F747EA0A075760D7683C40D46089
:10D3C000D76801FA00F401333C43102BD46000F11C
:10D3D0000200C2D1BDE8F08F034B1D6B2C431C63D0
:10D3E00065E700BFE40F04080038024010B103688D
:10D3F00082885A83704700BF10B1036882881A83FD
:10D40000704700BF18B10368828809B95A83704712
:10D410001A8370470E4B1B8801463BB90D4B0E4AD1
:10D420001B7810680BB981F00101EBE70B4B5A69CF
:10D430001AB118B91A68106058747047084A186809
:10D440001188084A92FBF1F2012102605974704779
:10D45000387C00203A7C00203C7C0020407C00206E
:10D46000587C002020A1070010B40A4B0A4A1C78FF
:10D4700001238340234052F8200029B9B3FA83F1F5
:10D4800049095DF8044BBDE7191C18BF01215DF87F
:10D49000044BB7E7287C00202C7C002030B10368C7
:10D4A00082881B691A4214BF01200020704700BF08
:10D4B0002DE9F0410B4E346873691C400FD0DFF842
:10D4C00028800127B4FA84F3C3F11F0307FA03F598
:10D4D00058F8230003689847AC437561F2D1BDE862
:10D4E000F08100BF003C014098B100202DE9F041DF
:10D4F0000B4E346873691C400FD0DFF82880012779
:10D50000B4FA84F3C3F11F0307FA03F558F82300B4
:10D5100003689847AC437561F2D1BDE8F08100BF64
:10D52000003C014098B100202DE9F0410B4E3468D9
:10D5300073691C400FD0DFF828800127B4FA84F308
:10D54000C3F11F0307FA03F558F82300036898474F
:10D55000AC437561F2D1BDE8F08100BF003C0140F1
:10D5600098B100202DE9F0410B4E346873691C40DE
:10D570000FD0DFF828800127B4FA84F3C3F11F032A
:10D5800007FA03F558F8230003689847AC43756120
:10D59000F2D1BDE8F08100BF003C014098B100200D
:10D5A0002DE9F0410B4E346873691C400FD0DFF851
:10D5B00028800127B4FA84F3C3F11F0307FA03F5A7
:10D5C00058F8230003689847AC437561F2D1BDE871
:10D5D000F08100BF003C014098B100202DE9F041EE
:10D5E0000B4E346873691C400FD0DFF82880012788
:10D5F000B4FA84F3C3F11F0307FA03F558F82300C4
:10D6000003689847AC437561F2D1BDE8F08100BF73
:10D61000003C014098B100202DE9F0410B4E3468E8
:10D6200073691C400FD0DFF828800127B4FA84F317
:10D63000C3F11F0307FA03F558F82300036898475E
:10D64000AC437561F2D1BDE8F08100BF003C014000
:10D6500098B10020084A094808B5536C43F4804348
:10D6600053640021402230F09CFA054B4FF0FF320A
:10D670001A60C3F8032008BD0038024098B10020AA
:10D68000D8B1002003685B6A184700BF2DE9F0415C
:10D69000044618460D46164698462DF02DF8276884
:10D6A000E6722844A07229467D69434632462046E8
:10D6B000AC46BDE8F0416047036810B504461B68FE
:10D6C0009847236820469B689847A37B0133A37340
:10D6D00010BD00BF10B5036804469B689847FF2340
:10D6E00001226373227310BD08B5FFF735FC38B112
:10D6F0002C2282710022C2712021BDE80840BDE5C4
:10D7000008BD00BF40F2E93300E0A3B10289013B4C
:10D7100012F0020F9BB2F8D089B2818140F2E93356
:10D7200000E043B10289013B12F0010F9BB2F8D037
:10D730008089C0B270470C4A904209D00B4B984286
:10D7400010D003F58063984201D0FF207047022378
:10D75000074A02EB03135A89013292B25A8158895F
:10D76000C0B270470123F3E70030014000380040A9
:10D77000F8A70020144B984224D003F58063984208
:10D7800020D0028822F040021204120C028002888B
:10D7900022F038031B041B0C59B141F4807100299D
:10D7A00091FAA1F2B2FA82F108BF4FF0FF310139CC
:10D7B000C9000B439BB2038003889BB243F0400334
:10D7C000038070474908DCE700380040F0B48489E2
:10D7D0004FF6FF764FF47A7463B300293CD00F788C
:10D7E000013101E0B4421AD00589013C15F002056F
:10D7F000A4B2F7D0BCB284814FF47A7402E0BCB218
:10D80000B4420CD0058915F0010504F1FF37F6D0BC
:10D810008589ADB20AB115700132013BDCE7104BCE
:10D8200098420BD0A3F57843984217D003F5806354
:10D83000984202D00120F0BC70470225094B03EB4F
:10D8400005156B8901339BB26B81688980B200300A
:10D8500018BF0120F0BC7047FF27C5E70125EDE7A1
:10D8600000300140F8A7002070B50546806810B16F
:10D8700004688088608341F08001686840F2E93480
:10D8800000E0E4B10689013C16F0020FA4B2F8D022
:10D8900089B2818140F2E93100E029B3048901397C
:10D8A00014F0010F89B2F8D081890021FFF78EFFB3
:10D8B000AB6813B11A689B881383012070BD1649A9
:10D8C000884208D0A1F57841884221D001F58061D5
:10D8D0008842EAD10224114901EB04146189013123
:10D8E00089B261816189E0E70B4CA04207D00C4905
:10D8F00088420FD001F580618842D6D10221074CC1
:10D9000004EB01114C890134A4B24C814989CCE764
:10D910000124E0E70121F2E700300140F8A70020F0
:10D9200000380040F8B5654C0601A7190546387A5D
:10D930002CF0E4FB3B7A03F01F015B090122032B6F
:10D9400002FA01F26DD0042B66D0022B5CD0A31931
:10D9500001351879FFF700FBEDB2074610B112232D
:10D96000C5718371A3195879FFF7F6FA10B1132323
:10D97000C5718371A3199879FFF7EEFA10B11423DA
:10D98000C5718371A5190A21EA793846FFF7AAFB08
:10D990006879FFF7E1FAEA790A21FFF7A3FBA87992
:10D9A000FFF7DAFAEA790A21FFF79CFBA359444A08
:10D9B000934247D0434A934250D0434A934259D06E
:10D9C000424A934262D0424A93426BD0414A9342C8
:10D9D0002CD03444227BE2B901200222198801F4C0
:10D9E000415141F445710A4302431A809A8B22F453
:10D9F00000621204120C07219A8319821A8892B2CB
:10DA000042F040021A80F8BD334B596A0A435A6209
:10DA10009DE700200246E1E72F4B19690A431A618E
:10DA200095E72D4B196A0A431A6290E702F56442A2
:10DA30004FF40010536A43F40013536229F08EFC34
:10DA4000A359C6E702F584324FF48050536A43F479
:10DA50008053536229F082FCA359BAE702F50032E1
:10DA60004FF48040136A43F48043136229F07EFC34
:10DA7000A359AEE702F5FE324FF40040136A43F4B7
:10DA80000043136229F072FCA359A2E702F5823227
:10DA90004FF40050536A43F40053536229F05EFC84
:10DAA000A35996E702F568424FF48010536A43F495
:10DAB0008013536229F052FCA3598AE7F8A700208B
:10DAC0000030014000380040003C0040003401407C
:10DAD000005001400054014000380240427A02B92F
:10DAE000704710B504460368406804F10A0198477E
:10DAF0000023637210BD00BF437A5A1C0344D2B2A4
:10DB000042729972037A934200D802B9704710B5F5
:10DB100004460368406804F10A01984700236372D1
:10DB200010BD00BF302828D0312828D0322828D076
:10DB3000332828D0342828D0352828D0202828D0A9
:10DB4000212828D0102828D0112828D0122828D001
:10DB5000132828D0142828D0152828D0162805D016
:10DB6000172808BF0F2202D0002070470E22114B49
:10DB700003EB420393F8210070470022F7E70122EC
:10DB8000F5E70222F3E70322F1E70422EFE705229B
:10DB9000EDE70622EBE70722E9E70822E7E709229B
:10DBA000E5E70A22E3E70B22E1E70C22DFE70D229B
:10DBB000DDE700BF50DD0308F8B50468C4F30D04C9
:10DBC00005460E4604B32F6829F0CEFC092840F024
:10DBD0008780454C236923F440732361236943F410
:10DBE00000732361236943F0010323613E6029F040
:10DBF000BBFC2369092823F00103236170D12B6842
:10DC000004332B600020F8BD384B394A93422AD99F
:10DC100002F58042934225D902F58042934229D9E8
:10DC200002F58042934227D902F58032934225D9EA
:10DC300002F50032934223D902F50032934221D9F2
:10DC400002F5003293421FD902F5003293421DD9EA
:10DC500002F5802293421BD9B3F1016F1AD305203C
:10DC6000FEF7C8FA082429F07FFC092814D04FF0E9
:10DC7000FF30F8BD1024F6E71824F4E72024F2E77B
:10DC80002824F0E73024EEE73824ECE74024EAE7E4
:10DC90004824E8E75824E6E7134F3B6923F4407330
:10DCA0003B613B6943F400733B613B6923F0F8033C
:10DCB0003B613B6943F002031C433C613B6943F415
:10DCC00080333B6129F050FC3B6923F002033B6148
:10DCD0003B69092823F0F8033B613FF474AFC6E7C2
:10DCE0006FF00100F8BD00BF003C0240004000089A
:10DCF000FF3F0008F8B504460D468E180027B542D0
:10DD000001D12069F8BDE368591CE160234415F88E
:10DD1000012B1A720429F2D1206918B9A168204692
:10DD2000FFF74AFF2061E760E9E770B544880646DF
:10DD30000D46C4F30B042246002128462FF031FF84
:10DD400033690A4A934209D3094A934206D22246CA
:10DD500028461946BDE870402DF00CBC23B1214681
:10DD60002846BDE87040184770BD00BF1006000887
:10DD700012070008064B07498B4202D300231846BE
:10DD800070471A88C2F30B029042F8D01433F3E7BD
:10DD90008801000810060008024A136823EA000000
:10DDA00010607047C05A00202DE9F04F9DB0B0F9C7
:10DDB00008500D81EDB2442D00AF0C46904600F0A6
:10DDC000CC82064643D9812D00F0048200F299806E
:10DDD000542D00F0CE8040F2E9816E2D00F08B8250
:10DDE000802D40F01981BF4B93F800A00AF1020A80
:10DDF0001AF0FF0A00F09980BB4BDFF82483BB4E7A
:10DE0000DFF820B39A4403F101090A2516E0322D08
:10DE100000F0D482A5F13C00C0B2132840F2D482B5
:10DE200000232268511C216015702268D14502F13F
:10DE300001012160137078D019F8015B0A2DE6D139
:10DE4000BBF80030FF2BA8BFFF23DBB2E9E7052DAD
:10DE500000F0718220D8022D00F0838040F293817F
:10DE6000032D00F03E82042D40F0D6802A46A049C2
:10DE70002046FAF76DFF00212046FAF7B1FF22682D
:10DE80000221531C0125236028462B46743711704C
:10DE90006381BD46BDE8F08F242D60D040F204813F
:10DEA000282D00F0E081382D40F0B6800A68914BB3
:10DEB0000125511C21601570226805215019206030
:10DEC000117022680A215019206011702268002107
:10DED0005019206011702268197850192060117053
:10DEE0002268597850192060117022689978531966
:10DEF00023602B461170284674376381BD46BDE808
:10DF0000F08FA02D19D040F21381B82D00F0E781D9
:10DF1000FE2D40F08180784D05F1080635F8021B92
:10DF20002046FAF75DFFB542F8D101252B46284679
:10DF300074376381BD46BDE8F08F704B08461968A1
:10DF4000FAF736FF6E4B20461968FAF731FF6D4B32
:10DF5000196820460125FAF72BFF2B46E7E76A4BA5
:10DF6000F6E70422694920460125FAF7F1FE2B461F
:10DF7000C1E70B68664ADFF8B081581C11212060A8
:10DF8000197023681278591C21601A70236898F858
:10DF90005B20591C21601A70236898F85A20591C7C
:10DFA00021601A70B8F856102046FAF719FF0021C0
:10DFB0002046FAF715FFB8F858102046FAF710FF78
:10DFC000A8F1020508F1480635F8021F2046FAF7C5
:10DFD00007FFB542F8D122684E4B0C21501C20603F
:10DFE0005D181170226813F8011F501C9D422060BB
:10DFF0001170F7D123680222591C21601A70B8F8F9
:10E000005C102046FAF7ECFE0125B8F85E102046B9
:10E01000FAF7E6FE2B466EE72146284601F01AFF86
:10E020000346002881D1742D00F0C680772D0DD1D4
:10E030003268716891421EBF531C33601178364AB2
:10E0400008BF194620462BF09DFE6EE7F52D01F026
:10E05000AF83762D00F08981472D00F074823268FD
:10E06000392D114600F05B8300F20882212D01F06A
:10E070005F83292D40F07083531C336013780A2B83
:10E0800001F04284502B40F076853046FAF74EFE80
:10E09000DFF89880A8F800003046FAF747FE01251F
:10E0A000A8F802002B4626E7202DB5D10B681B4DA2
:10E0B000591C6A7821601A7023682A78591C2160DB
:10E0C0001A702368AA78591C21601A702989204681
:10E0D000FAF786FE23686A79591C21601A70226853
:10E0E000A979CEE6E57C002090DD030848300020C9
:10E0F000A67400204F590020087D0020107AFF1FD1
:10E10000147AFF1F187AFF1FC05A002088120408D3
:10E11000B0740020DD58002089900308D4A60020A8
:10E12000676666667030002094580020303000200A
:10E13000822D7FF471AF0B68BB4ABC4D1178BC4A8D
:10E14000581C2060197011892046FAF749FEB94B16
:10E1500022681B88FF2B02F10101A8BFFF23216069
:10E160001370A96881F3100189B22046FAF738FECE
:10E17000296801F30F0189B22046FAF731FEAE4B50
:10E18000226819787DE6012D7FF446AF0B680022E6
:10E19000591C21601A7023685A1C22601D70226865
:10E1A0002421531C23602B461170A4E6522D7FF4CA
:10E1B00033AF2268002164E63268716891421EBF65
:10E1C000531C336011789D4A08BF194620462BF036
:10E1D000D9FDAAE69A4B1E78033616F0FF063FF4E7
:10E1E000A4AE984BDFF88C821E4403F1010A4FF075
:10E1F0000A0920E0B9F1500F00F0DE80B9F1320FCA
:10E2000000F0F780A9F13C00C0B2132840F2F4807E
:10E210000025294623685A1C2260204683F8009076
:10E22000FAF7DEFD29462046FAF7DAFD56453FF4B7
:10E230007CAE1AF8019BB9F10A0FDBD1824B9D68C5
:10E24000196805EB85054FF6FF736D009D42A8BF69
:10E250001D469942A8BF194625EAE57521EAE171F4
:10E26000ADB289B2D6E70B68DFF80C92774E591C35
:10E27000022221601A7023684FF006085A1C22609F
:10E2800083F8008023680A22591C21601A702368D1
:10E2900001255A1922601D70B9F800102046FAF7BE
:10E2A0009FFDB9F802102046FAF79AFD23685A1923
:10E2B000226083F8008023685022591921601A7067
:10E2C00023680022591921601A7031882046FAF714
:10E2D00087FD71882046FAF783FD2B460BE65C4BE1
:10E2E00036E60B685A1C0A601D700B680222591C26
:10E2F00021601A705DE74F4B0A681B884B4DFF2B5E
:10E30000A8BFFF23511C21601370A96881F310017D
:10E3100089B22046FAF764FD4E4B20461988FAF779
:10E320005FFD296801F30F0189B220460125FAF744
:10E3300057FD2B46DFE50B2247492046FAF708FD3B
:10E34000082246492046FAF703FD012507224449E1
:10E350002046FAF7FDFC2B46CDE5002A3FF4E5AD5B
:10E36000404B136001252B46C5E53268511C3160D6
:10E370001278002A01F0CF82102A07BF3A4B93E8A7
:10E3800022001D4629462368581C20601A7020462A
:10E39000FAF70EFD29462046FAF70AFD334B2046D0
:10E3A0005968FAF705FD20460021FAF719FD00210A
:10E3B0002046FAF715FDFCE62D4B40E73388FF2B8E
:10E3C000A8BFFF23DBB22CE522F08EFE00283FF42D
:10E3D00027AD03780A2B25D8B0F9023088FB031249
:10E3E000DB17C3EBA2039BB2FF2BA8BFFF23DBB25B
:10E3F00017E598E8220024E722F076FE00283FF493
:10E4000007AF03780A2B3FF603AFB0F90430B0F939
:10E41000061003EB830383F3500521EAE171ADB2EB
:10E4200089B2F7E60023E2E7FE7D0020B4A40020D5
:10E43000D4A60020E87D0020907F0020319C0308B6
:10E44000E57C0020A0DD0308FC2F002030300020F8
:10E4500074400020887F0020901204089C12040859
:10E46000A812040885FD0008C42A0020E424002026
:10E4700034300020403000205C840020552D00F016
:10E480002781572D40F06881531C336012F8378B79
:10E4900007F12F010133336013F8010C01F8010F6C
:10E4A0009342F7D1DFF8A4A29AF80050002DFDD1D5
:10E4B000DFF89CB20126DBF800008AF80060FEF766
:10E4C00095FF9F4B28461E702BF066FD28462BF0CB
:10E4D00063FD09202BF060FD40462BF05DFD07F148
:10E4E0003008454607F16609A5EB0806F6B20A2092
:10E4F0002BF052FD30462BF04FFD15F8016B0B2031
:10E500002BF04AFD30462BF047FD0020FEF792FB32
:10E510004D45E9D108202BF03FFDA0202BF03CFD1C
:10E52000A0202BF039FD00202BF036FD10F020004C
:10E53000F6D106460125DBF80000FEF75DFF8AF8FC
:10E5400000602B46D7E4726835687B623046551B05
:10E55000FAF7D4FB052D38627B6A01F2C881802668
:10E56000B346012594E80600521A103A9642C8BFF5
:10E570001FFA82FB734A396A92683A61521A9345CC
:10E58000396A7B622046FA6088BF1FFA82FBFAF77D
:10E590000FFC7B6A002B01F08981002D41F0658121
:10E5A0002368C7F800D05D71C0B00533C7F804D048
:10E5B000FB61BBF1000F01F07D823B6A3A69934237
:10E5C00081F0D3823E6A7D62AA46A846BC6080255F
:10E5D000FB68A3EB08085B4BB8F5807F9B6828BFFE
:10E5E0004FF4807806EB08029A4288BFA3EB060836
:10E5F000FCF78AF87C68424621463046FCF704F96D
:10E60000F969B86104EB000C0B787B6164452ED28C
:10E61000DFF840910CF1FF3C04F1FF3E1EF8013F92
:10E6200009EB830219F823405688ECB100234FF41C
:10E63000004204F1FF3816424FEA520202D0087835
:10E64000284308706D0806D10AF1010A4D701FFABF
:10E650008AFA01318025D34503D8E64532D398455F
:10E6600030DC01339C42E6D1E645D7D1F9617B6AC3
:10E67000BA6913449BB2D3457B6206D97B6A3A6A76
:10E680009846D6183B699E42A2D3BC68802D1CBF19
:10E690000AF101031FFA83FA0AF1020189B2204646
:10E6A000FAF79EFB2368796A01255A1922602046F1
:10E6B0001D70FAF795FB2368534423602B46D7F867
:10E6C00000D018E4FB69BC681A463B7D1370DDE797
:10E6D000531C336092F80080B8F1FF0F01F0B8814D
:10E6E000B8F1FE0F01F060813046FAF71FFB96E8A3
:10E6F0000C009B1A002B07DD531C336013781BB9E9
:10E70000B8F10B0F41F28881B8F1240F00F2C985EE
:10E710000D4B012523F818002B46FFF7ECBB531CCB
:10E72000336013780A2B01F0FB803046FAF70AFBBE
:10E730003046FAF707FB3046FAF704FBFFF7F5BB64
:10E740003A680020D41D0020945800203068002032
:10E7500094740020B0DD030870680B3D831AEF2D20
:10E7600000F29F850FF2040E5EF825F0CDF400084C
:10E77000A3F20008A3F20008A3F20008A3F2000825
:10E78000A3F20008A3F20008A3F20008A3F2000815
:10E79000A3F20008A3F20008A3F20008A3F2000805
:10E7A000A3F20008A3F20008A3F20008A3F20008F5
:10E7B000A3F20008A3F20008A3F20008A3F20008E5
:10E7C000A3F20008A3F20008A3F2000843F4000833
:10E7D000A3F2000821F40008A3F20008F7F30008F0
:10E7E000A3F20008A3F20008A3F20008CFF3000888
:10E7F000A3F200084FF30008A3F200081DF300087D
:10E80000A3F20008A9F30008A3F2000843F20008ED
:10E81000A3F20008ADF20008A3F2000855F20008C8
:10E82000A3F20008A3F20008A3F20008A3F2000874
:10E830002BDF0008A3F2000801F30008A3F2000890
:10E84000A3F2000847F00008A3F200082DEB00082F
:10E85000A3F20008A3F20008A3F20008A3F2000844
:10E86000EFF00008A3F20008A3F20008A3F20008EA
:10E87000AFF00008A3F2000861F00008A3F200085E
:10E88000A3F2000801F20008A3F20008A3F20008B6
:10E89000A3F20008A3F20008A3F20008A3F2000804
:10E8A000A3F200082DF10008A3F20008D3EF00083E
:10E8B000A3F2000861EF0008A3F20008ADEE000823
:10E8C000A3F2000885EE00081FEE0008A3F200087E
:10E8D000A3F20008A3F20008A3F20008A3F20008C4
:10E8E000A3F20008A3F20008A3F20008A3F20008B4
:10E8F000A3F20008A3F20008A3F20008A3F20008A4
:10E90000A3F20008A3F20008A3F20008A3F2000893
:10E91000A3F20008A3F20008A3F20008A3F2000883
:10E92000A3F20008A3F20008A3F20008A3F2000873
:10E93000A3F20008A3F20008A3F20008A3F2000863
:10E94000A3F20008A3F20008A3F20008A3F2000853
:10E95000A3F20008A3F20008A3F20008A3F2000843
:10E96000A3F20008A3F20008A3F20008A3F2000833
:10E97000A3F20008A3F20008A3F20008A3F2000823
:10E98000A3F20008A3F20008A3F20008A3F2000813
:10E99000A3F20008A3F20008A3F20008A3F2000803
:10E9A000A3F20008A3F20008A3F20008A3F20008F3
:10E9B000A3F20008A3F20008A3F20008A3F20008E3
:10E9C000A3F20008A3F20008A3F20008A3F20008D3
:10E9D000A3F20008A3F20008A3F20008A3F20008C3
:10E9E000A3F20008A3F20008A3F20008A3F20008B3
:10E9F000A3F20008A3F20008A3F20008A3F20008A3
:10EA0000A3F20008A3F20008A3F20008A3F2000892
:10EA1000A3F20008A3F20008A3F20008F5ED000835
:10EA2000A3F2000845EF0008A3F20008A3F20008D3
:10EA3000A3F20008A3F20008A3F20008A3F2000862
:10EA4000A3F20008A3F20008A3F20008A3F2000852
:10EA5000A3F20008A3F20008A3F20008A3F2000842
:10EA600097ED000845ED00080DED0008A3F2000841
:10EA70006BEC000851EC000835EC0008A3F200082C
:10EA80001BEC0008AFEB000887EB00087DEB0008EB
:10EA9000D1F60008A3F20008A1F60008A3F20008CE
:10EAA000A3F2000877F6000849F6000835F60008DA
:10EAB0000DF60008EDF50008C3F5000897F500080D
:10EAC000A3F20008A3F20008A3F20008A3F20008D2
:10EAD000A3F20008A3F20008A3F20008A3F20008C2
:10EAE000A3F20008A3F20008A3F20008A3F20008B2
:10EAF000A3F20008A3F20008A3F2000877F50008CB
:10EB0000A3F20008A3F200081DF50008A3F2000814
:10EB1000A3F20008A3F20008A3F20008A3F2000881
:10EB2000A3F20008A3F2000803F50008531C3360A9
:10EB3000C24B1278DFF844831A700023C8F8003003
:10EB40003046FAF7DBF83368D8F80020BC49BD4DF1
:10EB500010435A1CC8F8000032601B780B72304614
:10EB6000FAF7E4F828603046FAF7E0F868603046D3
:10EB7000FAF7DCF8A8603046FAF7D8F83046FAF72A
:10EB8000D5F8FFF7D2B9531C33601078060601F1AF
:10EB90006380AD4B1B78DD073FF5C7A9032828BF6D
:10EBA0000020012502F0D2F92B46FFF7A4B9531C2F
:10EBB0003360304692F800A0FAF7A0F8814630465C
:10EBC000FAF79CF805463046FAF798F88046304642
:10EBD000FAF7ACF83046FAF7A9F83046FAF7B2F887
:10EBE000BAF1000F01F02180BAF1100F7FF49DA956
:10EBF000964BC3F800905D60B8F1000F02D0944BC3
:10EC0000C3F804809349944B0222081F01251A700F
:10EC100018F086FE2B46FFF76EB98B4B1B78D80792
:10EC20003FF583A9012502F041FC02F05DFA2B4675
:10EC3000FFF761B9844B1B78DA073FF576A9874A5D
:10EC40001378012543F0040313702B46FFF753B9E3
:10EC50007D4B1B78D9073FF568A9814B4FF4C872EB
:10EC600001251A802B46FFF746B9092B40F319837B
:10EC7000DFF80C821346511CD8F80050316013F8AD
:10EC8000021B297033605378AB70D31C33609378C8
:10EC9000642B02F10401A8BF64236B713160D37847
:10ECA000642B02F10501A8BF6423AB7131601379B5
:10ECB000EB71931D33605379642B02F10701A8BFF8
:10ECC00064232B7231609379EB7002F10803336097
:10ECD000D3792B713046FAF729F872683368688166
:10ECE000D11A00290CDD591CD8F800003160521AE5
:10ECF000002A1978417203DD9A1C32605B784370F8
:10ED0000012517F0D1FF2B46FFF7F5B8554B1868D2
:10ED1000D31C014621329D1E356013F8035C0D7033
:10ED20005D1E356013F8025C4D70336013F8015CB2
:10ED30008D7003339A4201F10301ECD116F0FEFA13
:10ED4000FFF7F3B8531C336013784449002B00F0ED
:10ED50008E870B7843F00203901C0B70424D30609D
:10ED600053782B753046F9F7C9FF28603046F9F71C
:10ED7000C5FF68603046F9F7D9FF28813046F9F7BA
:10ED8000D5FF3A4AE8811378012543F00203137056
:10ED90002B46FFF7B0B8C3F34705122D00F281826E
:10EDA000C5B107F1700307F12E0A03EB4508D14600
:10EDB000A8F142083046F9F7B9FF29F8020FC84513
:10EDC000F8D12B4B3AF8022F23F8022FD145F9D175
:10EDD000112D09D8274A6B00023B1344002122322F
:10EDE00023F8021F9A42FBD1234A01231D461370C8
:10EDF000FFF781B81346511C316013F8025B336092
:10EE0000D31C507833609178002D00F0FD86012DE1
:10EE10007FF48BA810F062FD2B46FFF76CB80A4B0D
:10EE20001B7813F0010140F03C82531C33601078D2
:10EE3000012510F095FC2B46FFF75DB8AC5F002074
:10EE4000F0940020303E0020747D0020C42A002071
:10EE5000E4240020C82A0020906C0020ECA60020AA
:10EE6000E2B100205C590020F0A600208E6C00204A
:10EE70008AA200208CA20020B0A20020C05A00204C
:10EE80001C4B00201346511C31609C4913F8020BA7
:10EE9000C87033609A4953784B71D31C3360994BD7
:10EEA0009278DA7001252B46FFF725B83046F9F73E
:10EEB0003DFF3046F9F73AFF3046F9F737FF304665
:10EEC000F9F740FF3368904D1946581C2A683060A6
:10EED00011F8020B82F82C003160597882F8361054
:10EEE000D91C31609B7882F837303046F9F72AFF19
:10EEF0003046F9F727FF3046F9F724FF3046D5F8BA
:10EF00000080F9F713FFA8F83A003046D5F80080E2
:10EF1000F9F70CFF96E80C00991A0129A8F83800B7
:10EF20000ADD511C2B683160127883F82E203046A0
:10EF3000F9F708FF96E80C009B1A032B00F39C8658
:10EF40002868FBE6DFF8DC8100233046C8F8003093
:10EF5000F9F7D4FE0125C8F800002B46FEF7CBBF19
:10EF6000531C3360684DDFF8C081137888F8053092
:10EF70003046D5F80090F9F7D9FEA9F820003046C0
:10EF8000D5F80090F9F7D2FE96E80C00991A0729F7
:10EF9000A9F81E0000F31C86991A032900F30A86BB
:10EFA0009B1A002B05DD511C2B683160127883F809
:10EFB000262001F0F1FF1FF0C5F9544B1B68002B10
:10EFC00000F028862868012515F05EFE2B46FEF726
:10EFD00092BF1346511C3160DFF84C8113F8021BBD
:10EFE00088F8021033604A4953780B70D31C3360A1
:10EFF000484D93782B71131D3360D378092BA8BF2C
:10F0000009233046AB70F9F791FE96E80C00991A87
:10F010000129288005DD3046F9F788FE96E80C00C6
:10F02000E881934240F0BC8501F0B6FF3368726816
:10F030009A423EF47AAF5A1C32601B78EB7001257D
:10F040002B46FEF758BF344B03F10801501C3060CB
:10F05000127803F8012F99423EF467AF3268F5E762
:10F06000531C336092F80080B8F1110F00F219813F
:10F07000931C3360294D537805F818303046F9F762
:10F0800055FE40F6CA039842A8BF184640F2EE2348
:10F09000984205EB4801B8BF18460125A0F2EE22C0
:10F0A0002B46192092FBF0F24A70FEF724BF13465C
:10F0B000511C1B4D316013F8021B297133605378CA
:10F0C0006B713046F9F732FE336828805A1C326083
:10F0D0001B78AB713046F9F729FE336868805A1CFB
:10F0E00032601B78EB7101252B46FEF704BF01252A
:10F0F000FBF76CFB2B46FEF7FEBE00BF6C840020C6
:10F10000FC8100207C8400205C590020A45F00204A
:10F110006084002084760020EF9400205CA400200E
:10F120006442002074400020B47900203046F9F792
:10F13000FDFD054618F002FDFF283EF4F6AE3F2D1A
:10F1400000F2178507F17008002308F8403D4FEAE8
:10F15000D509414607F12F0087F82F3009F1010941
:10F1600018F0CCFC97F82F305FFA89F905F0070505
:10F170004B4505F1010503D197F83030AB4203D080
:10F180002946484618F0C6FC33687268D21A012A2C
:10F190007EF7CBAE5A1C07F17000326000221D785A
:10F1A00000F8412D18F09EFC97F82F30AB420AD0A2
:10F1B000B94B1B683BB19A79AA4204D31B681B69FF
:10F1C0000BB12846984733685A1C326040460022EB
:10F1D0001D7887F8302018F079FC97F83030AB4272
:10F1E0003EF4A3AEAC4B1B68002B3EF49EAE1B68F6
:10F1F0005B69002B3EF499AE28469847FEF795BE12
:10F20000A64B1B78012B3EF690AE1146531C336083
:10F21000DFF8AC8211F8023B88F802303160D31C71
:10F2200092F801E03360C31A012B917840F3918486
:10F230003046F9F77BFD0125A8F800002B46FEF7C4
:10F240005ABE531C3360964B12785A7501252B46D3
:10F25000FEF751BE0722B3FBF2F2C2EBC2055B1B05
:10F260001FD1D2B202F1FF395FFA89F9002A3EF4C8
:10F270005CAEDFF830A209F101091D464B1C33607A
:10F2800091F90010874B4FF0000893F902208A4251
:10F2900003F1080300F09B8308F10108B8F1060FA1
:10F2A000F3D14FF0FF352B46FEF725BE531C3360DC
:10F2B00013780E2BF5D8911C31605578032DF0D8BA
:10F2C0007948062101FB03F1431802F1030E5D7139
:10F2D000C6F800E095784554111D3160D178597019
:10F2E000511D316011799970911D31605179D9703A
:10F2F000D11D316092791A7101252B46FEF7FBBDB5
:10F300001346511C3160694913F8020B8870336051
:10F3100053784B7001252B46FEF7EDBD644D05F18A
:10F3200040083046F9F702FD3368A5F88000591C03
:10F330001A46316012F8021B85F8821032605B7841
:10F3400085F883300435A845EBD1FEF7EEBD531C9C
:10F35000534D336013782B723046F9F7E7FCA883DE
:10F360003046F9F7E3FC28833046F9F7DFFC3368D1
:10F3700068835A1C32601B78EB7473689A1A032AEC
:10F3800000F3C8833268991A052900F3B3839B1AE6
:10F39000002B7EF7CAAD531C3360137885F82130FB
:10F3A00001252B46FEF7A7BD511C316015781F2D96
:10F3B0003FF677AF052B7FF474AF3046F9F79EFC2C
:10F3C0003B4B43F825001DF051F9FEF7AEBD531C31
:10F3D0003360384915780D70C31A002B7EF7A5AD40
:10F3E000931C33605378003318BF012301254B7001
:10F3F0002B46FEF780BD3046F9F798FCDFF8C48055
:10F40000C8F800003046F9F791FCC8F8040030460F
:10F41000F9F78CFC0125C8F808002B46FEF76BBDF8
:10F42000DFF8A4800023C8F800303046F9F766FC06
:10F43000D8F8003001250343C8F800302B46FEF70A
:10F440005ABD531C33601578132D3FF62AAF931C19
:10F45000336050787A622AF0CFFC00283FF421AF65
:10F460007A6A154B017803F82510D11C316003EB43
:10F47000850391785970111D3160D0789870501DB6
:10F4800030600E491279DA700868012517F09AFB8E
:10F490002B46FEF730BD00BFA84B0020A75A002026
:10F4A000F0940020BC74002080400020888400205C
:10F4B000347E0020AC5F0020B05F00205C5900204B
:10F4C000AA5A0020303E0020C05A0020A84A102B23
:10F4D0004FF0000128BF1023116051609160D1608E
:10F4E0001174002B3EF421AD3168013A0B44013117
:10F4F000316011F8010C02F8010F9942F7D1FEF7C3
:10F5000014BD9C4B1B78DB073FF5CBAE012501F00A
:10F5100039FD01F0E9FD2B46FEF7EDBC531C3360CD
:10F5200013780F2B3FF6BDAE911C3160C3EBC303C4
:10F5300091495078C854D01C30600B449178597070
:10F54000111D3160D1789970511D31601179D970D8
:10F55000911D316051791971D11D316091795971C5
:10F5600002F108013160D2799A71012515F0F8FA9B
:10F570002B46FEF7C0BC3046F9F7D8FBDFF8048213
:10F58000A8F80E003046F9F7D1FB0125A8F80C00C9
:10F590002B46FEF7B0BC1146531C3360774B11F875
:10F5A000020B1870316051785970D11C316091781C
:10F5B0009970111D3160D278DA7001252B46FEF763
:10F5C0009ABC3046F9F7B2FBDFF8D481A8F81000F6
:10F5D0003046F9F7ABFBA8F812003046F9F7A6FB66
:10F5E0000125A8F814002B46FEF785BC1346511CD4
:10F5F000316013F8020B3360D31C5178336092787A
:10F6000023F0BAF800287EF490AC4AE61346511C69
:10F6100031605B4913F8020B087033605949537825
:10F620008B70D31C3360584B92789A7001252B460F
:10F63000FEF761BC554B564918684E2201252BF048
:10F6400099FF2B46FEF757BC1146531C3360514BB4
:10F6500011F8020B1870316051785970D11C31606B
:10F6600092789A703046F9F761FB4B4B0125D880B0
:10F670002B46FEF740BC3046F9F758FBDFF81881FF
:10F68000A8F800003046F9F751FBA8F80200304610
:10F69000F9F74CFB0125A8F804002B46FEF72BBC1C
:10F6A000DFF8009199F80030002B3EF43EACDFF813
:10F6B000F88000253046F9F739FB13F0F1FC99F892
:10F6C0000030A8EC010A01359D42F3DBFEF72DBCAA
:10F6D0000D2B7FF4E6AD531C33601578072D3FF6F4
:10F6E000E0ADDFF8C89030464FF00C08F9F71EFB8C
:10F6F00008FB05F809EB0805A8803046F9F716FB6A
:10F70000E8803046F9F712FB336828811A46591C05
:10F71000316012F8021BA97232605B78EB723046DE
:10F72000F9F7ECFA012549F808002B46FEF7E3BB90
:10F730001346511C3160194D13F8021B6970336078
:10F7400053782B70D31C33609378AB703046F9F745
:10F75000EDFA33682881591C1A46316012F8021BF1
:10F76000697132605B78AB7101252B46FEF7C3BB34
:10F7700048840020747D0020F84400202C6600207E
:10F78000B47900206C8400207C8400205C59002027
:10F79000F4F80308648400204C420020D4A6002022
:10F7A00084760020E57C0020A44100200444002051
:10F7B000336872689A4240F0C480C14BFF221A70CD
:10F7C0004FF0000ABF4D0FF0BDFD51462022BE484C
:10F7D00085F800A02EF0E5F987F830A097F83030D2
:10F7E000072B00F25781DFF80493B74E524697F883
:10F7F000303003EB430309EBC3035B7CE3B197F8C1
:10F80000303003EB430309EBC30320215B699BB159
:10F8100097F8303003EB430309EBC303586946F80C
:10F820002200FDF72BFD2B7856F82300FDF7E4FDB1
:10F830002A780132D2B22A7097F830300133DBB225
:10F8400087F8303097F83030072BD0D92368591C0F
:10F8500021601A70B8F1000F3EF467AB9B4BC8F8FB
:10F86000003001252B46FEF746BB994B3A6A9B6850
:10F87000D4F800905A449A4200F2D980FAF744FF33
:10F880005A464946386AFAF7BFFF236803442360A3
:10F8900086427EF74AAB002100E0236801305A1C03
:10F8A000864222601970F8D1FEF73FBB002DDCD1F3
:10F8B00059462046F9F794FA23685A1C22601D70B5
:10F8C000834B26689D683B6A0BEB0302954280F0F0
:10F8D000E3803B6AED1AFAF717FF2A463146386A89
:10F8E000FAF792FF236803442360FEF71EBB3046FD
:10F8F000F9F71CFA326871687B6A9142834649D1F4
:10F9000006461D46FEF72EBE3046F9F70FFADFF821
:10F91000E081FEF7BFBB6F4B93E82200FEF733BDDB
:10F92000931C33606C4B51781970D11C3160917805
:10F930005970111D3160D2789A7001252B46FEF75F
:10F94000DABA5A1C194632605D4811F8022B02706F
:10F9500031605B784370042A03D9FF2A7EF429AC16
:10F960002EE75E490978994205D8022A7EF421AC37
:10F97000FF2B7EF41EAC236801255A1922601D70EE
:10F98000B8F1000F3EF4D1AA554BC8F800302B4611
:10F99000FEF7B1BA511C316012781D46131C0646A1
:10F9A00018BF0123FEF7DEBD931C33605578022D8E
:10F9B0003FF677AC3046F9F7B9F94A4B03EB45030C
:10F9C0004FF0FF35A3F85C002B46FEF794BA0AEB24
:10F9D000C80B30468BF80210F9F7A8F933682AF8FB
:10F9E00038001A46591C316012F8021B8BF80310BC
:10F9F00032605A788BF80420DA1C32609A788BF8DF
:10FA00000620191D31600135DB788BF80530A945DA
:10FA10007FF434ACFEF789BA324B0030984418BFFB
:10FA20000120012588F84A002B46FEF764BA3A6A9D
:10FA3000A3EB0208FAF768FE42464946386AFAF72D
:10FA4000E3FE236803442360002D3EF46EAA1FE703
:10FA5000931C3360244B51781970D31C3360DFF84A
:10FA60008480937888F85B30131D3360D37888F8EE
:10FA70005A303046F9F75AF9A8F856003046F9F7E7
:10FA800055F93046F9F752F90125A8F858002B46E8
:10FA9000FEF731BA5246D9E6FAF736FE5A463146F3
:10FAA000386AFAF7B1FE23680125034423602B4628
:10FAB000FEF721BADA46C7F824B0FEF7EDBD00BF65
:10FAC000E4240020DF42002088A30020953D0208A6
:10FAD000D41D0020846C00204F590020E57C0020BC
:10FAE00091FD000894580020B0740020C4750020D7
:10FAF0005C840020531C33601378EB723046F9F7B6
:10FB0000FDF83368E8605A1C32601B782B7496E865
:10FB10000C003CE43046F9F709F9A8843046F9F7BF
:10FB200005F996E80C00991A0329E8847FF72BACB5
:10FB30001346511C316013F8021BA97733605378C8
:10FB400085F820303046F9F7F1F896E80C00688423
:10FB500019E4504B1A88012512FB0EF22B4692FB3A
:10FB6000F1F2A8F80020FEF7C6B97D62AA46FEF7BA
:10FB700093BD07F13008404617F09CFF3B8EAB4227
:10FB80003FF402AB444B1B68002B3FF4FDAA1B68FB
:10FB90009B69002B3FF4F8AA28469847FFF7F4BA70
:10FBA000531C33601378003318BF012388F80730E3
:10FBB000FFF73ABA3046F9F7B9F8A8F80E00304620
:10FBC000F9F7B4F896E80C00A8F81000FFF7E8B9C8
:10FBD0003046F9F7ABF8A8F80A003046F9F7A6F86E
:10FBE000A8F80C003046D5F80090F9F79FF8A9F86E
:10FBF00022003046D5F80090F9F798F896E80C0006
:10FC0000A9F82400FFF7C8B9012515F005FA2B461D
:10FC1000FEF771B921482249224A234B036001258E
:10FC20000B6013602B46FEF766B9204B1020C3F81B
:10FC300000905D600DF0B6FA1D4A137843F00103A1
:10FC40001370B8F1000F3EF470A91A4B0125C3F8E8
:10FC500004802B46FEF74FB900F07F00032828BF31
:10FC6000002001250FF056FE2B46FEF744B90B7815
:10FC700003F0FD03FFF770B83046D5F80080F9F7C0
:10FC800055F8A8F8320030462E68F9F74FF8B086DC
:10FC9000FFF756B9AC820020A84B00207045002029
:10FCA000C4450020C44900206D820008846C0020F7
:10FCB000ECA60020E424002038B50B4C23688BB15F
:10FCC0005A68821A002A054604DA0CE05A68AA1A11
:10FCD000002A07DB9A68226018461A689047236852
:10FCE000002BF3D138BD38BDC85E00200B4B00227D
:10FCF00010B4027203F58474042102E0072A09DCBF
:10FD00009979890702D51979815401329C4203F10E
:10FD10001803F3D15DF8044B704700BFBC0504081D
:10FD200010B40D4C04232146002200E08B7913F01F
:10FD3000010301F1180106D101320C2AF6D103703A
:10FD40005DF8044B704702EB420204EBC2025DF81F
:10FD5000044B137903707047BC050408012310B4E9
:10FD600033213124322244704171C2700370037117
:10FD700083705DF8044B70471F22032302704370A9
:10FD8000704700BF08B513F00DFAFBF7A5FD00BFE3
:10FD9000024A034B1278197817F0DCBEE4240020E5
:10FDA000E5240020038A2DE9F0478589ADB21D4086
:10FDB00029D00F4606464FF000484FF00009B5FA2B
:10FDC00085F328FA03F2D24391B21B3B15403182EE
:10FDD000042B16D8DFE803F03129211903007B6AD0
:10FDE000002B32D003F1FF3A1FFA8AFAC7F82490A9
:10FDF0003C6A34B123682046514698476468002C19
:10FE0000F8D1002DDBD1BDE8F0873868716B03684D
:10FE100089B29847002DD2D1F5E77868B16B0368B5
:10FE200089B29847002DCAD1EDE7B868F16B036835
:10FE300089B29847002DC2D1E5E7F868316C0368B4
:10FE400089B29847002DBAD1DDE7F36A1FFA83FA29
:10FE5000CEE700BF2DE9F04F2DED028BA0F10A0394
:10FE600089B00C46E72B00F21187DFE813F01C0184
:10FE70000F070F070F070F070F070F070F070F07D2
:10FE80000F070F070F070F070F070F070F070F07C2
:10FE90000F070F070F070F070F070F070F07900533
:10FEA0000F070F070F0780050F070F070F077905CB
:10FEB0000F0719050F0700050F07F4040F07EC04DF
:10FEC0000F07C7040F07B3040F070F070F07AD0491
:10FED000A6040F0799040F070F07E6010F07BE01DD
:10FEE0000F070F070F07A2010F070F070F070F07D5
:10FEF00083010F07FC000F07E60593060F070F07A6
:10FF00000F070F070F070F070F0781030F07530393
:10FF10000F071F030F0767020F071E020F070F07C8
:10FF20000F070F07FC02BB02F502ED01E800C20358
:10FF30007E0666068F040F0758043C040F070F0760
:10FF40000F070F0731040F070F0710040F070F07E4
:10FF50000F070104F70651060E060F070F070F07DC
:10FF6000FE05B7060F0764010F070F070F070F07FE
:10FF70000F070F070F070F070F070F070F070F07D1
:10FF80000F070F070F07FC020F070F070F070F07D9
:10FF90000F070F070F070F070F070F070F070F07B1
:10FFA0000F072D010F070F070F070F070F070F0789
:10FFB0000F070F070F070F070F070F070F070F0791
:10FFC0000F070F070F070F070F070F070F070F0781
:10FFD0000F070F070F070F070F070F070F070F0771
:10FFE0000F070F070F070F070F070F070F070F0761
:10FFF0000F070F070F070F070F070F070F070F0751
:020000040801F1
:100000000F070F070F070F070F070F070F070F0740
:100010000F070F070F070F070F070F070F070F0730
:100020000F070F070F070F070F070F070F070F0720
:100030000F070F070F070F070F07DA05AF05A54ECC
:10004000337853B1A44F002537F8021F2046F8F744
:10005000C7FE33780135AB42F6DC012009B0BDECB8
:10006000028BBDE8F08F9B4E3378002BF5D09B4F71
:100070000025B846236817F81520591C21601A700E
:1000800098F8011001EB810101EB810101F2EE21F1
:1000900089B22046F8F7A4FE33780135AB4208F167
:1000A0000208E7DCD9E78E4D28462AF025FB002818
:1000B000D3DD2B460544226813F8011B501C9D42DA
:1000C00020601170F7D1C8E70B68DFF868C2591CCF
:1000D0009CF8002021601A709CF80030002BBCD0E6
:1000E000804E814D814882490023226816F8017FA5
:1000F00002F1010EC4F800E01770226815F8017FC4
:1001000002F1010EC4F800E01770226810F8017FB8
:1001100002F1010EC4F800E01770226811F8017FA7
:1001200002F1010EC4F800E017709CF800200133C2
:100130009A42DADC91E70B686E4F591C3A782160DD
:100140001A703B78002B88D00025EEB2304620F0A4
:10015000CBFF23684278591C216030461A7020F08A
:10016000C3FF01892046F8F73BFE3B780135AB42DF
:10017000EBDC72E70B68604D591C2A7921601A701C
:1001800023686A79591C21601A7029882046F8F77B
:1001900027FE2368AA79591C21601A7069882046B5
:1001A000F8F71EFE2368EA79591C216001201A70B5
:1001B00054E7FAF79BF92368504D002803F1010139
:1001C0000CBF0222032221601A7029882046F8F70A
:1001D000EFFDA9682046F8F7EBFDFAF75FF9014655
:1001E0002046F8F7E5FD012038E70B68444A454D05
:1001F0001178454A581C2060197011682046F8F79C
:10020000D7FD2368414A591C127A21601A70298847
:100210002046F8F7E5FDA9882046F8F7E1FD298991
:100220002046F8F7DDFD00212046F8F7D9FD2046ED
:100230000021F8F7D5FD012010E7084608223349D0
:10024000F8F786FD012009E7314D324E9FED328AE5
:10025000DFF8E480DFED318A05F120070EE0FCEEE7
:10026000E77ACDED017ABDF8041020460435F8F7A1
:10027000B7FDAF4206F118063FF4EFAE717C0029DE
:10028000F3D0274BD5ED007A1B78012BE7D1254B16
:100290001B68DB0440F1B885F5EE407AF1EE10FA08
:1002A00040F0E58540F2DC51DFE70B681E4A1F494C
:1002B000D0781F4A5D1C2560187023684979581C46
:1002C000206019702368D278591C216001201A70AF
:1002D000C4E600BF7CA200205E7F00205CA400205A
:1002E000488400204766002057660020776600207B
:1002F00067660020E57C002064420020D41D0020B9
:10030000AC5F0020303E0020C05A0020F094002056
:10031000805F0020C47500200000404200E082445D
:10032000A8760020D87900206C840020FC81002071
:100330007C84002045660020DB9B91410021204603
:10034000F8F74EFD00212046F8F74AFD002120462F
:10035000F8F746FD2368B94D00265A1C22601E702E
:1003600023682A68591C92F82C2021601A7023688F
:100370002A68591C92F8362021601A7023682A686E
:10038000591C92F8372021601A7023685A1C226089
:100390001E7023685A1C22601E7023685A1C22603B
:1003A0001E702B682046598FF8F71AFD2B682046DF
:1003B000198FF8F715FD23682A68591C92F82E202A
:1003C00021601A7023685A1C22601E702B68204618
:1003D000598EF8F705FD2B682046998EF8F700FD39
:1003E00001203BE6964B9B8AB3F5006F00F2158522
:1003F000B3F5806F00F23885B3F5007F34BF012775
:100400000227904D05F10C0655F8041B91FBF7F1FE
:10041000204689B2F8F7E4FCB542F5D18A4D8B4FFE
:1004200005F10C06B5EC010AD7ED087A80EE270A33
:100430002BF0AAFA81B22046F8F7D2FCAE42F1D1F5
:10044000834D05F10C0655F8041B204689B2F8F7D8
:10045000C7FCAE42F7D100E6084610227D49F8F706
:1004600077FC0120FAE500258146DFF8FC81DFF802
:10047000FCB1059504950695079501214FF6FF7A85
:1004800005E001350B2D00F0218418F9011F4F1CE8
:100490004AFA05F3F5D0DE07F3D5BBF800302B415F
:1004A000D807EED506A8F8F7D1FFEAE76A4E0B6841
:1004B0007279624D591C21601A702B682046198C84
:1004C000F8F78EFC2B682046D98BF8F789FC7189E8
:1004D0002046F8F785FCB1892046F8F781FC2B68A7
:1004E0002046598CF8F77CFC2B682046998CF8F74D
:1004F00077FCF1892046F8F773FC318A2046F8F73B
:100500006FFC2A68236892F82620591C216001207C
:100510001A70A3E5504EF378002B00F081840B682D
:100520000822591C21601A70236801229918216041
:100530001A702368494D591C2A7921601A70236862
:10054000AA78591C21601A7029882046F8F748FCBF
:10055000E9892046F8F744FC2368F279591C2160A8
:100560001A702368EA78591C216001201A7075E519
:1005700017F0E4FAFF28064600F05F8408A900257A
:1005800001F8125D0DF10D008DF80D5017F0B6FA5F
:1005900008A800F8115D17F0A5FA08A800F8105D8A
:1005A00017F094FA08A820F8085D17F083FA23687A
:1005B0005A1C22601E7023689DF80D20591C216072
:1005C0001A7023689DF80E20591C21601A70236848
:1005D0009DF80F20591C21601A7023689DF8102087
:1005E000591C21601A702046BDF81810F8F7F8FB66
:1005F00033E51B4B0A681B781A4D511C03F00203AC
:100600002160137023682A7D591C21601A702968A3
:100610002046F8F7CDFB69682046F8F7C9FB298921
:100620002046F8F7DDFBE9892046F8F7D9FB20469C
:10063000298AF8F7D5FB012010E500BF5C5900209E
:100640007CA60020B4A60020CC79002028A8002099
:10065000C0420020705F0020B47900208476002022
:10066000ECA60020F0A60020E4E103088A7F002029
:10067000AE4D08462988F8F7B3FB69882046F8F79D
:10068000AFFB2046A988F8F7ABFB0120E6E4A84DB4
:1006900005F16006A9882046F8F7A2FBE988204604
:1006A000F8F79EFB29892046F8F79AFB2368AA7A77
:1006B000591C21601A702368EA7A591C21601A704B
:1006C00055F80C1B2046F8F773FBAE42E2D1C4E4A8
:1006D000984952232268501C2060137011F8013F82
:1006E000002BF7D1B9E4944800232268056803EB96
:1006F0004301561C6D5C26601570026825680A442B
:100700006E1C527826602A70026825680A440133FC
:100710009278691C0A2B21602A70E6D19DE4874DEE
:100720000B682A68591C127821601A702B6822689D
:100730009978531C2360002311702A6821681A4499
:1007400001335279481C032B20600A70F5D12368CD
:100750002A68591C127A21601A7023682A68591C69
:10076000D27821601A7023682A68591C1279216096
:100770001A702B6820465989F8F732FB2A682368DB
:10078000527A591C21601A702A680FE00021204615
:10079000F8F70EFB20460021F8F722FB01205DE46C
:1007A0000B68674A581C917820601970236852784A
:1007B000591C216001201A7050E40B68012299181D
:1007C000216010461A7049E408460021F8F7F0FA53
:1007D000012043E45B4D5C4E05F1300795F90210B2
:1007E0005A4B93F906208A4203F1080300F0518224
:1007F0009E42F6D10835BD42F0D12EE4544B03F1B0
:100800005A0522685979501C2060117022681978A5
:10081000501C2060117022685978501C20601170A3
:1008200022689978501C206011702268D978501C79
:1008300020601170226819790633501C9D42206097
:100840001170DED109E40B68424A591C527D2160C7
:1008500001201A7002E4404D05F1800655F8041F8E
:100860002046F8F7A5FAAE42F8D1FFF7F6BB3B4DAC
:1008700005F14006B5F880102046F8F7B1FA236874
:1008800095F88220591C21601A70236895F88320FE
:100890000435591CB54221601A70EBD1FFF7DDBB5E
:1008A0002C4D0B682A7A591C21601A70A98B20469E
:1008B000F8F796FA298B2046F8F792FA698B2046CA
:1008C000F8F78EFA2368EA7C591C21601A70A98C0B
:1008D0002046F8F785FAE98C2046F8F781FA236874
:1008E000AA7F591C21601A70236895F82020591C92
:1008F00021601A70698C2046F8F772FA2368EA7A48
:10090000591C21601A70E9682046F8F751FA2368EB
:100910002A7C591C21601A70236895F82120591CE3
:10092000216001201A70FFF799BB00BF4C420020E4
:1009300004440020B4E103085C5900201C4B002053
:1009400088840020BC740020487B0020187B002095
:1009500080400020F0940020307E0020347E002073
:100960000B68AA4A581C1178206019701EE7A84D20
:1009700008462988F8F734FAA9882046F8F730FAAB
:1009800020462989F8F72CFA0120FFF767BBA14D13
:1009900005F15006287829F049FA2368027A591C93
:1009A00021601A7023686A78591C21601A702368C4
:1009B000AA78591C21601A702368EA780435591CFA
:1009C000AE4221601A70E5D1FFF747BB924B03F1AD
:1009D000700522681978501C2060117022685978BF
:1009E000501C2060117022689978501C2060117092
:1009F0002268D978501C2060117022681979501C27
:100A00002060117022685979501C20601170226892
:100A100099790733501C9D4220601170D9D1FFF79E
:100A20001CBB7E4D0846E989F8F7DAF92046A9890A
:100A3000F8F7D6F90120FFF711BB0B6800255A1C07
:100A40000A601D700B685A1C0A601D700B685A1CE6
:100A50000A60204629461D70F8F7AAF92046294663
:100A6000F8F7A6F90120FFF7F9BA6D4D0846298A73
:100A7000F8F7B6F9698A2046F8F7B2F92046A98A4C
:100A8000F8F7AEF90120FFF7E9BADFF8CCE100276B
:100A9000FEB2714600232268501C20601670226846
:100AA000501C20601370226811F8010F0133551C8F
:100AB000062B25601070EED10137062F0EF1060EC1
:100AC000E6D1584900232268501C20601770226824
:100AD000501C20601370226811F8010F0133551C5F
:100AE0000B2B25601070EED123684F4A581C07214C
:100AF0002060197023680021581C20601970236839
:100B000092F8F020591C216001201A70FFF7A6BA54
:100B10000B68464A41491078454A5D1C25601870AB
:100B200023688978581C2060197023689278591CB2
:100B3000216001201A70FFF791BA3E4D08462988BE
:100B4000F8F74EF969882046F8F74AF9B5F9043004
:100B5000394AD91782FB0323C1EBA301204689B28E
:100B6000F8F73EF90120FFF779BA344B08461988A7
:100B7000F8F736F9324B20461988F8F731F9314B3E
:100B800022681B78511C03F00103216001201370BF
:100B9000FFF764BA0B682C4E01255A1C0A601D70C1
:100BA0000B68B278591921601A7022F055F8236841
:100BB000264A27495F1927601870B1F90010B2F969
:100BC0000000F8F787FA23685A19226018703188F4
:100BD0002046F8F705F92846FFF740BA0A681D4B8A
:100BE000501C19782060117022685978501C2060C0
:100BF000117022689978501C206011702268DB788F
:100C0000511C216001201370FFF728BAAC5F00204F
:100C1000303E0020B05F0020F84400206C840020AB
:100C200084760020177F0020347E0020B4790020D5
:100C30007C840020CCA6002067666666D46C002009
:100C4000D66C00208E6C0020AA5A0020AC820020B6
:100C5000AE8200202C660020F37E00200A68A34BA1
:100C6000A3491878551C2560107022685878551CC7
:100C70002560107022689B78501C206013702046FD
:100C8000C988F8F7ADF80120FFF7E8B90020FFF7B1
:100C9000E5B923685A1C2260197029882046F8F7A4
:100CA0009FF82368EA78591C21601A7023682A7912
:100CB000591C21601A702368AA79591C21601A7086
:100CC00023686A79591C21601A7093E5DFF844A201
:100CD00000254FF008080135C5F1200208FA02F29C
:100CE000A5F120032AFA05F6164328FA03F31E435A
:100CF000252D06F001024FF000030BD01343EAD07C
:100D0000E8B215F059FF0028E5D0294606A8F8F703
:100D10009DFBE0E7774B1B78DA0700F19580002513
:100D2000754E2F4602E00135252D0DD0294630465F
:100D3000F8F79CFB0028F6D0294606A8F8F796FBA2
:100D400000285CD10137EEE76C4B6D4DB3F85010C5
:100D50002046F8F745F800212046F8F741F8694B9E
:100D600019684B0103F02002C1F340031343C1F3A0
:100D7000800243EA4203C1F3C00243EA8203C1F3A3
:100D8000401243EAC20301F0100119432046F8F76C
:100D900027F804A904222046F7F7DAFF2368297808
:100DA000594A581C2060197011886429A8BF642111
:100DB0002046F8F715F8B9F1960F4AD000212046E1
:100DC000F8F70EF82168B7F1190348BFA7F112032D
:100DD000A3F3C4034A1C226020461A460B7005A9DF
:100DE000F7F7B6FF2368494A581C10212060197094
:100DF00020461188F7F7DCFF0120FFF72FB93946AD
:100E000004A8F8F723FB9DE7F4EEC87AF1EE10FA98
:100E10004ADA4FF47A71FFF728BA0827FFF7F1BAD8
:100E20000B68B1783A4A581C206019702368127810
:100E3000591C21601A70FFF77CBB23685A1C226082
:100E400001201E70FFF70AB9069B43F001030693C9
:100E500065E723680322591C21601A7023686A78A9
:100E6000591C21601A70ADE70427FFF7CABAF4EEE7
:100E7000C87AF1EE10FA3FF515AAF4EEE87AFDEE25
:100E8000E77AF1EE10FA17EE901A20D86FF4F973A2
:100E9000303903FB01F140F2E73391FBF3F101F24A
:100EA000DB5189B2FFF7E1B9FDEEE77A40F2E732B4
:100EB00017EE903A303B02FB03F388FB0312D9177D
:100EC000C1EB622101F2E93189B2FFF7CEB940F2FC
:100ED000F313A1F5836103FB01F140F2E73391FBCA
:100EE000F3F101F2DD5189B2FFF7BFB9648400204C
:100EF0004C420020747D0020F0A700201C1E002022
:100F0000A0740020E8A60020EA3E0020B87F002060
:100F10006084002090E33FF408B501210220FCF733
:100F2000A3FA094B1B7803F00503052B08D0002119
:100F30000120FCF799FA00210846FCF795FAFEE734
:100F400012F0C2F9F3E700BF043E0020022828BFD8
:100F5000022010B4084C094B207000EB8002C0EB5B
:100F6000C20207495DF8044B013003EB4203C0B2F3
:100F70000B600CF0FFB800BFA07400206A5900207D
:100F80005C59002008B524F0A5FDF7F7C5FCBDE8C5
:100F9000084024F087BD00BF38B5484B5A8999896D
:100FA000914224BF00225A81198ADA89914224BFD2
:100FB0000022DA81DA78CAB1072A41496AD091F869
:100FC0005700404D012400210A282C709C70D971D3
:100FD0005DD00C2807D0002A6CD0DFED3B7A072AC1
:100FE0000ED00A2862D0DFED397A09E0344A92F84F
:100FF00057000A2856D00C285BD1D979DFED347A16
:10100000344C9FED350AA278002918BFF0EE407AE3
:10101000062A04D8314901EB820191ED0F0A2179AA
:1010200079B1013A032A0BD8F7EE007A87EE800AED
:101030002AF0AAFC2388984228BF1846208038BD91
:1010400038BD9B781F4A07EE103A1178B8EEC77A80
:1010500067EE277A07EE101AB8EEC77A27EE277ADE
:10106000B4EEC70AF1EE10FAEADD80EE277AFDEE63
:10107000C77A17EE903A102BA8BF1023012BB8BFE8
:101080000123DBB28B4238BF0B46137038BDDFED56
:10109000147AA4E791F857000A2803D00C28ACD0A2
:1010A000D9799AE7D979DFED0E7AA9E7DFED0D7AE4
:1010B000A6E7D979DFED047AA2E700BFB479002072
:1010C00028A80020608400206F1203396F12833A31
:1010D0000AD7A339847600206F120338B4E10308DD
:1010E0005304E9380F506E3A2DE9F047AE4FAF4E3A
:1010F00024F0F0FCBE421ED2DFF83C83DFF83C93C4
:101100004446258862197DB14A450DD2052D0BD97B
:1011100033886188C3F30B03994200F0F3801446CF
:1011200025886219002DEFD1716830461436FCF71E
:10113000FCFDBE42E4D39E4A1378A3F117010229B5
:101140000FD99C4911F83300002840F0FD80D800E9
:101150000144497829B1984911F83330002B00F047
:101160001B81964C6378022B84BF00236370237825
:10117000022B84BF00232370914B9A78042A00F03D
:10118000028132B91A88B2F5F07F84BF4FF4F07251
:101190001A808C4D8C4A2B681A40002A00F0FF8080
:1011A000D80700F1EB80590400F1E3801A0700F141
:1011B000DB809B0400F1D180844D2B685A8C998C84
:1011C000914224BF00225A84FFF7E6FE22F0A4FEDB
:1011D00010B97F480AF038FB4FF40070FCF7DCFDD3
:1011E0004FF40030FCF7D8FD4FF40010FCF7D4FDAD
:1011F0004FF00070FCF7D0FD4FF08060FCF7CCFDA5
:101200006378022B06D8734A734903EB430302EB5E
:1012100083030B602378022B07D803EB83016F4A0B
:10122000C3EBC10302EB43032B6015F03DFD00212E
:1012300030226B482CF0B5FC286813F009FF694B8D
:101240002D6803F1500102E0043399427AD01A78F4
:10125000002AF9D19C78D8788442F5D26249634B50
:101260000A7028461D6016F0BDFB614B614A1E796D
:1012700061496248624B1160C825642212FB065224
:10128000604C406B31F8061C5A60002221809A6045
:10129000DA601A615A619A61DA6183F8202083F872
:1012A000212008B11AF066F9574B9FED585A1B8858
:1012B000574A9FED586A5579574C58495848086025
:1012C00006EE903AF8EEE66A1388C5EE265A07EE67
:1012D000103A53881279C4ED005A07EE903AB8EEEE
:1012E000C77A504BF8EEE77A1D725A7227EE067AEB
:1012F00067EE867ABDE8F04783ED017AC3ED007AA8
:1013000024F0D0BB63799B077FF409AF716894F830
:1013100004A03046FCF709FD3388BAEB133F04D034
:101320001436BE42FFF4ECAE05E773887068AA1F5E
:10133000C3F30B039A4204F10601A8BF1A462AF030
:1013400019F9EDE7012289E7D8000C186468002C30
:101350007FF4FEAE17241470FAE63348FCF71CFD48
:101360004020FCF719FD27E73048FCF715FD2B68F6
:101370001FE72F48FCF710FD2B6817E72D48FCF7F7
:101380000BFD2B680FE79A8AB2F57A7FBFF401AFA5
:101390004FF47A729A82FCE618231370E1E643F068
:1013A00008032B60FCE600BF100600088801000857
:1013B000AC5F0020E0070408B0FF0308A074002021
:1013C00084760020C05A0020096000025C59002089
:1013D000BC740020725A00201C4B00206A59002067
:1013E0008C2A0020B05F002048010020C02A002085
:1013F00064420020C8A70020728400207CA6002040
:10140000947F00204C630020D0280020C0C9FB48F6
:10141000EC24002017B7D138D42800204C400020FD
:101420003661023D284000200940000201600002B0
:101430000920000208600002024000080080000845
:1014400008B524F047FBF7F767FA24F02BFBFFF70A
:101450004BFE0120BDE808400BF08CBE38B50C4CAB
:101460000C4DAC4206D2616820461434FCF75DFC9A
:10147000AC42F8D3084A094B094C146000220949D0
:101480001A705A7008480860BDE838401BF0EEB882
:1014900088010008100600085C590020A074002094
:1014A0006A5900201C4B0020725A002008B5FFF733
:1014B000D5FF24F00FFBF7F72FFABDE8084024F022
:1014C000F1BA00BFF0B50C2934D8DFE801F0893358
:1014D00033335E333333343333330700048C96892C
:1014E000B2F802E01788734D24F480542404240CCD
:1014F0000484038C8488818B23F4005321F4E64117
:101500001B0409041B0C46EA0E06090C43EA0633C9
:1015100041EA0721A8429BB2A4B289B200F09E80A2
:1015200005F58065A84200F09980926884808183E7
:1015300002640384F0BD048C9589B2F802C0B2F84D
:1015400000E05C4F24F480742404240C0484038C95
:101550008688818B23F400731B0421F073011B0C1C
:1015600045EA0C04090443EA0423090CB8429BB27F
:10157000B6B241EA0E015CD04F4CA04259D09268FD
:1015800086808183C2630384F0BD048C9589B2F8A0
:1015900002C0B2F800E0474E24F010042404240CEA
:1015A0000484038C8788018B23F0200321F4E64117
:1015B0001B0409041B0C45EA0C04090C43EA041340
:1015C00041EA0E21B0429BB2BFB289B25DD03A4C23
:1015D000A0425AD092688780018382630384F0BD61
:1015E000048C9789B2F802E01688324D24F0010489
:1015F0002404240C0484038C8488018B23F00203CC
:101600001B0421F073011B0C47EA0E0709043B433E
:10161000090CA8429BB2A4B241EA060125D005F507
:101620008065A84221D0926884800183426303844C
:10163000F0BDD589148A578A23F4006343EA05254F
:101640004FF6FF332B40958826F440563C4343EA3F
:10165000052346EA04169BB2B6B290E7158A24F435
:10166000804444EA8514A4B25FE7D689158A578A74
:1016700023F00803334324F4407496883D4323F059
:1016800004032C433343A4B2CDE7D489158A568A88
:1016900023F0800343EA04134FF6BF741C40938881
:1016A00027F44067354344EA031347EA85079BB2B2
:1016B000BFB28FE700000140000401402DE9F04F68
:1016C000C822002183B08B488B4CDFF850928B4DA1
:1016D0008B4E8C4FDFF848822CF063FA8A488B4996
:1016E000DFF840E2DFF840C200221359834200F0E5
:1016F000D680B3F1804F00F0DD80AB4200F0E58092
:10170000B34200F0E480BB4200F0E380734500F098
:10171000E280634500F0E180434500F0E080DFF8BF
:101720000CA2534500F0DD800AF5806A534500F0B5
:10173000DA800AF5806A534500F0D780AAF5983A16
:10174000534500F0D4800AF5806A534500F0858047
:101750000AF5806A534508BF0D237FD01832B2F5D1
:10176000907FC2D1644C6A4E6A4F6B4D04F59078FD
:1017700002E01834A0456DD0A379002BF9D023796D
:101780004FEA131909F1FF39B9F1030F03F00F0301
:10179000EFD836F8190040FA03F2D207E9D54FF036
:1017A000010A0AFA03F3013B184029F06FFC17F80D
:1017B0000930184415EBC002DBD055F83000DFF8D3
:1017C00070E1217A00F13F4303F57E039B0A1EF886
:1017D000033003F01F0E5B09032B0AFA0EFA60D0E8
:1017E000042B69D0022B07D1DFF820E1DEF844306A
:1017F0004AEA0303CEF8443093880093B3FA83F3A4
:10180000C3F11F039BB2DA0800EB820203F0070367
:10181000D2F820E09B004FF00F0C0CFA03FC2EEAEC
:101820000C0EC2F820E0D2F820E001FA03F343EAFC
:101830000E03136269460023022218348DF8042037
:101840008DF805308DF806308DF8073025F052FC04
:10185000A04591D103B0BDE8F08F0C2309EBC30381
:101860004FF0010A93F85C3003F01F0B5B09032B68
:101870000AFA0BFA09D0042B0CD0022B7FF46EAFBE
:101880004B6C4AEA03034B6468E70B6C4AEA0303B8
:101890000B6463E70B6B4AEA03030B635EE7002309
:1018A000DCE7DFF868E0DEF840304AEA0303CEF810
:1018B0004030A1E70123D1E7DFF850E0DEF8303017
:1018C0004AEA0303CEF8303096E70223C6E7032343
:1018D000C4E70423C2E70523C0E70623BEE70723C6
:1018E000BCE70823BAE70923B8E70A23B6E70B23C6
:1018F000B4E700BFC86D0020BC0504080004004028
:1019000000080040000C0040000001400038024088
:10191000101004080C10040810B00020B4E10308F3
:10192000000401400010004000140040004001404D
:10193000E40F040801490248FEF734BA686E00203B
:101940000040014001490248FEF72CBA406E0020D9
:101950000004014001490248FEF724BA406E00200D
:101960000004014001490248FEF71CBA186E00202D
:10197000000C004001490248FEF714BAF06D002047
:101980000004004002494FF08040FEF70BBA00BF50
:10199000C86D0020F0B50468474DA30AAB426ED075
:1019A00009D8B3F5801F66D0023DAB4258D14FF045
:1019B000480E012608E0414DAB4264D00F35AB42E2
:1019C0004FD14FF0C00E04264779B0004FEA970C74
:1019D00000295CD063460227A5899F4083190CEB40
:1019E00043032F4303F1040C354DBFB245F82310D8
:1019F00045F82C20A781EFF31181502282F3128841
:101A0000821905EBC202136963B3136204338219AE
:101A100005EBC202576917B11F605369043382197D
:101A200005EBC202976917B11F60936904338219ED
:101A300005EBC202D76917B11F60D36904330027D1
:101A4000CAB21F6082F31188304405EBC000036AFC
:101A50005BB9A38923F001031B041B0CA381F0BD18
:101A6000F0BDF0BD05EB0E03D1E7A3899BB243F0B7
:101A70000103A381F0BD4FF0200E0026A4E74FF034
:101A8000700E0226A0E74FF0980E03269CE7022373
:101A9000BF0803FA07F7A389094D9BB223EA07039E
:101AA00087190CEB470CA3810CF1040345F82C10AB
:101AB00045F823209FE700BF0300100041001000FD
:101AC000C86D002010B5036883480139834282B095
:101AD00089B200F0CB80A0F58060834200F0C68020
:101AE00000F58040834200F0B88000F580608342BA
:101AF00000F0B38000F58060834200F0AE80774C48
:101B0000188824686408B4FBF2F4013CA4B282B2E1
:101B1000B3F1804F0AD07248834207D000F580604D
:101B2000834203D000F58060834202D122F070022C
:101B300092B26C48834200F0A28000F5806083423C
:101B400000F0A78022F4407200F56C4092B283420C
:101B50001A80D9621C854FD05F4A93424CD0012233
:101B60009A821A8892B242F001021A80B3F1804F31
:101B700000F099805A4A934200F0978002F5806203
:101B8000934200F0948002F58062934200F09180CD
:101B900002F58062934200F08E8002F580629342EB
:101BA00000F08B8002F57042934200F0888002F5CD
:101BB0007052934200F0858002F58062934200F0FB
:101BC000828002F5806293427FD0A2F598329342E0
:101BD0007DD002F5806293427BD002F58062934211
:101BE00008BF0D2215D002A84FF0012340F8043D94
:101BF0001EF0F6FC02B010BD0122002119869A8267
:101C00001A88394892B242F0010283421A80ADD15B
:101C10000A46364B03EBC20301A893F85D408DF8EA
:101C20000440012300228DF805308DF807308DF82F
:101C300006201EF0D5FC1B2C08D02E2CDAD12C4B04
:101C4000019301A81EF0CCFC02B010BD294B0193FA
:101C500001A81EF0C5FC02B010BD204C18882468F5
:101C6000B4FBF2F4013CA4B282B251E71B4C1888D9
:101C70002468B4FBF2F4013CA4B282B256E701201E
:101C80001A80D9621C8598821A8892B202431A80FF
:101C900070E701201A80D9621C8598821A8892B256
:101CA00002431A8062E70122B3E70222B1E703226E
:101CB000AFE70422ADE70522ABE70622A9E707223A
:101CC000A7E70822A5E70922A3E70A22A1E70B223A
:101CD0009FE70C229DE700BF00040140C075002073
:101CE000000400400010004000000140B4E103087F
:101CF0002C010001190100012C4B98423DD0B0F19C
:101D0000804F3CD0A3F57C4398423AD003F58063E2
:101D1000984238D003F58063984236D003F580634B
:101D2000984234D003F58063984232D003F5704373
:101D3000984230D003F5705398422ED003F580635B
:101D400098422CD003F5806398422AD0A3F59833AB
:101D5000984228D003F58063984207D003F580634A
:101D6000984208BF0D2202D0002070470C22104B71
:101D700003EBC20393F85C0070470022F7E70122EF
:101D8000F5E70222F3E70322F1E70422EFE7052259
:101D9000EDE70622EBE70722E9E70822E7E7092259
:101DA000E5E70A22E3E70B22E1E700BF000001407C
:101DB000B4E103082DE9F04F2DED028B93B083467B
:101DC00020F078F9914B1D7825B113B0BDEC028B52
:101DD000BDE8F08F8E4B1B685905F6D58D4B8E4EA6
:101DE0001B6863B18D4A31681368CB1A7C2B06D906
:101DF0008B48116003780133037026F02FF8894B6C
:101E00001B78002B72D0884C884AD4F81031ABEB89
:101E10000303934201F2548394F81891B9F1000F2F
:101E200035D1DFF83C82D8F80000FAF7EBFEC0B2FB
:101E300001280FD902287E4F42F066803B78002BA4
:101E400042F0B181D4F81C31ABEB0303B3F57A6FE8
:101E500082F0EF82D4F82031002B47D094F818316B
:101E6000C3B9744B1B689B7801211E3B00228B4237
:101E700084F8181184F82C2142F29682D8F80000D8
:101E80000221043025F09CFF94F8243111E0D4F8AD
:101E900020315BB3D4F8283140F6B732ABEB030303
:101EA000934223D994F82431002B01F0F986DFF80E
:101EB000B081013BDBB284F82431002B01F0268491
:101EC000D4F8207194F82C2117F8011B94F82D31C7
:101ED000D8F80000C4F820710A44013384F82C219A
:101EE00084F82D31FAF792FEC4F828B1524B3768C6
:101EF0001B7853B1DFF86C81D8F8000028B14F4B44
:101F00001B78013B012B41F211844D4B1B7873B1BF
:101F1000DFF85481D8F800304BB13368424C02935B
:101F20001A46D4F84431D31A632B01F2B281DFF898
:101F30003C8198F80030022B01F08A863C4F97F8DC
:101F40007430032B01F0CC833E4B1B7873B13E4DB4
:101F50002B685BB1344CFAF79DFBD4F850310290FA
:101F600044F61F62C31A934200F23081374B1B784C
:101F7000002B7DD1364B1B7843B12B4CD4F8A032CB
:101F800003F5C333A0339B4581F03E82314B1B7870
:101F9000002B3FF41AAF244E2F4C304D06F2C127D0
:101FA0002068FAF72FFE00283FF40FAF2068FAF7F9
:101FB00021FE2B7880465A1E33B120682A70FAF72A
:101FC00021FE0028F2D100E703223946781E2BF0CB
:101FD000CEFD96F8C03296F8C12286F8C38283F40B
:101FE0007F4383F0FF039B1A1FFA88F89BB2B8EB7C
:101FF000132FD5D196F8C222DBB29A42D0D1781EE7
:102000001FF0ECF82B7818442870C9E72F680020DF
:10201000D8790020A8A40020607C0020C8A6002059
:10202000C4A6002056800020FC2400203F0D0300A1
:102030002000002078A6002058800020608000202A
:10204000688000207080002074800020E0800020E4
:10205000F18000207A800020808000208480002091
:1020600074A60020ACA400206CA600207EA3002053
:10207000484C2278A2B1484B9B7A53B1FAF70AFB3D
:10208000464B1B68C31AA3F57A73B3F5FA6F07D8EA
:102090002278434B43491868FAF780FD00232370E8
:1020A000414CD4F8983203F5C333A0339B45FFF479
:1020B00061AF3E4DC4F898B22B78002B41F03587C4
:1020C0003B4D2B78002B41F08D8694F89C223949AA
:1020D0008D5CEA0701F1E787AF0701F1A787680781
:1020E00002F12B802A0748D5334B344F0B9312AAA9
:1020F0001146A3F13D0241F8202D0020A3F140023A
:102100000D4603F8400C0391022311215170937086
:1021100028463968F6F726FE28467968F6F722FE43
:10212000FB89274903EBC3039B00053381FB032194
:10213000DB17C3EBA101284689B2F6F72BFE3B8AD9
:1021400003EB8303590089B22846F6F723FE1D4BA3
:10215000039D1B789B0743BF398901F57A7189B2CA
:102160004FF47A712846F6F715FE0A9B3A7D591C02
:102170000A9128461A701FF02DFF134A94F89C32DA
:102180001178013393FBF1F201FB123384F89C3296
:10219000F0E600BF48800020F0940020005F00209F
:1021A000E480002008800020FC240020E88000203B
:1021B000E9800020EC80002008800020F0A60020AC
:1021C00067666666ECA60020F080002094F8563121
:1021D000002B41F08A85DB4B1A6802F00803002BC4
:1021E0004AF60B4048F603414BF60F4349F60747C2
:1021F00004BF03460F4612F0040F4FF0190118BF39
:102200001F46900684F8561103D547F4804747F0DF
:102210002007CD4B5A79C7F30909002A42F03181D2
:102220009B79002B42F03D82984664204FF0FF3AA4
:102230004FF0000C0A970B97ADF834C0CDF83AC0B8
:10224000CDF83EC0CDF842C0CDF83090ADF8368024
:10225000ADF838A08DF846000AAF0FCFDFF800E3E5
:1022600084F805C0AEE80F0097E80F00AEE807005D
:102270002EF8023B71464FF0010C1B0CFE271F206D
:10228000C82201F81E39A770A27184F807C0E07057
:1022900094F86601207180F0F10383EA0313DAB247
:1022A000130983F0E70343EA022383EAC2031BB264
:1022B00083EA0312D2B2C3F3072383EA121343EA79
:1022C000022383EAC2031BB283F0C80282EA02122D
:1022D000D2B2C3F3072383EA121343EA022383EA49
:1022E000C2031BB283EA0C0787EA0717FFB2C3F3E6
:1022F000072282EA171242EA072200EB0C0382EA65
:10230000C7070EEB0C0084F86631278011F8013BFB
:102310007B4083EA0313DBB21A0982EA172242EAFE
:10232000032282EAC3031BB29FB281422780EDD110
:1023300083F07C0383EA0313DBB24FEA131E8EEAB9
:10234000172E8EEA032E8EEAC30E0FFA8EFE1FFAA8
:102350008EF9DFF810C2A4F800905FFA8EFE4FEA03
:10236000192984F8289084F827E00CF5C77804F13F
:10237000220ADCF80000DCF80410DCF80820DCF8A5
:102380000C3047460FC70CF1100CD445B846F0D1BD
:10239000DCF8000038606D4F9CF8043088F8043099
:1023A00007F1270884F8B5E184F8B69117F8011F02
:1023B0002868FAF72BFCB845F8D194F85731002B70
:1023C00041F08E846249326809780A2084F8570106
:1023D000002901F021865F4F01293888069042F2DA
:1023E00057810229B7F802E002F06580B8880590AD
:1023F000032902F05D81F8880490042902F06E81BF
:102400000529388902F065810629B7F80A9002F09B
:102410005C810729B7F80C8002F05481FB89039393
:1024200094F866110A920B4683F0300282EA021297
:10243000D2B217094849079387F07A0747EA02277B
:102440000988237187EAC202444FC1EB012187FB4F
:10245000013A069B4FF0000C63F30F0C059B6EF3E3
:102460001F4C4FF0000E63F30F0E049BCDF82CC0F1
:1024700012B28A440027C91763F31F4EC1EB6A2AC0
:10248000039BCDF830E082EA021160F30F070020D1
:10249000C9B268F30F00C2F3072269F31F4782EA4B
:1024A000111263F31F404FF000090D978DF83DA006
:1024B0000E908DF83C9042EA01220DF1280C82EA40
:1024C000C107BCE80F003FB287F0C80888EA0818C7
:1024D000DFF88CE084F805905FFA88F8C7F30727E7
:1024E000AEE80F0087EA181747EA08239CE80300C4
:1024F00083EAC8031BB283F023024EF8040B82EA7E
:102500000212D2B2C3F30723079F83EA1213704665
:1025100043EA022383EAC20207F1010C20F81419EE
:102520004FF023081621FE27C82384F866C12280B5
:1025300084F807800EF1020EA770E170A3711146B6
:1025400012E000BFE8A60020D4A600208B260020C1
:102550007CA20020607F0020887F0020030820806C
:1025600004250020FE24002010F8013B4B4083EAA4
:102570000313DBB21A0982EA112242EA032282EA39
:10258000C3031BB299B270452180EDD183F0F403EF
:1025900083EA0313DBB24FEA131E8EEA112E8EEA92
:1025A000032E8EEAC30E0FFA8EFE1FFA8EF8CA4F64
:1025B000A4F800804FEA182C5FFA8EFE84F81EE023
:1025C00084F81FC07968BA683868FB6807F5C7786F
:1025D000A8E80F0038697969BA6904F28F17A8E88A
:1025E000070004F2AD1884F8ADC184F8ACE117F827
:1025F000011F2868FAF70AFBB845F8D194F85A3158
:10260000002B41F07783B54B1B681922990684F89B
:102610005A2140F1FC82B24BB24F1B789A0741F12C
:1026200028873B7D042B8CBF4FF003084FF0020836
:10263000FAF730F83B8A3A890A9003EB83035B0090
:10264000ADF842304FF47A703B680C93F98997F8F3
:1026500014E07B688DF8448000FB02F24FF0000C20
:102660000AA84FF0FF398DF845E0CDF82CC0CDF821
:102670003C900E920D93ADF8401080460390B8E860
:102680000F00DFF870E2AEE80F0098E80F00AEE848
:1026900007007246182122F81C39E17194F866117E
:1026A00084F805C081F0780383EA0313D8B20309E4
:1026B00083F0F60343EA002383EAC0031BB283EAF4
:1026C0000310C0B2C3F3072383EA101343EA0023C5
:1026D00083EAC0031BB283F0C80080EA001C5FFAE3
:1026E0008CFCC3F3072080EA1C1040EA0C2080EA2F
:1026F000CC0000B280F0180383EA0313DBB2C0F30E
:10270000072080EA131040EA032080EAC30301F1A6
:1027100001081E204FF0FE0C4FF0C809E0700EF1CA
:10272000020E217184F86681238084F802C084F847
:102730000690184612F8011B414081EA0111C9B206
:102740000B0983EA102343EA012383EAC10109B29A
:1027500088B272452080EDD181F0180181EA011123
:10276000C9B20A0982EA102383EA012383EAC1037A
:102770001BB29AB2DFF860A12280DBB2120A059286
:10278000049384F8272084F82630D6460AF5C779C2
:1027900004F12208DEF80000DEF80410DEF808205C
:1027A000DEF80C30CC46ACE80F000EF1100EC6453A
:1027B000E146EFD1DEF80000CCF800009DF81030C3
:1027C000DFF8348184F8B4319DF8143084F8B531E1
:1027D000C14619F8011F2868FAF718FA424B4B4511
:1027E000F7D1F9F757FF414B414AB3F90410B7F855
:1027F00008E03B680B930A907B680C9382FB0127EF
:102800004FF47A70C9174FF0000C00FB0EF0C1EBCB
:10281000A701DDF80CE0ADF83CC0ADF83EC0ADF866
:1028200040C0ADF842100D900E90BEE80F00314F41
:1028300084F805C00FC79EE807004FF0210C87E819
:1028400007001C23C8224FF0FE0EE37084F807C077
:1028500084F802E0A27194F86611217181F06A0394
:1028600083EA0313DAB2130983F0D50343EA0223A0
:1028700083EAC2031BB283EA0312D2B2C3F3072373
:1028800083EA121343EA022383EAC2031BB283F0F2
:10289000C80282EA0212D2B2C3F3072383EA1213F8
:1028A00043EA022383EAC2031BB283EA0C0282EAF0
:1028B0000210C0B2C3F3072282EA101242EA0022D9
:1028C000013182EAC0020C3784F866112280A7F138
:1028D0001C01104612E000BFFE240020E8A60020E4
:1028E000ECA60020F0A60020B1260020CCA60020F7
:1028F00067666666042500208B26002011F8013BE0
:10290000434083EA0313DBB21A0982EA102242EA47
:10291000032282EAC3031BB298B2B9422080EDD1F0
:1029200083F0680383EA0313DBB2190981EA1022FA
:1029300082EA032282EAC3031BB29AB2DB4F2280EF
:10294000DBB24FEA122C049384F8243004F1220302
:1029500084F825C007F5C7790593FB68386879685E
:10296000BA68CE46AEE80F00059B10379F42F1468D
:10297000F3D13B88AEF800309DF81030CC4F84F88E
:10298000B231C14684F8B3C119F8011F2868FAF7BB
:102990003DF94F45F8D194F866C1C64AC64F84F850
:1029A00004C08CF0EB0383EA0313D9B20B0983F064
:1029B000C50343EA012383EAC1031BB283EA031080
:1029C000C0B2C3F3072181EA101141EA002181EA74
:1029D000C0010CCA09B281F0C80E8EEA0E1E5FFA61
:1029E0008EFE4FF000090A92C1F30721039A0B9360
:1029F000CDF8309081EA1E1343EA0E2307CA83EA1A
:102A0000CE031BB283F0310E87E807008EEA0E1E5C
:102A10005FFA8EFEC3F3072383EA1E1343EA0E23F5
:102A200083EACE0394F808E0607AA17AE27A277B01
:102A300084F805901BB28EEA030E8EEA0E1E5FFA32
:102A40008EFEC3F3072383EA1E1343EA0E2383EAB1
:102A5000CE031BB2584080EA0010C0B2C3F3072374
:102A600083EA101343EA002383EAC0031BB25940F0
:102A700081EA0110C0B2C3F3072181EA101141EAD3
:102A8000002181EAC00109B24A4082EA0212D2B2B0
:102A9000C1F3072383EA121343EA022383EAC20342
:102AA0001BB25F4087EA0717FFB2C3F3072383EA2D
:102AB000171343EA0723607BA17BE27B94F810E0C5
:102AC00094F8119083EAC7031BB2584080EA0010C3
:102AD000C0B2C3F3072383EA101343EA002383EA57
:102AE000C0031BB2594081EA0111C9B2C3F30723E5
:102AF00083EA111343EA012383EAC1031BB25A405C
:102B000082EA0212D2B2C3F3072383EA121343EA22
:102B1000022383EAC2031BB28EEA030E8EEA0E1E64
:102B20005FFA8EFEC3F3072383EA1E1343EA0E23E4
:102B300083EACE031BB289EA030989EA09195FFA1D
:102B400089F9C3F3072383EA191343EA092383EAC4
:102B5000C903A17CE27C594F1BB2594081EA0111A3
:102B6000C9B2C3F3072383EA111343EA012383EABB
:102B7000C1031BB25A4082EA0212D2B2C3F3072346
:102B800083EA121343EA022383EAC2031BB283F0EF
:102B9000270989EA0912D2B2C3F3072989EA12196F
:102BA00049EA022989EAC2090FFA89F91FFA89F26A
:102BB0000CF101034FEA122E5FFA89F931204FF030
:102BC000FE0C0C2184F86631C8232280E07184F861
:102BD00002C0E170A37184F8149084F815E0DAF86B
:102BE0000410DAF80820DAF80C30DAF80000BAF845
:102BF00010C00FC727F803CB84F8A3E184F8A29193
:102C000018F8011F2868FAF701F84745F8D194F839
:102C10005EC1BCF1000F41F07880294B94F866E169
:102C2000B3F90010B3F90220B3F904309FED256A1F
:102C3000214F84F805C007EE103A33680A938EF0EE
:102C40006A0383EA031306EE901AD9B20B0983F0E4
:102C5000D50343EA012383EAC1031BB283EA0311CC
:102C60005242C9B207EE902AC3F3072383EA111335
:102C700043EA0123F8EEE77AF8EEE66AB8EEC77A9F
:102C800083EAC1031BB267EE867A66EE866A27EE98
:102C9000067A002083F0C808CDED0C7ACDED0B6AE2
:102CA0008DED0D7A0E900F900EE000BFFE240020F7
:102CB000AF260020846C0020042500208C260020F4
:102CC000CCA6002088C3E43A109088EA08160DF1DB
:102CD0002809F6B2C3F30728B9E80F0088EA1618E6
:102CE00048EA062888EAC6080FFA88F80FC788F06D
:102CF0001E0699E8070086EA0616F6B2C8F307230F
:102D000083EA161343EA062387E8070083EAC60628
:102D1000C8214FF005084FF01E0CFE231C200EF1B9
:102D20000102A17184F85E8184F807C0A370E0708D
:102D3000A7F1100184F804E00C37268084F866219E
:102D400011F8013B734083EA0313DBB21A0982EAEC
:102D5000162242EA032282EAC3031BB29EB2B942A0
:102D60002680EDD183F0270383EA0313DBB24FEA19
:102D7000131E8EEA162E8EEA032E8EEAC30E0FFA6B
:102D80008EFE1FFA8EFCD94FA4F800C05FFA8EFEAB
:102D90004FEA1C2C84F825C084F824E007F5C77896
:102DA00004F1220938687968BA68FB6846460FC69C
:102DB00010374F45B046F5D1CD4E3B88A8F80030CE
:102DC00006F1240784F8B2E184F8B3C116F8011FB4
:102DD0002868F9F71BFFB742F8D194F85F81B8F182
:102DE000000F40F08C87C34B1B6805229B0684F8BC
:102DF0005F2141F10B81C04BDFEDC06ADA891B898D
:102E000007EE902A07EE103AF8EEE77AB8EE477A26
:102E100067EEA67A94F866C1B94BBA4AB3F90410C2
:102E2000B2F90620B84EB948CDED0B7A8CF02203EA
:102E300083EA0313DFB23B0983F0590343EA072314
:102E400083EAC703B2F5FA6F1BB2A8BF4FF4FA6268
:102E500083EA0317FFB2B2F57A7FC3F3072383EA4D
:102E60001713B8BF4FF47A724FF0640E43EA07238A
:102E7000A2F57A720EFB02F283EAC70786FB02E62E
:102E800080FB01E03FB2C917D217C2EBA612C1EB1B
:102E9000A0034FF000090AA987F0C8068DED0C7A4F
:102EA000ADF83A20ADF83830CDF82890CDF8349010
:102EB0008E4686EA0616F6B20391C7F30727BEE8E8
:102EC0000F0087EA161747EA062787EAC606904FDB
:102ED000DEF800E084F804C00FC736B286F04A037B
:102EE00083EA0313DBB2C6F3072181EA13113A46E2
:102EF00041EA03210CF1010C81EAC303142042F8DA
:102F000010E9FE264FF04A0E002184F866C14FF00A
:102F1000C80CE0702380043784F807E0A670617164
:102F200084F806C0184612F8011B414081EA0111DD
:102F3000C9B20B0983EA102343EA012383EAC101E2
:102F400009B288B2BA422080EDD181F0140181EA41
:102F50000111C9B24FEA111E8EEA102E8EEA012E1F
:102F60008EEAC10E0FFA8EFE1FFA8EF6DFF87CA1F4
:102F700026804FEA162C5FFA8EFE84F81CE084F857
:102F80001DC0DAF80410DAF80000DAF80820DAF8E0
:102F90000C30BAF818900AF5C7770FC7DAF81000A6
:102FA000DAF8141003C704F28F16A7F8009037461A
:102FB00084F8ABC184F8AAE104F2AB1917F8011F39
:102FC0002868F9F723FEB945F8D1524B524A1B78CD
:102FD0001278013B12F00100DBB214BFC021402186
:102FE000172B03D84D4A134493F830804C4B1A8862
:102FF00097071ABF002341F01001012312F4027F4A
:1030000018BF022312F0100F18BF062312F0200F72
:1030100018BF1023002841F002824FF0030C94F8EF
:1030200066E10A938EF0460383EA0313DAB21309CA
:1030300083F0920343EA022383EAC2031BB283EACA
:103040000310C0B2C3F3072282EA101242EA002240
:1030500082EAC00212B282F0C80787EA0717FFB2FD
:10306000C2F3072282EA171200238DF82FC0032033
:1030700042EA072C039A8DF82C808DF82D308DF8BC
:103080002E108DF8300007CA8CEAC70C0FFA8CFCA2
:103090001F4FE3718CEA0C1803C75FFA88F8CCF372
:1030A000072C8CEA181C4CEA082181EAC80894F81D
:1030B00008C03A700FFA88F88CEA080C8CEA0C1CED
:1030C0005FFA8CFCC8F3072282EA1C1242EA0C2247
:1030D000607AA17A94F80B80637182EACC0212B212
:1030E000504080EA001C5FFA8CFC1BE0FE240020AC
:1030F0008B260020E8A60020F0A600200AD7233C5B
:10310000CCA60020607F0020D34D62106766666603
:1031100004250020AC5F0020747D00207CE20308C1
:103120008A7F0020C2F3072080EA1C1040EA0C20AE
:1031300080EACC0000B2414081EA0111C9B2C0F37B
:10314000072282EA111242EA012282EAC10212B285
:1031500088EA020888EA08185FFA88F8C2F30722AA
:1031600082EA181242EA082294F80CC0607BA17B24
:1031700084F804E082EAC80212B28CEA020C8CEAFB
:103180000C1C5FFA8CFCC2F3072282EA1C1242EA92
:103190000C2282EACC0212B2504080EA0010C0B287
:1031A000C2F3072282EA101242EA002282EAC00237
:1031B00012B2514081EA0111C9B2C2F3072282EA78
:1031C000111242EA012282EAC102E17B94F81080E6
:1031D00013B281EA030282EA0212D2B2C3F30723D6
:1031E00083EA121343EA022383EAC2031BB288EA8A
:1031F000030282EA0212D2B2C3F3072383EA121354
:1032000043EA022383EAC2031BB283F0320282EA5A
:103210000212D2B2C3F3072383EA121343EA022352
:1032200083EAC2031BB29AB24FF0FE0C0920C821F8
:103230000EF1010EDBB284F802C04FEA122CE070EE
:10324000A17184F866E1228084F812C06374DAF810
:103250000000DAF80410DAF80820BAF80C9007F544
:10326000C07EAEE8070007F5C8778EF80280AEF89A
:10327000009084F8A0C184F89F3116F8011F2868D7
:10328000F9F7C4FCB742F8D1029BC4F85031FEF7FD
:103290006DBEDFF824A27C4FDFF82092412024F09D
:1032A0003BFDBAF9023087FB0320DB17C3EBA0001C
:1032B00080B224F015FDBAF9003087FB0320DB173C
:1032C000C3EBA00080B224F00BFDBAF9043087FBF9
:1032D0000320DB17C3EBA00080B224F001FD99F8B6
:1032E0000010D8F80000F9F791FC94F848A11AF002
:1032F000010700F01085654B1B689A0672D5644B78
:10330000644F1B789B0741F14B803B7D042B8CBFA6
:103310004FF0030A4FF0020A472024F0FDFC386802
:1033200024F0AAFC786824F0A7FCFB895A4AD8F854
:103330000000A2FB0323C3F3471319460393F9F7D5
:1033400065FC3A8999F80010039B64204B4000FB10
:1033500002F089F8003024F08FFC3F7DD8F800009F
:103360004AEA8707FFB23946F9F750FC99F800306E
:10337000D8F800005F40394689F80070F9F746FC3C
:1033800094F848A1BAF1000F2CD1444F4F2024F0FB
:10339000C3FC386824F070FC786824F06DFC50465B
:1033A00024F06AFC0121D8F80000F9F72FFC384A14
:1033B00099F800301778D8F8000007F0010739466F
:1033C00083F0010389F80030F9F720FC99F8003008
:1033D000D8F800005F40394689F80070F9F716FC0C
:1033E00094F848A1029B2E4AC4F844310AF1010323
:1033F000DBB2A2FB0312D20802EB8202A3EB420370
:1034000084F84831FEF793BD94F8A432254AC4F8F5
:10341000A0B202EB8302926C42B312AD04F2AB2372
:10342000214E45F8203D002104F2BD2331800B934D
:1034300080211523A52784F8AA32284684F8A912EA
:1034400084F8A872904728463188F5F7C9FC0A9D90
:10345000164804F52A716D1A152DA8BF15252A46A0
:1034600028F088F8124A94F8A4321570114A0133F2
:1034700082FB0312A2EBE37202EB42029B1A84F876
:10348000A432FEF783BD00BF67666666E8A600202B
:10349000ECA60020F0A600201F85EB51846C0020D4
:1034A000CDCCCCCC7CE20308C47F0020C05D0020E2
:1034B000D55D002056555555CCA6002070A600209D
:1034C000C24AC34BD4F8141130681B8892F80BE041
:1034D000C04A401A4FF47A71DFB201FB0EF11B0AA9
:1034E0009777177588424FF00007D3775375977019
:1034F000177180F0F784B849DFF808C30B68896852
:10350000B648B74F007897F814A08CFB03E8DB1798
:103510008CFB01EC4FEAE17EC3EBA80111770912A5
:10352000CEEBAC0E5177F4214FEA2E2C82F820E03E
:1035300091764FF0010E302182F81BE082F82210C4
:10354000A84B82F821C04FF0750E782182F823E055
:1035500082F82410820783F81AA040F1BF84D7F8BC
:1035600000C0A14AD7F804E0A04882FB0C194FEA3A
:10357000EC7182FB0E82C1EBA9514FEAEE79C9EBE7
:10358000A25200FB01C9029200FB02E009EB4909CB
:10359000974A4FEA490982FB0982049200EB4000F6
:1035A000934A4000039082FB0008049A9014029A08
:1035B0000490F8893F8902EB820200EBC00002EB25
:1035C000820207F5FA770692BAF1050F4FEA8002F8
:1035D0001FFA87FA0398049F029201EB81014FEAD8
:1035E000E97201EB810105914FEAE071A7EB02005E
:1035F000804F83F815A0024607FB1292059F4FEA01
:10360000A84840B200EB8709A8EB0100794F039965
:10361000804607FB1010069F77494FFA88F84FEA5B
:10362000DC7C4FEADE7E83F809C083F80EE0DFF829
:10363000D8C108EB870E029F81FB07814FEAE7782C
:10364000BCF800700397C8EBA1116C4F029187FB87
:10365000021887FB00170299DFF8B0C11FFA89F939
:103660001FFA8EFE4FEAE2724FEAE070C2EB681872
:1036700083F80A90C0EB671283F80FE04FEA19272E
:103680004FEA1E29C1F3072E0399BCF80000DF7230
:1036900083F810904FEA222783F80C805A749DF823
:1036A0000820DA714FEA282C4FEA1A2A4FEA11292A
:1036B00034BF4FF032084FF033089DF80C2083F8E8
:1036C0000DC09F7483F816A083F808E0DA7483F8BD
:1036D000149083F81B801877C4F810B1FEF79CBBD8
:1036E000DFF82C91D9F80000F9F77CFA00283EF4B5
:1036F0002BACD9F800000121F9F770FA022200235F
:1037000087F8742088F80030FEF71EBC94F82C115E
:1037100094F82D31D8F800004A1C013384F82C218C
:1037200084F82D31F9F772FAFEF7DEBB344CDFF87E
:10373000E4904FF0000A0BE01B2B00F09F820D2B52
:1037400000F079814FF0010389F80130D8F80000CA
:10375000F9F758FA00285FD0D8F80000F9F74AFACC
:1037600083B27E2B32682AD099F801100029EDD15E
:1037700094F82E21002ADFD07D2B00F0648294F88B
:103780003CE1BEF1000F04D080F02003DBB284F8EE
:103790003C11511CC9B22244092984F82E1182F827
:1037A000303100F044820829D0D8B4F83A211344CB
:1037B00003EB132303F0FF03A4F83A31C6E784F8C0
:1037C0002EA184F82FA189F801A0BFE7F07D002089
:1037D000E87D002088800020B4A40020ECA6002012
:1037E000F0A60020B48000206BCA5F6B806967FF81
:1037F00083DE1B4340420F00D34D62101F85EB5107
:10380000FC24002067666666D46C0020D66C00201D
:103810000CA400202000002094F83D3133B194F82E
:10382000313184F83D01302B00F0D78594F82F21F9
:10383000BA4BBB49DFF818A3DFF8189302954FF095
:10384000010E90464246002A00F05B833268D21B8C
:10385000012A00F21F8294F83E21002A40F03482AF
:1038600094F83FC133F81C00F0B984F83FE10A68CE
:103870009506E7D59AF800209007E3D5A94FAA4905
:10388000FA89029D4FF4F36303FB02F381FB0321EA
:10389000DB17C3EB61114FF4036024F077FA0023C8
:1038A00084F82F31FEF731BB0CF1010C5FFA8CFC70
:1038B000B0F5E06F84F83FC100F09A801BD8B0F5F6
:1038C000047F00F0498136D8B0F5887F00F0D380BE
:1038D000B0F5007F00F0B880B0F5807FB2D10A6803
:1038E0005207AFD50021029D24F050FA002384F83E
:1038F0002F31FEF70ABBB0F5026F00F05E816CD885
:10390000B0F5E46F00F08480B0F5006F00F0DD806A
:10391000B0F5E26F96D1854B029DDA6B998A6423EC
:1039200003FB02F393FBF1F124F030FA002384F857
:103930002F31FEF7EABAB0F5826F00F05581B0F58D
:10394000C06F00F02981B0F5806F7FF47BAF94F8F1
:103950004031029D0133DBB2032B00F2AF8142F212
:10396000107184F8403101FB03F1714B1B88002B6F
:1039700040F0A28101316F4B1B78DB076E4B1B8837
:1039800048BF0431DF0748BF0A31980748BF1431E8
:103990001A0648BF2831DF0548BF2831580748BFFD
:1039A00064311A0748BFC8319F0548BF01F5C87187
:1039B000980648BF01F57A71DA0648BF01F5FA6149
:1039C0005F0648BF01F57A614FF4806024F0DEF9AC
:1039D000002384F82F31FEF798BAB0F5046F1CD09D
:1039E000B0F5116F56D0B0F5036F7FF42BAF3EE703
:1039F0004E4B029D90469A6B998A642303FB02F317
:103A000093FBF1F124F0C2F984F82F81FEF77DBA1F
:103A1000464B029D90461A6CEEE7484B029DB3F967
:103A2000041001EB81019046490024F0AFF984F8BD
:103A30002F81FEF76ABA4FF0010184F82E1184F845
:103A40003031A4F83A2181E699F80620002A3FF4A3
:103A5000F9AE3B4B3B491B68029D81FB0321DB1701
:103A6000C3EBA1014FF4007024F090F9002384F817
:103A70002F31FEF74ABA0A6852077FF5E3AE0021FC
:103A80004FF48870029D24F081F9002384F82F31CF
:103A9000FEF73BBA99F80520002A3FF4D3AE2A4A34
:103AA000107800283FF4CEAE284B029D1B8803EB14
:103AB0008303590091FBF0F14FF4116024F066F993
:103AC000002384F82F31FEF720BA0A6895067FF5A7
:103AD000B9AE9AF8002090077FF5B4AE1CF0010F44
:103AE000029D104F104900F068847A6882EAE27300
:103AF000A3EBE27303EB5303A1FB0331C908002AD4
:103B0000ACBF41F0004141F040414FF4006024F06F
:103B10003DF9002384F82F31FEF7F7B97CE2030862
:103B2000E8A60020F0A600201F85EB517CA600200F
:103B3000B87F0020747D00208A7F0020CCA6002062
:103B4000B4A4002067666666FE7D0020E87D002044
:103B5000ECA60020D4A6002099F80520002A3FF406
:103B600071AEC64A107800283FF46CAEC44B029D7B
:103B70005B7B002B00F08184C24B1B8893FBF0F031
:103B800000EB800041004FF4047024F0FFF80023A4
:103B900084F82F31FEF7B9B999F80620002A3FF4CE
:103BA00051AEB94B029D99684FF4C06024F0EEF815
:103BB000002384F82F31FEF7A8B90D68AD067FF514
:103BC00041AE9AF800C01CF0020F3FF43BAEAF4F7D
:103BD000029D3B896421904601FB03F124F0D6F855
:103BE00084F82F81FEF791B90A68900640F10181AF
:103BF000A74BA64F1878397D029D00F00203002BD9
:103C00000CBF00234FF47A7340F6B83208BF4FF46C
:103C1000FA6210F0010F18BF134619444FF4826086
:103C200024F0B4F8002384F82F31FEF76EB9B4F80D
:103C30003A21C2F1FF0293427FF484AD4FF00103B9
:103C400084F83D317EE54FF0010384F83C317DE599
:103C5000F8F720FD8F4B1B68C01A40F6B833984226
:103C600000F25881DFF858A29AF804303A2B00F09D
:103C7000C782002388F80030FEF766B9D8F8000044
:103C8000F8F7C0FF00287FF45DAD4FF0010384F822
:103C90002F315BE50023029D84F82F31FEF735B903
:103CA000C4F8203184F81831DFF8188224F0BCF809
:103CB00094F82431FEF7FDB802315CE6012384F864
:103CC000403142F2107150E67349029D062023F004
:103CD00047FE002384F83E0184F82F31FEF715B922
:103CE000013B84F85731FEF789BC013B84F856311B
:103CF000FEF763BB013B84F85A31FEF788BF08F139
:103D0000FF3884F85F81FFF7BFBA0CF1FF3C84F8FD
:103D10005EC1FFF762B8614B1B88D80513D4D90682
:103D200000F17B839A0600F1DA83580600F1DC8308
:103D3000190700F1DB83DA0700F1EC8313F0020FBF
:103D40000CBF04270C27564B564A1B78D27803F039
:103D500001030AB143F002035320039323F0DCFF75
:103D6000484A128802EB820202EB8202900080B283
:103D700023F0B6FF002023F0B3FF4B4A4B491288D3
:103D8000D8F80000C2EBC212520081FB023111448C
:103D90004FEAE27ACAEB612A5FFA8AFA5146F8F7EB
:103DA00035FF99F80020039BD8F800001F438AEAEA
:103DB000020A002189F800A0F8F728FF3946D8F850
:103DC0000000F8F723FF99F80030D8F800007B4096
:103DD000DBB2194689F80030F8F718FF94F848A1CB
:103DE000FFF7D0BA32493A2023F0BAFD2870FEF727
:103DF000C1B8304A1268120600F1F782204A127BDD
:103E0000002A3FF41FAD94F84111029D032900F2EE
:103E10008383DFE801F059281902274B1B68597981
:103E20009A79DB7901F1407101EB022101EB034149
:103E3000002384F841314FF4826023F0A7FF002370
:103E400084F82F31FEF761B81C4B1A68137A507949
:103E500092781B0403EB002313444A1C84F841218D
:103E600003EB0161E7E7154B1A68D37910795278B3
:103E70001B0403EB00231344EFE700BFFE7D00208B
:103E8000F07D0020E87D0020B4A40020F0A60020F2
:103E9000ECA6002084A30020857D03088A7F0020F3
:103EA000747D0020947F0020887F002003082080FC
:103EB00035200308D87900201C4B00205C590020D5
:103EC0006CA3002074A60020BA4B1A689379D078AE
:103ED00012781B0403EB00231344BEE72D22DA768D
:103EE000FFF7FABBB44B31681B78C4F81411013BDF
:103EF000012B3FF600AB1021022391701371FFF7E5
:103F0000FABA029DFEF701B823F07EFF01233B7051
:103F1000FDF7A0BFA94AB2F84A3100210133A2F847
:103F20004A3188F80010FEF70FB8A54EA54B009354
:103F30000024A6F13F01A44BA44A089106F8404C86
:103F4000A34909960AA8F5F723F8089E731C08935D
:103F50003470089B2922591C08911A70089BEA2288
:103F6000591C08911A70089BC822591C08910AA86C
:103F70001A7026F0C1FB471C0AA93A46089827F098
:103F8000F9FA089AD31901330893D455089B5A1C9F
:103F900008921C70089B5A1C08921C70089B5A1CA3
:103FA00008921C70089B5A1C08921C70089B5A1C93
:103FB00008921C70089B5A1C08921C70089B5A1C83
:103FC00008921C70089B5A1C08921C70089B5A1C73
:103FD00008921C70089B5A1C08921C70089B5A1C63
:103FE00008921C70089BFF22591C08911A70089BAC
:103FF0000122991812A808911A7050F8283D9B1BAD
:1040000033701DF0E7FF2C70FDF7B4BFDFED717A60
:10401000B0EE677AFEF7FEBE8846894608460491F0
:1040200005918E4606910391FEF7FAB9644A6A4BF0
:104030000B9212AEA2F13D0046F8200D1988674F91
:10404000A2F1400300204FF00A0E02F8400C0822B3
:1040500083F801E030469A70F4F79CFE3B686049B3
:10406000DA1781FB0313C2EBA30399B23046F4F7CE
:1040700091FE0CF0BDF8BF680A9B3A0C591C0A91DE
:104080001A700A9B3A0A591C0A911A700A9B5A1C08
:104090000A921F700A9B5A1C0A92187030461DF033
:1040A00099FFFEF71CB84F4F9FED4F8AB7F90220DA
:1040B00043480B9007EE902AF8EEE77A12AE67EECF
:1040C000887AA0F13D01FDEEE77A46F8201D00F860
:1040D000403C0823CDED027A00F83F3C1E23BDF89A
:1040E000081000F83E3C3046F4F754FEB7F90030B3
:1040F00007EE903AF8EEE77A304667EE887AFDEE02
:10410000E77ACDED027ABDF80810F4F743FEB7F96F
:10411000043007EE903AF8EEE77A304667EE887A98
:10412000FDEEE77ACDED027ABDF80810F4F732FE25
:1041300030461DF04FFFFDF7CFBF2C4A204B1268D1
:104140000B93A3F14007002103F8401C2123D10069
:10415000BB7040F1B88126490326264B1B885A05BF
:1041600000F1A681D80700F1BC8103F00203224AC6
:10417000002B1CBF03261146DFF8808032464046E4
:1041800027F0F8F906EB080312A80133A8F10201A1
:1041900040F8203D00225B1A06F808207B701DF0D5
:1041A00019FFFDF79FBFC4F81CB187F80090FDF719
:1041B00051BE00BF5C590020907F0020FC240020ED
:1041C00008800020A674002054120408B8120408C5
:1041D000C412040800000000E87D0020B4A4002000
:1041E00067666666CCA6002058A08B41208400201C
:1041F000441004088A7F002060100408CB7F002050
:104200009AF80240C4B1013CE4B20134544451462E
:10421000002211F8013B534083EA0313DBB2120A78
:10422000DF0042EA03228C4287EA131382EA030288
:10423000EFD1002A7FF41DADBC4ABD4FBD4B1288A3
:10424000BD4CFA61DFF824931A68FA629B68B4F8EF
:104250004A21F8660021FB64D9F80000F963FA6589
:10426000F7F7D4FD029000287DF469AE0221D9F859
:104270000000F8F7B3FC94F84C319AF8032003924D
:10428000642B4FF0040287F8742040F0738194F897
:104290004D31072B04BF9DF8083084F84D3194F858
:1042A0004D31069307EB031ADAF804100291084621
:1042B00026F022FADAF8081005915FFA80FA08462B
:1042C00026F01AFAC0B204900AEB0002069B9B4843
:1042D000029902900832C27123F00F028646827260
:1042E000049803F00F0300EBCA008EF80D3052461D
:1042F0008EF80E000EF10F0027F03CF9904B049A57
:1043000005990AF10900184427F034F90298C37995
:1043100003F1010ACBB1013B5FFA83FC0CF1080CFD
:10432000DFF84CE284440023073010F8011B5940A9
:104330008B00CA0883EA410302F018024B404EFA90
:1043400002F253408445DBB2EFD17D4A03980AF86C
:10435000023020F0A9FC94F84D310022013384F89A
:104360004D3184F84C21029BDDF808A09B785BB1AD
:104370001AF80510D9F80000F8F748FC01359AF84A
:104380000230EDB2AB42F3D894F84C310322013342
:1043900084F84C3187F8742088F80020FFF7A2B920
:1043A0004FF0010AFEF7B8BF0221D8F80000F8F775
:1043B00015FC94F82431FDF77CBD3A6882EAE2737B
:1043C000A3EBE27303EB5303A1FB0331C908002AFB
:1043D000B8BF41F08041FFF798BB5A49881F23F0CE
:1043E00063FB84F83E01FFF721BA10230027042263
:1043F00018460AA9029D8DF828308DF829208DF8DD
:104400002A708DF82B708DF82C708DF82D7023F09C
:104410009DFC84F82F71FDF778BD342793E44A4A58
:10442000D278002A0CBF4FF0040C4FF0050CFEF7B9
:10443000F6BD0123D8F800003B70F8F7DBFB074618
:10444000D8F80000F8F7D6FB7B067DF403AD8A2888
:104450004ED08E287DF4FEAC94F81831002B7DF4FC
:1044600016AD3A4BC4F820312D2384F82431FDF7E2
:10447000F8BC4FF00108FEF7DBB82C4B1888FFF7AB
:104480007FBB2A499A790B8803EB830303EB8303F1
:104490004FEA83081FFA88F8002A00F01081254BA4
:1044A0001B680FFA83FA0BF0A3FE40B2FDF7C0BE03
:1044B0000326274960E698469946184604930593D3
:1044C0000393FDF7ADBF234B234A1B68234903F435
:1044D0008003002B16BF1146042603263DE6242741
:1044E00031E41F49042647E610272CE420272AE45C
:1044F0001C4B1B689F067DF5ADAC94F81831002B62
:104500007DF4C5AC184BC4F820312D2384F8243138
:10451000FDF7A7BC082716E44B1CDBB2042B84F87C
:1045200041314FEA01613FF483AC84E4E87D00202F
:1045300020000020B4A40020FC240020889D00203E
:104540008E9D002034260020947F0020888000204B
:10455000B4120408D8790020441004084810040854
:1045600058100408E8A60020B48000200CA4002005
:104570000007090E97F875A05B4904951AF00F0F14
:1045800004BF0AF1010A5FFA8AFABAF1070F28BFDD
:104590004FF0010A4FEA0A1C07EB0C03187C534B3F
:1045A00002930A18002392F82410504A93725FFA7B
:1045B0008CF31A464E4B964607EB0C024EEA00006F
:1045C00001291870D26803F101000CD90239C9B26F
:1045D0008D1C1D44034603F8012BAB424FEA122207
:1045E000F9D101310844BC4422F060030AF1010A08
:1045F0009CF811205FFA8AFA1343BAF1080F03708E
:1046000000F1010340D04FEA0A1C07EB0C01384AC5
:10461000087C354901449A1A91F8241055180EF176
:10462000100E132D5FFA8EFEC6DD049D0298DFF892
:10463000CCE0D2B2931DDBB243F04001C17103F173
:10464000010CCBB10532D3B20833C31804930EF179
:104650000100002310F8011B59408B0083EA41033D
:10466000CA084B40234902F0180241FA02F25340B3
:10467000049A8242DBB2EDD103980CF80E3087F831
:1046800075A020F011FB6EE6194A049D9A1ACDE739
:10469000984699461846049305939E460393FDF762
:1046A000BFBE154B9046B3F900A06420FDF7C0BD16
:1046B00098469946184604930393FDF7B1BE4FF010
:1046C000FF33EEE60393FDF7ABBE98460393FDF789
:1046D000A7BE984699460393FDF7A2BE9846994611
:1046E00018460393FDF79CBE7CE20308889D0020DA
:1046F000959D00200007090EB4A400208E9D002087
:104700002DE9F04F2DED0A8B3C4B1B7895B0012B1A
:10471000089001F086863A4C94F80021002A41F076
:10472000CB80072B374D01F07786002304936B680D
:1047300034489847002800F06981B5F8B470002229
:1047400085F85520002F40F04387B5F93E00AA6A4E
:10475000B5F93C60696AB5F94030DFF8B4B0821A47
:10476000E86A6A63711A1B1A2963274895F856107C
:10477000AB6316F081FEDBF80030990040F1F08069
:10478000D5ED0D5AD5ED0C7A204A94ED676AD4ED3B
:10479000686A94ED697AD4F8A8311268B8EEE58AAF
:1047A000D5ED0E5AF8EEE77AF8EEE58A013377EEAA
:1047B000867A38EE268A78EE878A9342C4ED677A45
:1047C00084ED688AC4ED698AC4F8A83101F0DC83FD
:1047D0000A4B1F78142F02F02F870023D4F8B06102
:1047E0000593062E00F2AF80DFE816F0E215A7165B
:1047F0008714BB1614005215EB1400BF047D002073
:10480000C027002028A8002058A8002014600020FD
:10481000D8790020D94B1A78D4F8B4E1DFF8CCC3AA
:104820009FEDD77A4FEACE000CEB000383ED007AC0
:10483000002A7DD0D349B0EE476AF0EE476A0023E4
:10484000F1EC017A013367EEA77A05EE903AB4EE07
:10485000E77AF1EE10FAF8EEE55AB8BFB0EE677AF3
:10486000934276EEA76AA7EEA56AE9D1F5EEC06A93
:104870000CEB0003F1EE10FA83ED007A58DDC6EE82
:10488000265AC14BC14A1288F7EE007A75EEE75AF4
:10489000D3ED007A65EEA77AFDEEE77A17EE903A4F
:1048A000812B43F3DA859342A8BF134607EE903A73
:1048B000F8EEE77AB64B00EB0E0103EB810393EDC4
:1048C000057AD3ED003A93ED066A93ED014AD3EDF4
:1048D000046AD3ED034A93ED025AA3EEA77AA4EE3D
:1048E000276A66EEC76AA7EE646ABDEEC77AE5EE90
:1048F000276A17EE101A812983ED056AC3ED066A4F
:1049000043F3A8858A42A8BF0A4607EE902AF8EE2C
:10491000E77AFCEEE77ACDED067ABDF818300CEBBD
:1049200000029380BEF1000F02D1132F04F04882E1
:10493000152F42F037846044DFF8B482838828F86A
:104940001E30D4F8B061934B013683FB06239A19CD
:10495000F317C3EBA203C3EBC303F61AC4F8B061A9
:104960008D4B1B78002B01F0AE808C4EDFF88492CB
:10497000DFF87CA206F2DC680027894BD5ED087AC7
:104980001B78172B01F09A8396ED007AB8EEC78A50
:10499000082B28EE278A07D1B0EE480A059326F0A7
:1049A000F3FF059B2AF81700DBF8002092000BD5D7
:1049B000002F04F05B85B0EE480AD5F8783708F18F
:1049C00070009847B0EE408AB0EE480AD5F89836A5
:1049D000A8F170009847D5F8083740469847704BC3
:1049E0001B78032BB0EE408A01F06283D6F85C0698
:1049F000D5F8B830B0EE480A98470137032F08F1D0
:104A00002408A9EC010A06F10406B6D1644B93F818
:104A10000090B9F1070F00F0988694F8C031002B90
:104A200040F0A0865F4B5B79002B40F0CB850123E3
:104A30005B4A84F8C0311278072A02F042800023D2
:104A40000B93594B94ED729A93ED007A574BDFF824
:104A5000A881D3F800A0564B0593F7EE007A37EE05
:104A6000C9BA544B07932BEE07BA534B0993534BD8
:104A70000693B4EEE7BA08F168030025F1EE10FAE8
:104A80000A93D4ED71BA4E4BDFF870B1DFED4D8A69
:104A90009FED4DAADFED3AAADFED4C9ADFF8609169
:104AA0004B4F049388BFB0EE67BA2E46494B98ED42
:104AB000008A2B44D3ED007AF5EE407AF1EE10FA3D
:104AC00017D0454B2B44D3ED006A38EE667AB0EE32
:104AD000C76AF4EEC67AF1EE10FA08D5B5EEC07AE0
:104AE000F1EE10FACCBF37EEA68A36EEE78A83EDF8
:104AF000008A059B1A88930700F08680022E00F03A
:104B00008380364B9AF82E1033F9163007EE103AA0
:104B10000A9B07EE901A2B44F8EEE76AB8EEC77AC4
:104B2000D3ED007A4B42A6EEA77A700007EE903ADA
:104B3000F8EEE77AB4EEE77AF1EE10FA0AD407EE6F
:104B4000901AF8EE677AF4EEC77AF1EE10FA88BFA1
:104B5000F0EE477A224B23490344085EB3F90C3048
:104B6000C01A07EE100AB8EEC77AD007E7EE687AE7
:104B700040F100861C4B93ED008A43E01A60002050
:104B800000000000C02700201C60002018600020EA
:104B900050620020932449920D60002058A8002004
:104BA000047D0020B4790020184A00205C590020C0
:104BB0008A7F002098000020747D0020C8790020A2
:104BC0004C5F0020CDCCCC3DAE47813F0000C842B9
:104BD000585F00200C4A00208C290020502900201A
:104BE0006C840020CCA60020F4490020386200200C
:104BF000087D0020CC790020C42800206C450020CE
:104C0000645F002027EE888A069B94F8D8212B4405
:104C1000D3ED01CA38EE6CCA002A3DD0D24BD4F88D
:104C2000DC2108991B688A1A9A4235DD9AF84830C7
:104C3000022B01F0BA87022E04F08583CB4B1B6850
:104C4000990740F12787CA4BCA49DFF890E331F949
:104C500016C09EED008ADFF888E3C7ED00AA03EBDB
:104C6000460028EE288AB0F90C00A0EB0C0007EEF5
:104C7000900AF8EEE77ADEF8000027EE888A904284
:104C800038EE6CCAC1F23281F7EE007AB4EEE79AE0
:104C9000F1EE10FA01F10181B74B2B4493ED000ABC
:104CA000049B2BEE800A022E20EE0C0AA3EC010AD4
:104CB000049304F06283079BDBED007A93ED007AA6
:104CC000AE4BD7ED006A93ED006AAD4B67EE277AE5
:104CD0002B4427EE8B7AD3ED007A67EE277AF0EE3D
:104CE000665AE7EE8C5AB1EE467AB4EEE57AF1EE0A
:104CF00010FA08DCB4EEE56AF1EE10FA8CBFB0EE03
:104D0000657AB0EE467A94ED726AF7EE007AB4EE08
:104D1000E76AF1EE10FAACBF0123002343B1F0EED5
:104D2000E66AF0EEC77AF4EEE67AF1EE10FA01D513
:104D300087ED007A022E04F0F082924A924B52F8EC
:104D400026001B68B0EE6C0A9847904A904B52F8C8
:104D500026001B6898479AF8373023B1059B1B88BB
:104D6000002B00F07185B0EE6A8A8A4B9BED007AC9
:104D700038EE400A2B4493ED008A83ED000A9AF83E
:104D8000483030EE480AC0EE077A2BB3099B1B78F7
:104D9000DB0721D5B7EE007AB4EEC79AF1EE10FA30
:104DA00004DB94F8D831002B00F05F87D4F8DC31B5
:104DB000089AD31A6C4A12689A420DDD764B93ED2D
:104DC000007AB0EECCCAB4EEC7CAF1EE10FA41F1E7
:104DD000A980002384F8D831704B94F8E8212B4443
:104DE00093ED007A2BEE877A67EE277AC9ED007A89
:104DF00032B9049BC7ED00AA43ED01AAC9ED00AA90
:104E00000136032E08F1040809F1040907F104072B
:104E100005F104057FF44AAE614B1B78072B01F0C6
:104E20005283012B01F03A86002794F8F031002BD1
:104E300040F0FA855B4A5C4B10681B6810F4805A9E
:104E400093F82C3040F06886584A594992ED006A30
:104E5000498B584A84ED806A92ED007A564A84ED77
:104E6000817A07EE901AF8EEE76AD2ED037A534A98
:104E700084ED7E6A37EE467A77EEE67AD2ED006A06
:104E800084ED7D7A012284F80822C7EEA65A4C49A7
:104E90004C4A91ED005A4C499FED4C6A91ED004A05
:104EA0004B49DFED4C6AD1ED004A92ED007A35EEC8
:104EB000045AF7EE007AF4EEE75A35EE245AF1EE92
:104EC00010FA88BFF0EE675A25EE065AF4EEE65A5D
:104ED000B1EE476AF1EE10FAB4EEC65AB8BFF0EE82
:104EE000665AF1EE10FAC4ED835A01F1DA80B4EE9D
:104EF000C75AF1EE10FA88BFB0EE475A304ADFEDDC
:104F0000336AD2ED017A304A92ED014A304A77EEA7
:104F1000847AD2ED014A77EEA47A67EEA67AB4EEEF
:104F2000E76AF1EE10FA08DCB4EEE77AF1EE10FA77
:104F30008CBFB0EE676AB0EE476A214ADFED236AA4
:104F4000D2ED027A204AD2ED024A234A77EEA47AC1
:104F500092ED007A67EEA67AB1EE473AF4EEC37AA4
:104F6000F1EE10FA47D43DE0204A0020E8A60020E8
:104F70006C840020CCA60020C84900203C4A0020B8
:104F8000D44900207445002070450020C845002009
:104F9000C4450020A02900202C4A0020E049002020
:104FA000047D0020D87900205C590020C8820020B0
:104FB000F09400203C840020007E00205442002019
:104FC0004C5F0020404A0020585F00206F12833A57
:104FD000645F002000000000444A0020F4490020E3
:104FE0001C4A0020F4EEC77AF1EE10FA8CBFB0EE46
:104FF000473AB0EE673AF04A52780AB9B1EE433A0E
:10500000002B41F08183F7EE003AEC4D2A78002A1C
:1050100002F0B686EA4BDFEDEB6AD3ED024A93ED80
:10502000017AD3ED037A66EE244AE5EE074AE3EE11
:10503000274A63EEA44AF4EEE64AF1EE10FAB4BF52
:10504000B0EE664AB0EE644A98BFF0EE646A012A98
:10505000CDED0C4A02F0B98693ED067AD3ED052A20
:10506000D3ED077A26EE077AA5EE227AA3EE277A09
:1050700023EE877AB4EEE67AF1EE10FAB4EEC47A53
:105080008CBFF0EE667AF0EE477AF1EE10FA98BF38
:10509000F0EE676AB4BFF0EE447AF0EE477A022A87
:1050A0008DED0D7A00F0DE8093ED0A7AD3ED092ABA
:1050B00093ED0B4A26EE077AA5EE227AA3EE047A48
:1050C00023EE877AB4EEE67AF1EE10FAB4EEE77AE0
:1050D0008CBFB0EE664AB0EE474AF1EE10FA98BFC8
:1050E000F0EE446AA8BFF0EE477A032A8DED0E7AFF
:1050F00000F0B88093ED0E7AD3ED0D2A93ED0F4AB0
:1051000026EE077AA5EE227AA3EE047A23EE877ABA
:10511000B4EEE67AF1EE10FAB4EEE77A8CBFB0EEB8
:10512000664AB0EE474AF1EE10FA98BFF0EE446AD4
:10513000A8BFF0EE477A042A8DED0F7A00F0928036
:1051400093ED124AD3ED112A93ED137A26EE044A19
:10515000A5EE224AA3EE074A23EE844AB4EEE64ABD
:10516000F1EE10FAB4EEE74A8CBFB0EE667AB0EE1C
:10517000447AF1EE10FA98BFF0EE476AA8BFF0EE5D
:10518000447A052A8DED104A6CD093ED164AD3ED82
:10519000152A93ED177A26EE044AA5EE224AA3EECD
:1051A000074A23EE844AB4EEE64AF1EE10FAB4EE72
:1051B000E74A8CBFB0EE667AB0EE447AF1EE10FAB0
:1051C00098BFF0EE476AA8BFF0EE447A062A8DED4C
:1051D000114A47D093ED1A4AD3ED192A93ED1B7A61
:1051E00026EE044AA5EE224AA3EE074A23EE844A9D
:1051F000B4EEE64AF1EE10FAB4EEE74A8CBFB0EE38
:10520000667AB0EE447AF1EE10FA98BFF0EE476A93
:10521000A8BFF0EE447A072A8DED124A22D093ED12
:105220001E7AD3ED1D2A93ED1F4A26EE077AA5EECE
:10523000227AA4EE037A27EE237AB4EEE67AF1EE30
:1052400010FAB4EEE77A8CBFB0EE666AB0EE476A49
:10525000F1EE10FA8DED137A98BFF0EE466AA8BF12
:10526000F0EE477A77EEE67AF7EE006AF4EEE67A49
:10527000F1EE10FAC4ED727A43F3878586EEA77AD1
:10528000022ADDED0D7A67EE244A67EE877ACDEDCE
:105290000C4ACDED0D7A2DD0DDED0E7A67EE877AD2
:1052A000032ACDED0E7A25D0DDED0F7A67EE877AF1
:1052B000042ACDED0F7A1DD0DDED107A67EE877AE6
:1052C000052ACDED107A15D0DDED117A67EE877ADB
:1052D000062ACDED117A0DD0DDED127A67EE877AD0
:1052E000072ACDED127A05D0DDED137A27EE877A05
:1052F0008DED137A344B1E6816F0805601F0AA80AB
:10530000F6EE005AC4ED835A002A02F011852F4BA5
:10531000D4ED814A93F8038094F908320999D4EDC9
:10532000806A91F800E0DFF8B0C02949DFF8AC905E
:10533000B1F906109CED007A049106EE103AFDEEEC
:10534000E44A244B99F80090B3F81AB094ED7D5AD2
:10535000D4ED7E7A14EE903AFDEEE64A00F0100CA1
:1053600000F480000EF0010EB8EEC66A14EE901A3A
:105370000590B8F1000F41F00982DFF84480BCF1DC
:10538000000F41F0B58098ED007ADDED0C6ADFF892
:1053900050C025EE877AA6EE267AF0EE676AE5EE33
:1053A000076ABDEEE67A17EE106A17EE100A9E4203
:1053B000A8BF184616E000BFAC5F0020E57C0020C7
:1053C000C44100200000000020840020947F0020C1
:1053D000607F0020F0940020A0410020A8760020EB
:1053E000805F0020B142C8BF084607EE100AB8EE41
:1053F000C77A012A8CED007A00F0DC8098ED047AFF
:10540000DDED0D6A25EE877AA6EE267AF0EE676A64
:10541000E5EE076ABDEEE67A17EE106A17EE100A9F
:105420009E42A8BF1846B142C8BF084607EE100A00
:10543000B8EEC77A022A8CED017A00F0BB8098EDB5
:10544000087ADDED0E6A25EE877AA6EE267AF0EE72
:10545000676AE5EE076ABDEEE67A17EE106A17EEA8
:10546000100A9E42A8BF1846B142C8BF084607EEC0
:10547000100AB8EEC77A032A8CED027A00F09A80FF
:1054800098ED0C7ADDED0F6A25EE877AA6EE267A86
:10549000F0EE676AE5EE076ABDEEE67A17EE106A8F
:1054A00017EE100A9E42A8BF1846B142C8BF084670
:1054B00007EE100AB8EEC77A042A8CED037A79D089
:1054C00098ED107ADDED106A25EE877AA6EE267A41
:1054D000F0EE676AE5EE076ABDEEE67A17EE106A4F
:1054E00017EE100A9E42A8BF1846B142C8BF084630
:1054F00007EE100AB8EEC77A052A8CED047A59D067
:1055000098ED147ADDED116A25EE877AA6EE267AFB
:10551000F0EE676AE7EE056ABDEEE67A17EE106A0E
:1055200017EE100A9E42A8BF1846B142C8BF0846EF
:1055300007EE100AB8EEC77A062A8CED057A39D044
:1055400098ED187ADDED126A25EE877AA6EE867A56
:10555000F0EE676AE7EE056ABDEEE67A17EE106ACE
:1055600017EE100A9E42A8BF1846B142C8BF0846AF
:1055700007EE100AB8EEC77A072A8CED067A19D022
:1055800098ED1C7ADDED136A65EE875AE6EE265A31
:10559000E5EE257AFDEEE77A17EE900A8342A8BF82
:1055A00003468142C8BF0B4607EE903AF8EEE77A11
:1055B000CCED077ABEF1000F40F04382002A40F0A4
:1055C0003B823EE2AE4B1B78013BDBB2FFF730BAC9
:1055D000AC4B06934FF47A761B68B6FBF3F3C3EB40
:1055E0004316A949DFF8CC8291F801A0A749B8F980
:1055F000060091F8009003EB8603DE00B6B2B742D6
:1056000002F0FD80D5F88810B5F93CE0EB6E4A1C3D
:1056100007EE90EA7344012AC5F88820EB66F8EE9D
:10562000E77A02F0F780D5ED1E5AD5ED206A07EE35
:10563000102A37EEE56AB8EEC75A012F86EE057AD2
:1056400037EE257A77EEC77A85ED1F7AE7EE866A20
:1056500085ED1E7AF0EE667AC5ED216AC5ED206A09
:1056600002F0D384D5F89C10B5F93EE02B6F4A1CAC
:1056700007EE90EA7344012AC5F89C202B67F8EEE8
:10568000E77A02F0E080D5ED235AD5ED256A07EEE2
:10569000102A37EEE56AB8EEC75A012F86EE057A72
:1056A00037EE257A77EEC77A85ED247AE7EE866ABB
:1056B00085ED237AF0EE667AC5ED266AC5ED256A9A
:1056C00002F0D884D5F8B010B5F940E06B6F4A1CF1
:1056D00007EE90EA7344012AC5F8B0206B67F8EE34
:1056E000E77A02F0C980D5ED285AD5ED2A6A07EE8F
:1056F000102A37EEE56AB8EEC75A012F86EE057A12
:1057000037EE257A77EEC77A85ED297AE6EE276AB5
:1057100085ED287AF0EE667AC5ED2B6AC5ED2A6A2A
:1057200002F09C84A8F80600B5F8B430574A013B53
:1057300092F80090A5F8B43006990023B9F1070F4C
:105740004B608B60CB607FF468A9F6F7A3FF049BE6
:10575000DFF86081C01A94F8C031A8F80000002B6F
:105760003FF460A9013B84F8C03115B0BDEC0A8B51
:10577000BDE8F08F94ED5E7AB1F90000D4ED5F6A78
:10578000B1F902E0424AF4EEC76A80EAE0738EEAB9
:10579000EE71A3EBE073F1EE10FAA1EBEE71B4BF82
:1057A000B0EE476AB0EE666A8B42B8BF0B4607EEB2
:1057B000103A1378B8EEC77A27EE287A002B40F01B
:1057C0002582344BD3ED005AF4EECA5AF1EE10FAAA
:1057D00041F1F880B7EE005A75EE654ADFED2E6AAA
:1057E0009FED2E5A2E4B36EEC77A24EE855AD3ED16
:1057F000006AE7EE055A65EEA65AF5EEC05AF1EEDC
:1058000010FA40F22386C9EEA56AB7EE007AF0EEF0
:10581000475AE6EE665AF0EE656AF4EEC76AF1EEB4
:1058200010FA88BFF0EE476AF5EEC06AF1EE10FAA2
:10583000B8BFF0EE6A6A1B4B93ED007A67EE877A89
:10584000A7EEA68AFFF7E0B9174B184A2B4493ED51
:10585000007AD2ED007A164B67EE277AF7EE006AEF
:10586000F4EEE67AF1EE10FA93ED007A88BFF0EEEE
:10587000667A67EE877A27EE888AFFF776BA00BFE6
:1058800060840020C8790020B4790020047D0020C5
:10589000004A0020084A002000003443610BB63B58
:1058A000FC490020F849002038290020F049002058
:1058B000EC490020087D0020072B02F081820026A1
:1058C000DFF83CB3B64DDBF800305F0501F17F80B7
:1058D000B44B1B78002B40F0F381DFF80C9394F865
:1058E000127127B1B04B1B88980742F0348094F8AE
:1058F0001821002A41F0758099F81E70002F00F0E1
:10590000F383022F02F02080032F01F0D082A74BF7
:10591000598899F81F300233DBB2002A02F0088060
:10592000002902F00580A2480768B1FBF7F10FB229
:10593000A4F84871002B03F0308207EE907AF8EE5D
:10594000E77AF7EE006A86EEA77A9A49012BD4ED42
:10595000576AD1ED007A77EEE67A67EE877AC4ED82
:10596000537A21D0D1ED017AD4ED586A77EEE67AF8
:10597000022B67EE877AC4ED547A15D0D1ED027A06
:10598000D4ED596A77EEE67A032B67EE877AC4ED99
:10599000557A09D0D1ED037AD4ED5A6A77EEE67ADA
:1059A00067EE877AC4ED567A83480078092803F0B9
:1059B000A082002F40F39E8393B394ED577AD4EDE9
:1059C000537A77EE877A012BC4ED577AC1ED007ACE
:1059D00021D094ED587AD4ED547A77EE877A022B61
:1059E000C4ED587AC1ED017A15D094ED597AD4ED11
:1059F000557A77EE877A032BC4ED597AC1ED027A96
:105A000009D0D4ED5A7A94ED567A77EE877AC4EDC0
:105A10005A7AC1ED037A013B022BB8BF0223DBB2F5
:105A2000002A18BF022366E3099B644D1B78DE073A
:105A300000F164812A7822B192006149614825F021
:105A400099FD614B1B68002B40F02F835F4B1B7847
:105A50009BB1287870B1DFF86C81DFF8A89100263F
:105A6000F0B2D9F80030B8EC010A9847287801362E
:105A70008642F5DB564B1B6898474F4B1B78072B2C
:105A800000F01A85012384F8003115B0BDEC0A8BB3
:105A9000BDE8F08F4F4BC7ED00AA1B689342BFF6DD
:105AA000F3A84D4B1A88002384F8D831002A41F01E
:105AB0009C864A4A4A4B1178186881F00101F7F731
:105AC000A1FCFFF7E9B8474FDFF83C9107F24C76AD
:105AD00007F5F768F7EC017A95ED080AD5F87837FD
:105AE000F8EEE77A304627EE800A9847A6F1E00004
:105AF000D5F898369847A6F17000D5F8083798473A
:105B0000D7F85806D5F8B83098472436B045A9ECF0
:105B1000010ADFD1FEF77ABF099A1278D50703D4BC
:105B2000314A128BA4F8FC21304A2249128891EDA7
:105B3000037A07EE902AF8EEE77AB4EEE77AF1EE10
:105B400010FA41F296802A49098807EE901AF8EE79
:105B5000E77AB4EEE77AF1EE10FAC0F2FC87254955
:105B6000254AD1ED006A92ED006A2449C4ED806AAD
:105B7000BCEEC75A76EE665A15EE102AC4ED7E6A60
:105B8000C4ED7D5A84ED816AA4F8FC210122D1ED97
:105B9000006A84F8082277EE677AFFF776B900BFCB
:105BA00028A80020480100208A7F00207CA2002035
:105BB000A45F0020007E0020047D0020E57C002002
:105BC000A4410020805F002068450020B0790020BB
:105BD000A47600201C4A0020387C00203A7C00205B
:105BE0003C7C002058A80020F0940020584200205F
:105BF0005A420020444200203C84002060420020A1
:105C0000D87900209C760020CC790020CD4B93EDF4
:105C1000005AB5EEC05AF1EE10FA40F31784CA4BA1
:105C2000D3ED006AF5EEC06AF1EE10FA40F30E848F
:105C300036EEC77A66EE695A87EE266AC5EE856A41
:105C4000B7EE007AB4EEC76AF1EE10FA88BFB0EE94
:105C5000476AB5EEC06AF1EE10FA76EE876AB8BF11
:105C6000B0EE6A6A66EE266AD7E5B84A92ED007A27
:105C7000F0EEE76AF4EEC76AF1EE10FA7FF796A845
:105C8000B34A92ED007AF0EECC6AF4EEC76AF1EE18
:105C900010FA7FF78BA8AF4A98ED007AD2ED006A30
:105CA000B0EEC77AB4EEE67AF1EE10FA7FF57EA890
:105CB00001220899C4F8DC1184F8D821FFF77AB8DA
:105CC000A54BDFF8B892B3F90620B9F81A309A421A
:105CD0003FF705AEA14B1B78012B01F01486192B61
:105CE00001F011860E2B3FF4FAAD082B3FF4F7AD0F
:105CF0009B4900238B60C4F80C31F0E52B78002B16
:105D00003FF49FAED4ED5F3A94ED5E6AD4ED7E7AB7
:105D1000944A94ED7D7AD2ED005A94ED5C4AD4ED2C
:105D20005B4ADFF85C82DFF85CC2F4EEC63AF3EE61
:105D3000046AF1EE10FA37EEA65A01F1098098EDE7
:105D4000026A26EE446AF0EE674AE6EE074AF4EE8F
:105D5000C54A34EEE66AF1EE10FA48BFB0EE656A65
:105D6000012B8CED006A3FF46CAE98ED066A26EECE
:105D7000446AF0EE674AE6EE074AB4EEE45A34EEBF
:105D8000E66AF1EE10FA88BFB0EE656A022B8CED80
:105D9000016A3FF456AE98ED0A6A26EE446AF0EEC8
:105DA000674AE6EE074AF4EEC54A34EEE66AF1EEDB
:105DB00010FA48BFB0EE656A032B8CED026A3FF41F
:105DC00040AE98ED0E6A26EE446AF0EE674AE6EEC3
:105DD000074AB4EEE45A34EEE66AF1EE10FAC8BFB0
:105DE000B0EE656A042B8CED036A3FF42AAE98EDA1
:105DF000126A26EE446AF0EE674AE6EE074AB4EE0F
:105E0000E45A34EEE66AF1EE10FAC8BFB0EE656A05
:105E1000052B8CED046A3FF414AE98ED166A26EE5D
:105E2000446AF0EE674AE6EE074AF4EEC54A74EEBD
:105E3000E66AF1EE10FAB8BFF0EE656A062BCCED1B
:105E4000056A3FF4FEADD8ED1A6A66EEC46AF0EE5C
:105E5000674AE6EE874AB3EE046AB4EEE45A74EE9B
:105E6000C66AF1EE10FAC8BFF0EE656A072BCCEDFA
:105E7000066A3FF4E6ADD8ED1E6A26EEC44AE4EEAB
:105E8000077AB4EEE75A77EEC67AF1EE10FAC8BF99
:105E9000F0EE657ACCED077AD3E50699324BD1ED79
:105EA000017A93ED007AF0EEE77AF4EEC77AF1EE3C
:105EB00010FA7EF5F1AED1ED027AF0EEE77AB4EEAB
:105EC000E77AF1EE10FA7EF7E7AED1ED037AF0EE65
:105ED000E77AB4EEE77AF1EE10FA7EF7DDAE234B07
:105EE0001B689A077FF5DDAD2149224BB3F90C20E1
:105EF000B1F900E02048AEEB020E00688EEAEE72C7
:105F0000A2EBEE728242BEF6C7AEB3F90E30B1F923
:105F10000220D21A82EAE273A3EBE27398427EF780
:105F2000BBAEBEE50B4B98ED007AD3ED006AB0EE48
:105F3000C77AB4EEE67AF1EE10FA7EF74DAFFEF7CF
:105F400048BF00BFFC490020044A0020304A00201E
:105F50002C4A0020344A0020607F0020AC5F0020E3
:105F6000007E0020A0410020284A0020E8A6002052
:105F7000CCA600206C840020244A0020F09400204D
:105F8000C4410020805F002007EE103A524BDFF83A
:105F900054811B78C4F8A871B8EEC77AF7EE006A8E
:105FA000132B86EE879AB8F90400B4F8AC7195ED1E
:105FB000080A01F0A583494B494A93ED001A93ED75
:105FC000053A93ED122A93ED176AD3ED091A93ED72
:105FD0000E4AD3ED015AD3ED063A93ED0A7A93EDCA
:105FE0000F5AD3ED132AD3ED186AD3ED044AD3ED3B
:105FF000030A67EE897A69EE288A29EE088AA1EEFB
:10600000273A02EB87060021A2EE286AC4F89C1109
:10601000C4F8A011A1EE884AE5EEA73AA7EE085A07
:1060200093ED167AD3ED0D5A93ED021AD3ED0C1AB7
:1060300086ED003AE2EEA86A64EEC34A27EE467A9D
:1060400093ED0B2AD3ED152A86ED204AE0EEC33AF4
:1060500065EEC45A93ED143AC3ED053AE1EE274AD2
:10606000F0EE477AA1EEC45AE2EE085AE2EEC66AB2
:10607000E3EE287AC3ED064A83ED0E5AC3ED0F5ABC
:1060800086ED406AC3ED176AC3ED187AC4F8A4110F
:106090007B1C03F01F03A4F8AC31A8F80400FEF742
:1060A00097BBB0EE465AFEF729BF0EF0A9F9CDE432
:1060B00025F06AFC2AF81700FEF798BC96ED007AE6
:1060C00005EB4702B8EEC78A928F2AF8172028EE10
:1060D000278AFEF769BC00BF047D0020BC62002057
:1060E00038600020087D0020A4F84871002A00F0E4
:1060F0007281DB490223DB4ADFEDDB6A1068DB4A91
:1061000090F802E092F800C0027807EE902AF8EECC
:10611000E77AB0EE007A67EEA67AF4EEC77AF1EE8F
:1061200010FA40F3228337EEC77ADFEDD16AB0EE82
:10613000676AA7EE266AB0EE467A9FEDCE6AD1ED89
:10614000006A66EE866AB0EEE66AC4ED5B6A84EDCC
:106150005E6ABEF1000F13D005EE90EAB8EEE55A84
:10616000DFEDC15A66EEA64A25EE255AF7EE005A33
:1061700075EEC55A64EE864AE4EE855A66EEA56A67
:10618000DFEDBD5A427927EE257A27EE267ACAB18D
:10619000DFEDB56ADFEDB95A26EE266A06EE902AE3
:1061A000F8EEE66A26EE266AB4EEE56AF1EE10FA3B
:1061B00000F38685F7EE005A35EEC66AC5EE866AAC
:1061C00027EE267ABCF10C0F9FEDAD8ADFEDAD6AAC
:1061D00000F02785B4EEC87AF1EE10FA98BFB0EE61
:1061E000478AB4EEE68AF1EE10FAB8BFB0EE668ADE
:1061F00084ED418A002B00F0E280B0EE007AF4EEEC
:10620000C77AF1EE10FA05DD37EEC77ADFED986A4E
:10621000E7EE267A91ED017ADFED966A27EE267A8F
:10622000B0EEC76A84ED5C7A84ED5F6ABEF1000F60
:1062300013D006EE90EADFED8C5AF8EEE66A27EE10
:10624000075A66EEA56AF7EE005A75EEE65A25EE95
:10625000065AE5EE265A27EE257ADFED876A82791F
:1062600067EEA67A67EE877AAAB107EE102AB8EE33
:10627000C77ADFED7D5ADFED816A27EE067A27EED9
:10628000257AB4EEE67AF1EE10FA40F31D85DFEDE3
:106290007E6A67EEA67ABCF10C0F00F0A184DFEDF8
:1062A000786A9FED787AF4EEE67AF1EE10FA88BF1C
:1062B000F0EE667AF4EEC77AF1EE10FAB8BFF0EEBF
:1062C000477A012BC4ED427A79DD4378DFED666AC7
:1062D00007EE903AF8EEE77AB0EE007A67EEA67A2B
:1062E000437AF4EEC77AF1EE10FA05DD37EEC77A9D
:1062F000DFED5F6AE7EE267A91ED027ADFED5D6A07
:1063000027EE267AB0EEC76A84ED5D7A84ED606A86
:106310009BB106EE903ADFED545AF8EEE66A27EEAE
:10632000075A66EEA56AF7EE005A75EEE65A25EEB4
:10633000065AE6EE855A27EE257ADFED4F6AC379D5
:1063400067EEA67A67EE877A0BB307EE103AB8EEDF
:10635000C77ADFED455ADFED496A27EE067A27EE68
:10636000257AB4EEE67AF1EE10FA0CDCB5EEC07ADE
:10637000F1EE10FA01F1D282B7EE006A36EE477AFA
:10638000C6EE076A01E0DFED406A67EEA67ABCF16F
:106390000C0F00F01B84DFED3A6A9FED3A7AF4EEC1
:1063A000E67AF1EE10FA88BFF0EE667AF4EEC77A7C
:1063B000F1EE10FAB8BFF0EE477AC4ED437ABCF1C3
:1063C000090F00F0E78399F82170002F40F07E83D9
:1063D000002384F818312D4B1B68990609D52C4BE6
:1063E0001B8803F0300323B12A4B1B78DA0701F135
:1063F000BA87294B1B7823B9284FBB78002B41F073
:10640000E7821A4B1B78072B00F028840022072B09
:1064100084F800217EF489A9F6F73CF90490FEF790
:1064200086B91F4B1F4C1A681F4BDFF8888094F801
:106430000001D2691B88A8F80020A8F802300028C3
:106440007FF43DAA0490194DFEF771B9DFED186A8B
:10645000FFF7F1B941023EF553AFFEF755BF00BF5C
:10646000007E00201C4B00200AD7233C047D002026
:10647000D7A368416F12033B00004843A4707D3FDF
:1064800000C0F94400C0F9C40000C842E8A60020DA
:106490008A7F0020ECA600202F680020AA5A002046
:1064A00010820020C0270020EA3E002028A80020FB
:1064B00000000000087D0020F6F7ECF8AC4BC01B94
:1064C000D880FFF7DFBAF6F7E5F8AA4B0B9A1B78EE
:1064D000DFF89C82801A012BA8F8020000F0E0820D
:1064E000072B7EF4A1ACF6F7D5F80746FEF79DBC66
:1064F000BEF1000F41F07B8498ED007ADDED0C6A6F
:10650000DFF884C225EE877AA6EE867AF0EE676A17
:10651000E7EE056ABDEEE67A17EE106A17EE100A8E
:106520009E42A8BF1846B142C8BF084607EE100AEF
:10653000B8EEC77A012A8CED007A3FF47DAA98ED77
:10654000047ADDED0D6A25EE877AA6EE867AF0EE06
:10655000676AE7EE056ABDEEE67A17EE106A17EE97
:10656000100A9E42A8BF1846B142C8BF084607EEAF
:10657000100AB8EEC77A022A8CED017A3FF45CAAC1
:1065800098ED087ADDED0E6A25EE877AA6EE867A1A
:10659000F0EE676AE7EE056ABDEEE67A17EE106A7E
:1065A00017EE100A9E42A8BF1846B142C8BF08465F
:1065B00007EE100AB8EEC77A032A8CED027A3FF490
:1065C0003BAA98ED0C7ADDED0F6A25EE877AA6EEF0
:1065D000867AF0EE676AE7EE056ABDEEE67A17EEB8
:1065E000106A17EE100A9E42A8BF1846B142C8BFF3
:1065F000084607EE100AB8EEC77A042A8CED037A33
:106600003FF41AAA98ED107ADDED106A25EE877A2C
:10661000A6EE867AF0EE676AE7EE056ABDEEE67AE8
:1066200017EE106A17EE100A9E42A8BF1846B14234
:10663000C8BF084607EE100AB8EEC77A052A8CEDE7
:10664000047A3FF4F9A998ED147ADDED116A25EE8C
:10665000877AA6EE867AF0EE676AE7EE056ABDEE07
:10666000E67A17EE106A17EE100A9E42A8BF184687
:10667000B142C8BF084607EE100AB8EEC77A062A2C
:106680008CED057A3FF4D8A998ED187ADDED126A01
:1066900025EE877AA6EE867AF0EE676AE7EE056A5F
:1066A000BDEEE67A17EE106A17EE100A9E42A8BFFA
:1066B0001846B142C8BF084607EE100AB8EEC77ABE
:1066C000072A8CED067A3FF4B7A998ED1C7ADDED28
:1066D000136A65EE875AE6EE265AE5EE257AFDEE58
:1066E000E77A17EE900A8342A8BF03468142C8BFEB
:1066F0000B4607EE903AF8EEE77ACCED077A002ADF
:106700007FF49AA9FFF79DB91B4B5A79002A3EF4F2
:106710007AAC1A4A1278002A3EF475AC1B78DFED89
:10672000184A07EE903A174BB8EE677A1B8807EEC7
:10673000902A06EE903AF8EEE77AF8EE666A67EE8F
:10674000277AB7EE007AC7EEA63AF4EEE43AF1EE15
:1067500010FA88BFF0EE643AF4EEC73AF1EE10FAA0
:10676000B8BFF0EE473AFEF750BCB0EE677AE4E40B
:10677000087D0020047D0020D4A60020FE7D00209E
:10678000713DAA3FE87D0020805F0020BCF1000F32
:1067900000F09783BEF1000F42F04780DFF8A0853C
:1067A000B9F1000F41F09286D8ED006ADDED0C4A98
:1067B000DFF890C565EEA66ABDEEC77A17EE101A2F
:1067C000B0EE667AA4EE867AF0EE676AE7EE056AC6
:1067D000BDEEE67A17EE106A17EE100A9E42A8BFC9
:1067E0001846B142C8BF084607EE100AB8EEC77A8D
:1067F000012A8CED007A3FF41FA998ED047ADDEDB3
:106800000D6A25EE877AA6EE867AF0EE676AE7EEE5
:10681000056ABDEEE67A17EE106A17EE100A9E4280
:10682000A8BF18468E42B8BF084607EE100AB8EE59
:10683000C77A022A8CED017A3FF4FEA898ED087A17
:10684000DDED0E6A25EE877AA6EE867AF0EE676AAF
:10685000E7EE056ABDEEE67A17EE106A17EE100A4B
:106860009E42A8BF18468E42B8BF084607EE100ADF
:10687000B8EEC77A032A8CED027A3FF4DDA898EDD2
:106880000C7ADDED0F6A25EE877AA6EE867AF0EEB9
:10689000676AE7EE056ABDEEE67A17EE106A17EE54
:1068A000100A9E42A8BF18468E42B8BF084607EE9F
:1068B000100AB8EEC77A042A8CED037A3FF4BCA81C
:1068C00098ED107ADDED106A25EE877AA6EE867ACD
:1068D000F0EE676AE7EE056ABDEEE67A17EE106A3B
:1068E00017EE100A9E42A8BF18468E42B8BF08464F
:1068F00007EE100AB8EEC77A052A8CED047A3FF449
:106900009BA898ED147ADDED116A25EE877AA6EE44
:10691000867AF0EE676AE7EE056ABDEEE67A17EE74
:10692000106A17EE100A9E42A8BF18468E42B8BFE2
:10693000084607EE100AB8EEC77A062A8CED057AEB
:106940003FF47AA898ED187ADDED126A25EE877A81
:10695000A6EE867AF0EE676AE7EE056ABDEEE67AA5
:1069600017EE106A17EE100A9E42A8BF18468E4214
:10697000B8BF084607EE100AB8EEC77A072A8CEDB2
:10698000067A3FF459A898ED1C7ADDED136A65EE9E
:10699000875AE6EE265AE5EE257AFDEEE77A17EEFF
:1069A000900A8342A8BF03468142D8BF194607EE2A
:1069B000901AF8EEE77ACCED077A002A7FF43CA82B
:1069C000FFF73FB8C74BD3ED005AFEF716BFAB68D1
:1069D000002B3EF47DAF05F1500128469847FEF7A5
:1069E00077BFC14BC149D3F8EC30096844F6206049
:1069F0008342A8BF0346B3F57A7FB8BF4FF47A73DA
:106A000098B2C906A4F81A01DBF8003041F1F88207
:106A1000DB0400F16B83B64BD3F800E0BEF93270B3
:106A2000B449DFF824C3D1ED037AD4F81C31ACFBB0
:106A300000108009642191FBF0F11429BDEEE77A82
:106A400004EB430CA8BF142101338B42C4F81C3162
:106A500017EE108AA4BF0023C4F81C3104EB4303D3
:106A6000ACF82081B3F9203107EE103AB8EEC77ABE
:106A700077EEC77AFDEEE77ACDED047ABDF9101016
:106A800081EAE173A3EBE173BB4202F36F819A4B9E
:106A900019464FF07E530B60FEF72EBFDFF8AC8235
:106AA000F5F7F8FD954AD4F8EC311268C4F8EC011A
:106AB000C31A9A1A0746A8F80430A8F80620FEF769
:106AC000B4B9F5F7E7FD0B90FDF7BBBF1E21874872
:106AD000F2F7CCFC00283FF47BAC894B1B885806AE
:106AE0003FF576AC94F88431BB4242F08B81824B07
:106AF000D4ED627AD3ED016A94ED435ADFED815A09
:106B00009FED816A27EEC57A68EE277AA8EE267A8D
:106B1000E5EE267AB4EEE57AF1EE10FA88BFB0EE33
:106B2000657AB4EEC67AF1EE10FAF4EEE57AB8BF03
:106B3000B0EE467AF1EE10FA88BFF0EE657AF4EE28
:106B4000C67AF1EE10FAB8BFF0EE467A84ED417ADB
:106B5000C4ED437A3CE4B4F8FC11914240F28185E3
:106B60006A496B4AD1ED007A92ED007A6949C4ED29
:106B7000807A77EE676AC4ED7E7A0122C4ED7D6A81
:106B800084ED817AD1ED006ADFED637A84F8082222
:106B9000FEF77BB9FDEEC87ADFF8B08117EE903AC8
:106BA000A8F80470A8F806300DE45C4B1B88002B95
:106BB00040F076855A4A5B4B11781868F6F722FC4C
:106BC000D4F8DC21089B9A1AFEF735B8BDEEE77AB7
:106BD000DFF8788117EE103AA8F80430FFF7DBBB36
:106BE0009FED487ADFED486ADFF86081F4EEC77AFE
:106BF000F1EE10FA98BFB0EE677AFDEEE77AB4EEE8
:106C0000E67AF1EE10FA17EE902AB8BFB0EE667A87
:106C1000012B84ED427AA8F802203FF756ABFFF72C
:106C2000D2BBB4EEC87AF1EE10FA98BFB0EE478A44
:106C3000BDEEC77AB4EEE68ADFF81081F1EE10FA05
:106C400017EE102AB8BFB0EE668A84ED418AA8F824
:106C50000020002B7FF4D1AAFFF7B5BBF5F71AFD92
:106C6000DFF8E880304B801B1B78A8F80400FFF7A2
:106C7000CDBB2E4A2E49D2ED006A2E4A91ED006A14
:106C80001278C4ED806A84ED816A002A40F0E584C0
:106C900076EEC65AF0EE466ABCEEC76A2649C4EDE7
:106CA0007D5A16EE102AC4ED7E6AA4F8FC21FF225C
:106CB000D1ED006A84F8082277EEC77AFEF7E5B8CE
:106CC000DFED1E6AFFF77CBAB5EEC07AF1EE10FA7E
:106CD00000F12086B7EE006A36EE477AC6EE076A04
:106CE000FFF7D7BAFC4900201C1E0020208400209A
:106CF0005C590020007E002098000020A45F002046
:106D00008A7F002000C0F94400C0F9C4444200203A
:106D10003C8400206042002000000000387C0020FD
:106D20003A7C00203C7C0020047D0020C8820020AA
:106D300048420020A87600205C4200200000C842A3
:106D4000C4410020805F0020D34D6210087D0020E8
:106D500098ED016A26EE646AB0EE674AA6EE074A2D
:106D6000B4EEC45A34EE666AF1EE10FAC8BFB0EE63
:106D7000656A012B8CED006A3EF463AE98ED056AFE
:106D800026EE646AB0EE674AA6EE074AB4EEC45A2D
:106D900034EE666AF1EE10FAC8BFB0EE656A022BF7
:106DA0008CED016A3EF44DAE98ED096A26EE646AF8
:106DB000B0EE674AA6EE074AB4EEC45A34EE666AED
:106DC000F1EE10FAC8BFB0EE656A032B8CED026AD3
:106DD0003EF437AE98ED0D6A26EE646AB0EE674A6F
:106DE000A6EE074AB4EEC45A34EE666AF1EE10FA23
:106DF000C8BFB0EE656A042B8CED036A3EF421AE89
:106E000098ED116A26EE646AB0EE674AA6EE074A6C
:106E1000B4EEC45A34EE666AF1EE10FAC8BFB0EEB2
:106E2000656A052B8CED046A3EF40BAE98ED156A8D
:106E300026EE646AB0EE674AA6EE074AB4EEC45A7C
:106E400074EE666AF1EE10FAC8BFF0EE656A062BC2
:106E5000CCED056A3EF4F5ADD8ED196A66EEE46A4C
:106E6000B0EE674AA6EE874AB3EE046AB4EEC45A9F
:106E700074EE466AF1EE10FAC8BFF0EE656A072BB1
:106E8000CCED066A3EF4DDADD8ED1D6A66EEE44A4F
:106E9000E4EE877AF4EEC57A77EEC67AF1EE10FA70
:106EA000B8BFF0EE657ACCED077AFEF7CABD99F867
:106EB0002030C3EB431103EB8101C90089B2FEF717
:106EC00028BDDFF8DC84B9F1000F41F00D81D8ED69
:106ED000006ADDED0C4ADFF8CCC465EEA66ABDEEB3
:106EE000C77A17EE101AB0EE667AA4EE867AF0EE44
:106EF000676AE7EE056ABDEEE67A17EE106A17EEEE
:106F0000100A9E42A8BF1846B142C8BF084607EE05
:106F1000100AB8EEC77A012A8CED007A3EF44AAB2B
:106F200098ED047ADDED0D6A25EE877AA6EE867A75
:106F3000F0EE676AE7EE056ABDEEE67A17EE106AD4
:106F400017EE100A9E42A8BF18468E42B8BF0846E8
:106F500007EE100AB8EEC77A022A8CED017A3EF4E9
:106F600029AB98ED087ADDED0E6A25EE877AA6EE5C
:106F7000867AF0EE676AE7EE056ABDEEE67A17EE0E
:106F8000106A17EE100A9E42A8BF18468E42B8BF7C
:106F9000084607EE100AB8EEC77A032A8CED027A8B
:106FA0003EF408AB98ED0C7ADDED0F6A25EE877A9A
:106FB000A6EE867AF0EE676AE7EE056ABDEEE67A3F
:106FC00017EE106A17EE100A9E42A8BF18468E42AE
:106FD000B8BF084607EE100AB8EEC77A042A8CED4F
:106FE000037A3EF4E7AA98ED107ADDED106A25EEFB
:106FF000877AA6EE867AF0EE676AE7EE056ABDEE5E
:10700000E67A17EE106A17EE100A9E42A8BF1846DD
:107010008E42B8BF084607EE100AB8EEC77A052AB6
:107020008CED047A3EF4C6AA98ED147ADDED116A6F
